:100000000C94820E0C94AA0E0C94AA0E0C94AA0EB8
:100010000C94AA0E0C94AA0E0C94AA0E0C94AA0E80
:100020000C94AA0E0C94AA0E0C94AA0E0C940B67B6
:100030000C94A16A0C9438670C94AA0E0C942418A2
:100040000C9412180C94AA0E0C94726F0C94AA0EB5
:100050000C94AA0E0C94AA0E0C94AA0E0C94AA0E40
:100060000C94616A0C9480180C94A3670C947068CB
:100070000C94AA0E0C94AA0E0C94AA0E0C94AA0E20
:100080000C94AA0E0C94AA0E0C94AA0E616C656CCA
:100090006D6C776C8E6CA86CBD6CCC6CE16CF86C84
:1000A000026D206D266D2B6D316D376D916D9B6DE1
:1000B000406D466D4C6D556D596D5E6D666D786D1C
:1000C0007E6D846D896D696C696D6E6D736D537035
:1000D0006C617368008040000000000000000000B8
:1000E0000000000000000000000000000000000010
:1000F0000000000000000000000000000000000000
:1001000000000000000000000000000000000000EF
:1001100000000000000000000000000000000000DF
:10012000000080C0E0E0F0F8F8FCFCFCF8F8F8F023
:1001300040000000000080808000000000000000FF
:1001400000000000000000000000000080C0C0E0CF
:10015000E0E0F0F0F0E0C00000000000C0F8FFFFB9
:100160009F8783838383838383838383838383833F
:1001700083838383838383830383808383838383D2
:10018000838383838383838383838383838383833F
:100190008383C3E3733F1F0000000080E0F0F8FC9E
:1001A000FEFFFFFFFF7F3F1F1F0F0783C3E1E1E05B
:1001B000E0C0000E1F3F7F7FFFF3E0E08000000003
:1001C0000000000000000080F0FCFEFFFFFFFF7F4A
:1001D0003F0F0301010100000080F0FEFFFFC7C1D7
:1001E000C1C1C1C1C1C1C1C1C1C1C1C1C1C1C1C1FF
:1001F000C1C1C1C1C101C1F0FEFF3F0F070F0D0D0D
:100200000D1D191919193131313171616161E1C166
:10021000C1C18100000080E0F8FCFFFFFFFF2F1745
:100220000F038180C0E0F0F8FCFEFFFFFFFFFFFF3F
:100230007F010000000000000001010307070E1EFF
:100240001C3870E0F0F8FEFFFF7F1F0F0300010075
:10025000000000000000000000000000000000009E
:10026000000000000000000000000000000000008E
:10027000000000000000000000000000000000007E
:10028000000000000000000000000000000000006E
:1002900000000000007EFFFFFFFFFFFFFBF8FCFCFB
:1002A000FEFF7F3F1F0F07C3FFFFFFFFFFFF7F071B
:1002B0000000000000000000000000000000C0E09E
:1002C000F8FEFFFF7F1F0F1F3D7CF8F8F0E0800075
:1002D000000000000000000000000000000000001E
:1002E000000000000000000000000000000000000E
:1002F00000000000000000000000000000000000FE
:1003000000000000000000000000000000000000ED
:1003100000000000000000010101010103070707C0
:100320000301000000E0FCFFFFFFFFFF1F030000D0
:10033000000000000000000000C0F078DE27130974
:100340000E0703000000000000000001030F7FFF04
:10035000FC7878F800000000000000000000008039
:10036000808080808080808000808000808000008D
:1003700000000000008080808080808080808080FD
:1003800080808080808080000000000000000000ED
:10039000000000000000000000000000000000005D
:1003A000000080F0FEFFFFFFFF3F0F010000000094
:1003B00000000000C0E0381E0F0300010000000034
:1003C000000000000000000000000000000000002D
:1003D0000000030301000000000000000000000E08
:1003E0000E02020202020303000F0F000F0F0808A3
:1003F00008080808080F0F08080808080F0F000071
:1004000000000F0F000000000000000000000000CE
:1004100000000000000000000000000000000000DC
:10042000C0F8BFFFFFFF1F7F0100000000000000B9
:1004300000F0FCFF7F7830000000000000000000AA
:1004400000000000000000000000000000000000AC
:10045000000000000000000000000000000000009C
:10046000000000000000000000000000000000008C
:10047000000000000000000000000000000000007C
:10048000000000000000000000000000000000006C
:100490000000000000000000000000000000301C10
:1004A000070E0F0701000000000000000000000020
:1004B000000000000000000000000000000000003C
:1004C000000000000000000000000000000000002C
:1004D00000000000000000001B1E272D36394B4E87
:1004E000636C7278878D939CB1B4C6C9D2D8E1E4AD
:1004F00001020304010302040402030104030201D4
:1005000003010200040506076D656E75537461638F
:100510006B206F766572666C6F77006D656E7553D4
:100520007461636B20756E646572666C6F770070C2
:100530007265737320616E79204B657900414C457B
:100540005254004D455353414745004C4F41444997
:100550004E47002020202020202020202020202066
:1005600020202020202020202000506C6561736511
:1005700020526573657420537769746368657300EE
:100580005377697463686573205761726E696E672B
:1005900000204F6C642056657273696F6E2045456C
:1005A00050524F4D202020434845434B2053455443
:1005B00054494E47532F43414C494200416C6172AC
:1005C0006D732044697361626C6564005265736584
:1005D00074207468726F74746C65005468726F7400
:1005E000746C65206E6F742069646C650050726570
:1005F000737320616E79206B657920746F20736B43
:10060000697000414C45525400454550524F4D20B1
:100610006C6F77206D656D004F46464142535255D1
:1006200073525525454C73454C2554487354482501
:10063000414C73414C2550312050312550322050CF
:1006400032255033205033250054485252554445EA
:100650004C4549443049443149443241494C47456D
:100660004154524E535731535732535733535734E3
:1006700053573553573653573753573853573953C2
:100680005741535742535743004F4646004F4E2061
:10069000002D2D2D004348002D2D2D2000525544B6
:1006A00020454C45205448522041494C20005031AF
:1006B000202050322020503320204D4158204655D4
:1006C0004C4C4359433143594332435943335050BF
:1006D0004D3150504D3250504D3350504D3450509C
:1006E0004D3550504D3650504D3750504D38434891
:1006F0003120434832204348332043483420434884
:100700003520434836204348372043483820434863
:10071000392043483130434831314348313243482E
:100720003133434831344348313543483136002D65
:100730002D2D2D00564552533A2056312E35343941
:10074000392D6572657A00444154453A2031312E85
:1007500030322E323031320054494D453A2031305A
:100760003A31303A3334002053564E3A20657239CC
:10077000782D7237303800204D4F443A204E4D4589
:10078000412020200012081200081C0808081C083C
:100790000000082200490022080000000000227F1B
:1007A0002200000008220049002208000008220060
:1007B00049002208000000227F22000000000008FB
:1007C0002200490022080000081C0808081C080034
:1007D0002F316A434E42B32B9B2498547A519E4842
:1007E000384AA150DD4A9B1D561F8C1F2C20A72183
:1007F00054546D00457870457846466E654D656485
:1008000043727300544F540053544B1153542500FA
:10081000544D45115453570053544154005B4D45BA
:100820004E555D20746F2072656672657368005363
:100830007461636B0F6200746D61696E0F6D73009C
:10084000746D7231204A69747465720F7573007427
:100850006D72314C6174206D696E0F757300746D2B
:1008600072314C6174206D61780F7573005354417F
:100870005432004D6F64650042616E6447617000E0
:10088000506F745363726F6C6C00416C61726D20B9
:100890005761726E696E67004D656D6F7279205792
:1008A00061726E696E6700545245303132414700C3
:1008B00054524530313241470044656661756C746D
:1008C00020537700537769746368205761726E69AB
:1008D0006E67005468726F74746C65205761726E35
:1008E000696E670053706C617368204E616D6500BE
:1008F00053706C6173682073637265656E004F4658
:1009000046004C69676874206F6E2053746B204DED
:1009100076004C69676874206F666620616674654E
:1009200072004C6967687420737769746368004665
:100930006C617368206F6E2062656570004265654A
:100940007020636F756E74646F776E004D696E759D
:1009500074652062656570005468726F74746C65AC
:1009600020726576657273650053494E474F534D4B
:100970005046494C540046696C74657220414443AA
:1009800000496E616374697669747920616C617283
:100990006D0042617474657279207761726E696E60
:1009A0006700436F6E74726173740048617074699C
:1009B0006320537472656E67746800537065616B71
:1009C0006572205069746368004265657065725095
:1009D0006953706B7200536F756E64204D6F646560
:1009E000005175696574204E6F4B657920785368A6
:1009F0006F727453686F7274204E6F726D20204C4A
:100A00006F6E672020784C6F6E67200042656570BE
:100A10006572004F776E6572204E616D65005241C0
:100A200044494F2053455455500043616C004D7567
:100A30006C7469706C6965720063683163683263F5
:100A40006833636834006F6666202B3D203A3D00B2
:100A50006D6F64650A2520737263202073770053DD
:100A60006C61766500545241494E455200000303C3
:100A700003030056455253494F4E005472696D2D81
:100A8000202B00204D656E75204578697420446FD9
:100A9000776E20202055705269676874204C656617
:100AA00074004449414700424700414E41005B4DBC
:100AB000454E555D205748454E20444F4E45004D0C
:100AC0004F564520535449434B532F504F545300D6
:100AD000534554204D4944504F494E54005B4D45B9
:100AE0004E555D20544F20535441525400535441AD
:100AF00052542043414C4942524154494F4E0043C5
:100B0000414C4942524154494F4E0066726565005E
:100B10004D4F44454C53454C00434F4C2044697263
:100B2000656374696F6E0041494C20446972656366
:100B300074696F6E00454C45204469726563746941
:100B40006F6E0053776173682052696E6700436F60
:100B50006C6C656374697665002D2D2D2020203125
:100B600032302020203132305820203134302020C3
:100B70002039302020202000537761736820547979
:100B800070650048454C4920534554555000004479
:100B9000454C455445204D4F44454C0F5B4D454E0B
:100BA000555D00543254685472696700547261692B
:100BB0006E657200452E204C696D69747300504F4C
:100BC000534E45470053686966742053656C004C6A
:100BD00050342F4C5035202044534D326F6E6C7979
:100BE0002044534D322F44534D580044534D20540C
:100BF0007970650053656E64205278204E756D6281
:100C00006572205B4D454E555D0050504D2046723B
:100C10004C656E0D6D536563002052784E756D0006
:100C20003443482036434820384348203130434835
:100C3000313243483134434831364348007553001C
:100C4000755365630050504D202020505858202087
:100C50002044534D32202050504D313620005072E8
:100C60006F746F00524554413132330042656570F4
:100C700020436E74005472696D205377004578707C
:100C8000202020457846696E6546696E6520204DB6
:100C9000656469756D436F61727365005472696D47
:100CA00020496E6300542D4578706F00542D5472A6
:100CB000696D00436F756E7420446F776E436F7576
:100CC0006E7420557020200054696D6572200054A8
:100CD0007269676765720054696D6572004E616D77
:100CE0006500534554555000000901000000000004
:100CF000000602004475706C69636174696E672058
:100D00006D6F64656C005B4D454E555D20205B4505
:100D10005849545D005945530B4E4F0044454C45CE
:100D20005445204D4F44454C004455504C49434197
:100D30005445204D4F44454C0020414243444546D4
:100D40004748494A4B4C4D4E4F50515253545556BB
:100D50005758595A6162636465666768696A6B6C63
:100D60006D6E6F707172737475767778797A3031D1
:100D700032333435363738395F2D2E0065787020A0
:100D80002025202073773120737732004558504F4B
:100D90002F445200000344522048696768004452BF
:100DA000204C6F77004452204D69640044725377A1
:100DB00032004472537731005765696768740045A3
:100DC00078706F004558504F2F445200002B2A5224
:100DD000004D49584552005072657373205B455869
:100DE00049545D20746F2061626F7274004D6178A8
:100DF000206D69786572732072656163683A2000BE
:100E000044454C455445204D4958205B4D454E5571
:100E10005D00536C6F772020557000536C6F772006
:100E200020446F776E0044656C61792055700044F2
:100E3000656C617920446F776E00416464202020E6
:100E400020204D756C7469706C795265706C6163AB
:100E50006520004D756C747078004F4646005761F0
:100E6000726E696E670053776974636800437572C8
:100E7000766573004F4E204F4646005472696D00F0
:100E80004F46464F4E2000466C4D6F646574726944
:100E90006D004F666673657400466D5472696D56D9
:100EA000616C0057656967687400536F757263659C
:100EB0000045444954204D49582000494E5345525D
:100EC00054204D495820002D2D2D2D202020763ED8
:100ED0006F66732020763C6F667320207C767C3EA4
:100EE0006F66737C767C3C6F6673414E4420202095
:100EF000204F522020202020584F522020202076A2
:100F0000313D3D7632207631213D76322076313EBC
:100F10007632202076313C7632202076313E3D7686
:100F2000322076313C3D76322000535700435553F2
:100F3000544F4D20535749544348455300000253E2
:100F4000414645545920535749544348455300009E
:100F500002434C454152204D49584553205B4D4575
:100F60004E555D002052455441004368616E6E65E8
:100F70006C204F726465720054454D504C4154458D
:100F80005300434F5059205452494D205B4D454E1C
:100F9000555D002D2D2D494E56004C494D49545359
:100FA0000000030303030303030303030303030317
:100FB00003030043560043555256455300505245D3
:100FC00053455400454449542D3E0043555256451F
:100FD0000009002D2D2D494E56004F46464F4E20FC
:100FE000002D2D2D783E30783C307C787C663E306C
:100FF000663C307C667C633120633220633320633F
:10100000342063352063362063372063382063390A
:1010100020633130633131633132633133633134D2
:1010200063313563313600454550524F4D206F7660
:101030006572666C6F7700454550524F4D206F7654
:101040006572666C6F770067656E7772697465208C
:101050006572726F7200454550524F4D20466F7257
:101060006D617474696E67004261642045457072F9
:101070006F6D2044617461004D4F44454C20202029
:101080002020004D45202020202020202000500836
:101090005000000000000000006F00000700070083
:1010A000147F147F14242A7F2A12231308646236C3
:1010B000495522500005030000001C224100004158
:1010C000221C0014083E081408083E08080050308E
:1010D00000000808080808006060000020100804EC
:1010E00002003E49453E0000427F400062514946B1
:1010F0000041494936001814127F00274545390040
:101100003E49493200017905030036494936000657
:1011100049291E000036360000005636000008142B
:10112000224114141414144122140800020151091C
:101130000600060909067E0909097E7F49494936E4
:101140003E414141227F4141221C7F494949417F23
:10115000090909013E4149497A7F0808087F004191
:101160007F41002040413F017F081422417F4040E1
:1011700040407F020C027F7F0408107F3E414141C6
:101180003E7F090909063E4151215E7F0919294622
:10119000264949493201017F01013F4040403F1F3C
:1011A0002040201F3F4030403F631408146307086D
:1011B0007008076151494543007F4141000204081E
:1011C00010200041417F00040201020440404040E1
:1011D00040000102040020545454787F48444438AD
:1011E0003844444420384444487F38545454180800
:1011F0007E0901020C5252523E7F080404780044DA
:101200007D40002040443D007F1028440000417F85
:1012100040007C041804787C080404783844444472
:10122000387C14141408081414187C7C080404086E
:101230004854545420043F4440203C4040207C1CEF
:101240002040201C3C4020403C44281028440C50A6
:1012500050503C4464544C44000836410000007F28
:10126000000000413608000808221C08081C22085B
:1012700008A06080000000000000000000000000E6
:101280000000FFFF0000000000001F3F00003F1FA4
:1012900000003030FFFF3030FFFF30303078CCCCF2
:1012A000FFFFCCCC8C0C060F0F86C0E070381C0CF6
:1012B0003CFEC7E3F33B1E0C00000000333B1F0F56
:1012C000000000000000F0F81C0E07030000000002
:1012D00003070E1CF8F000003030E0C0FCFCC0E05A
:1012E0003030C0C0C0C0FCFCC0C0C0C000000000A6
:1012F000000000000000C0C0C0C0C0C0C0C0C0C06E
:101300000000000000000000000000000080C0E0BD
:1013100070381C0C000000000000000000000000FD
:10132000000038380000000000000000000000004D
:10133000000003033F3F03033F3F03030C0C0C0C6F
:101340003F3F0C0C07030C0E07030100183C3C1830
:101350000F1F383133331E1E3333000000000000EE
:1013600000000000000003070E1C383000000000E1
:1013700030381C0E07030000030301000F0F0001AB
:101380000303000000000F0F000000000000333BCB
:101390001F0F00000000000000000000000000001F
:1013A0000000183C3C18000000000C0E0703010070
:1013B000000000000000FCFE87C3E377FEFC000095
:1013C0000C0EFFFF0000000000000C0E0783C3E7B7
:1013D0007E3C00000303C3C3C3E7FE3C0000C0E043
:1013E00070381C0EFFFF00003F3F33333373E3C3FD
:1013F0000000FCFEC7C3C3C78E0C00000303C3E399
:10140000733B1F0F00003CFEE7C3C3E7FE3C000038
:101410003C7EE7C3C3E7FEFC0000183C3C1800001C
:1014200000000000183C3C18000000000000C0E074
:10143000F0381C0E07033030303030303030303070
:1014400003070E1C38F0E0C000000C0E07030383F6
:10145000C3E77E3C00000F1F3B3130381F0F0000F8
:1014600030303F3F3030000000003C3E37333130F9
:10147000303000003030303030391F0F00000303AF
:10148000030303033F3F00000C1C383030381F0FAC
:1014900000000F1F383030391F0F000000003F3FA1
:1014A0000000000000000F1F393030391F0F00000E
:1014B000000030381C0E07030000060F0F06000066
:1014C00000000000333B1F0F00000000000000017F
:1014D00003070E1C38300303030303030303030352
:1014E00030381C0E070301000000000000003333F9
:1014F0000100000000003C7EE7C3C3E77E3CF0F83B
:10150000DCCEC7C7CEDCF8F0FFFFC3C3C3C3C3E75D
:10151000FE3CFCFE0703030303070E0CFFFF03035F
:1015200003070E1CF8F0FFFFC3C3C3C3C3C3030309
:10153000FFFFC3C3C3C3C3C30303FCFE0703C3C38B
:10154000C3C7CECCFFFFC0C0C0C0C0C0FFFF0000FB
:101550000303FFFF03030000000000000303FFFF7D
:101560000303FFFFC0E0F0381C0E0703FFFF00007D
:10157000000000000000FFFF0E1CF8F81C0EFFFF2B
:10158000FFFF3870E0C08000FFFFFCFE070303038D
:101590000307FEFC000000000000000000003F3FC9
:1015A0000000000000003F3F3F3F30303030303916
:1015B0001F0F0F1F3830303030381C0C3F3F303099
:1015C00030381C0E07033F3F303030303030303081
:1015D0003F3F00000000000000000F1F3830303097
:1015E00030303F3F3F3F0000000000003F3F000021
:1015F00030303F3F303000000C1C383030381F0F87
:1016000000003F3F000103070E1C38303F3F3030E1
:101610003030303030303F3F0000000000003F3FAE
:101620003F3F0000000103033F3F0F1F38303030C1
:1016300030381F0FFFFFC3C3C3C3C3E77E3CFCFEAC
:10164000070303030307FEFCFFFFC3C3C3C3C3E7D2
:101650007E3C3C7EE7C3C3C3C3C78E0C03030303B6
:10166000FFFF03030303FFFF000000000000FFFF74
:10167000FFFF000000000000FFFFFFFF0000000070
:101680000000FFFF0F1F38F0E0E0F0381F0F3F7F32
:10169000E0C08080C0E07F3F03030383C3E3733B6C
:1016A0001F0F0000FFFF0303030300000C1C387032
:1016B000E0C080000000000003030303FFFF000000
:1016C00030381C0E07070E1C3830000000000000E8
:1016D000000000003F3F00000000000000000F1F5E
:1016E000383033371E1C3F333F3F000003070E1CCA
:1016F00038300C1C3830303030391F0F00000000FB
:101700003F3F000000000F1F3830303030381F0FCF
:1017100003070E1C38381C0E07030F1F38381F1F15
:1017200038381F0F3C3E0703010103073E3C000011
:1017300000013F3F010000003C3E37333130303084
:10174000303000003F3F30303030000000000000FB
:10175000000103070E0C0000303030303F3F000026
:101760000000000000000000000030303030303059
:1017700030303030000003070E1C3830000000000D
:10178000303030303070E0C0FFFFC0E0703030707B
:10179000E0C0C0E07030303030300000C0E0703069
:1017A0003070E0C0FFFFC0E0703030303070E0C01B
:1017B000C0C0FCFEC7C303070E0CF0F89C0C0C0C59
:1017C0000C0CFCFCFFFFC0E070303070E0C000008B
:1017D0003030F3F300000000000000003030F3F37D
:1017E0000000FFFF0080C0E0703000000000030335
:1017F000FFFF00000000F0F03070E0E07070E0C02B
:10180000F0F0C0E070303070E0C0C0E070303030D8
:101810003070E0C0000000000000000000000C1E5E
:101820003F33333333333F3F3F3F30303030303856
:101830001F0F0F1F3830303030381C0C0F1F38305E
:10184000303030303F3F0F1F3B33333333330303EC
:1018500000003F3F0000000000000001333333333D
:10186000333B1F0F3F3F0000000000003F3F0000E0
:1018700030303F3F303000000C1C383030381F0F04
:1018800000003F3F03070F1C3830000000003030DD
:101890003F3F303000003F3F0000030300003F3F68
:1018A0003F3F0000000000003F3F0F1F3830303046
:1018B00030381F0FF0F03030303030F0E0C0C0E092
:1018C000F0303030E0C0F0F0F0F0C0E07030307058
:1018D000E0C0C0E0F0303030303000003030FFFF8A
:1018E000303000000000F0F0000000000000F0F0D8
:1018F000F0F0000000000000F0F0F0F00000000048
:101900000000F0F03070E0C08080C0E07030F0F097
:10191000800000000000F0F03030303030B0F0F0E7
:1019200070300000C0E03C3E0703000000000000F3
:10193000FFFF00000000000003073E3CE0C0000085
:10194000C0C0C0C00C1CF8F0E0C0C0E0F0F81C0C37
:10195000C0C0C0C03F3F03030303030301000001F5
:101960000303030303033F3F3F3F00000000000069
:101970000000303133333333333F1E0C00000F1F70
:10198000383030381C0C0F1F383030381C0C3F3FBB
:1019900003070E1C38381C0E07030F1F38381C1C99
:1019A00038381F0F30381C0F07070F1C3830000164
:1019B00033333333333B1F0F30383C3E3733313012
:1019C0003030000000010F1F383000000000000020
:1019D0003F3F00000000000030381F0F01000000F2
:1019E000000000000C0E07030100000103070E0CAD
:1019F0000000000040800804201002010C1A181A90
:101A00001E1A2B1A321A3F1A4A1A551A53696D7048
:101A10006C6520342D434800542D43757400537475
:101A200069636B7920542D43757400562D54616998
:101A30006C00456C65766F6E5C44656C7461004843
:101A4000656C69205365747570004779726F205317
:101A50006574757000536572766F205465737400F9
:101A60000000891112239B322446AD573665BF749E
:101A7000488CC19D5AAFD3BE6CCAE5DB7EE9F7F84E
:101A80008110080193331A22A5562C47B7753E647E
:101A9000C99C408DDBBF52AEEDDA64CBFFF976E82E
:101AA00002218B30100299132667AF763444BD555E
:101AB0004AADC3BC588ED19F6EEBE7FA7CC8F5D90E
:101AC00083310A2091121803A7772E66B5543C453E
:101AD000CBBD42ACD99E508FEFFB66EAFDD874C9EE
:101AE00004428D5316619F702004A9153227BB361E
:101AF0004CCEC5DF5EEDD7FC6888E1997AABF3BACE
:101B000085520C4397711E60A1142805B3373A26FD
:101B1000CDDE44CFDFFD56ECE9986089FBBB72AAAD
:101B200006638F7214409D512225AB343006B917DD
:101B30004EEFC7FE5CCCD5DD6AA9E3B8788AF19B8D
:101B400087730E6295501C41A3352A24B1163807BD
:101B5000CFFF46EEDDDC54CDEBB962A8F99A708B6D
:101B6000088481951AA793B62CC2A5D33EE1B7F09D
:101B70004008C919522BDB3A644EED5F766DFF7C4D
:101B8000899400859BB712A6ADD224C3BFF136E07D
:101B9000C1184809D33B5A2AE55E6C4FF77D7E6C2D
:101BA0000AA583B4188691972EE3A7F23CC0B5D15D
:101BB0004229CB38500AD91B666FEF7E744CFD5D0D
:101BC0008BB502A499961087AFF326E2BDD034C13D
:101BD000C3394A28D11A580BE77F6E6EF55C7C4DED
:101BE0000CC685D71EE597F42880A1913AA3B3B21D
:101BF000444ACD5B5669DF78600CE91D722FFB3ECD
:101C00008DD604C79FF516E4A9902081BBB332A2FC
:101C1000C55A4C4BD7795E68E11C680DF33F7A2EAC
:101C20000EE787F61CC495D52AA1A3B03882B193DC
:101C3000466BCF7A5448DD59622DEB3C700EF91F8C
:101C40008FF706E69DD414C5ABB122A0B9923083BC
:101C5000C77B4E6AD5585C49E33D6A2CF11E780F6C
:101C60002020475053204E4D45412064617461202F
:101C70003F2F342020004C6F6E67697475646500D7
:101C80004C61746974756465202020202053617450
:101C900000436F75727365206F7665722067726F8F
:101CA000756E640047726E6453706565645B6B6E3D
:101CB000745D2020536174002F53004F4646004F3F
:101CC0004E0042656570004C69667400486F6D6532
:101CD00000416C7469747564652053617420202020
:101CE0004D617800446174650054696D65720055FA
:101CF00054432D54696D65202020202020536174A9
:101D000000000B1A11241FBECFEFD0E1DEBFCDBF04
:101D100011E0A0E0B1E0E0E3FAEE02C005900D9220
:101D2000A434B107D9F71EE0A4E4B1E001C01D92CC
:101D3000A23EB107E1F71DE1C4E0DDE104C0229756
:101D4000FE010E94D174C230D107C9F70E943B192D
:101D50000C9416750C9400003091B70422B7809152
:101D6000B7043817C9F7932F80E030E0282B392BC0
:101D7000C901089529E28202900111243595279521
:101D80003595279587FD815C86FB880F880B80F948
:101D9000992787FD9095281B390BC9010895F89460
:101DA0002091D70D3091D80D7894C9010895482F0E
:101DB00050E09A01220F331F63E0440F551F6A95CC
:101DC000E1F7240F351F22543E4FC901089590E0DA
:101DD0009C01220F331F220F331F280F391F22505F
:101DE0003D4FC9010895AF92BF92CF92DF92EF921B
:101DF000FF920F931F93CF93DF93C82E162FEA0104
:101E0000F22ED02E57FF10C022FF02C08CE101C07D
:101E10008FE09C2D981B892F612F4DE22F2D0E9462
:101E2000F75CD095C195DF4F2D2D2F218C2D612F83
:101E30004AE30E94F75C8F2D90E0B4E0AB2EB12C0A
:101E4000A822B922F2FE02C0E2E001C0E0E0CE0129
:101E50006CE370E00E947F749B01442737FD40953E
:101E6000542F0F2D00618E2F8C0D612FA2E0EA2ED2
:101E70000E94F75EA114B10411F0ECE101C0E1E1B0
:101E8000CE016CE370E00E947F749C01442737FD13
:101E90004095542F0D2D00618E2F8C0D612FF2E097
:101EA000EF2E0E94F75EDF91CF911F910F91FF906F
:101EB000EF90DF90CF90BF90AF9008950F931F9356
:101EC000062F122F206250E00E942D6017FD07C0E0
:101ED0008091A90D602F46E7212F0E94F75C1F918A
:101EE0000F910895242F409108010E945E0F0895DC
:101EF0000F93022F442319F44FE257E020C04530DE
:101F0000A8F4E0918801F0E0EE0FFF1FEE0FFF1F35
:101F10003197E40FF11DE051FB4F449150E0440F25
:101F2000551F440F551F4756594F09C0453250F4AD
:101F300050E0440F551F440F551F4656594F24E09B
:101F40000E94BA5D0F910895FF920F931F93182F6F
:101F5000F62E022F442321F448E956E024E00EC077
:101F60008A5E4A3008F485506F2D50E0202F0E9481
:101F70002D60812F6F2D45E956E022E00E94BA5D69
:101F80001F910F91FF9008950F931F93DF93CF93AD
:101F900000D0CDB7DEB7382F162F942F022F442351
:101FA00029F0463139F04A3E81F408C08A5F41E9A0
:101FB00056E007C08A5F4DE856E003C08A5F49E8F3
:101FC00056E0202F0E94EA5D28C04095441F442718
:101FD000441F81E2841B482F832F39839A830E94F8
:101FE000F75C3981832F8A5F9A81E92FFF27E7FD0C
:101FF000F095F7FF03C0F095E195FF4FFF27E7FD50
:10200000F0953197AF01440F551F4E0F5F1F475B8F
:10201000594F612F23E00E94BA5D0F900F90CF912E
:10202000DF911F910F91089589E496E00895DF9262
:10203000EF92FF920F931F93D82EE62EF42E10915D
:10204000AF01E12FFF27E7FDF095F7FF03C0F09503
:10205000E195FF4FE031A4F483E0E802F0011124A0
:10206000E85EF94F8D2D6E2DAF0123E00F2D0E94FC
:10207000BA5D1F3F3CF58D2D86506E2D41E21FC08D
:102080008D2D8650E53264F411161CF4412F4F500B
:1020900002C0412F415F6E2D2F2D0E94C40F12C030
:1020A00011161CF4412F445202C0412F4C5D6E2D7D
:1020B0002F2D0E94C40F8D2D8E5E6E2D4DE62F2D7F
:1020C0000E94F75C1F910F91FF90EF90DF900895B1
:1020D0008C3038F4E82FF0E0EE0FFF1FEF50FB4F8D
:1020E0002AC0803198F4E82FF0E0DF01AA0FBB1F6F
:1020F000A257BB4FEE0FFF1FE25AFE4F2D913C91AE
:10210000119780819181281B390B0AC0843158F4C2
:10211000E82FF0E0EE0FFF1FE257FB4F20813181E7
:10212000220F331F0DC0843248F4E82FF0E0EE0F89
:10213000FF1FE952FB4F2081318102C020E030E0D7
:10214000C9010895AF92BF92DF92EF92FF920F9371
:102150001F93DF93CF9300D0CDB7DEB7F82E463074
:1021600008F0DEC0882309F4DEC0863119F08A3E0B
:1021700019F4D6C061E0D7C0992787FD90959C01DE
:1021800097FF04C022273327281B390B2A307CF401
:102190001F144CF02DE030E0A901481B590BCA0177
:1021A0000E949761BAC00D960E949761BBC02A50E9
:1021B000A22EBB249501220F331F2A0D3B1D2C5547
:1021C0003E4FF901E85AFD4F5081552309F4A8C04C
:1021D000453029F4F501EE57FB4F80819CC0F90191
:1021E000EA5AFD4FD080295A3D4FF901E080553021
:1021F00008F4A6C0583060F08D2D81504A83598371
:102200000E9468108C018E2D81500E946810A2C01F
:1022100020E030E000E010E0583088F4553088F5D8
:10222000523009F462C0533020F4513009F06EC0CE
:1022300057C05330D1F0543009F068C01CC05A3038
:1022400009F44EC05B3038F4583009F43FC05930BF
:1022500009F05CC040C05C3009F44CC05C3008F44C
:1022600044C05D3009F052C04AC017FF39C0109514
:1022700001951F4F35C017FF38C0109501951F4FAE
:1022800034C0142F1F5F8D2D60E0412F0E94A210DB
:10229000082F8E2D60E0412F0E94A210F501EE0F55
:1022A000FF1FEA0DFB1DE450FC4F9081953029F48F
:1022B000002361F1882341F52AC0963029F40023D8
:1022C00019F5882319F120C0802721C081E0021769
:1022D0001307E1F41CC081E002171307C1F416C014
:1022E00081E0201731079CF011C081E0021713072D
:1022F00074F00CC081E0021713074CF407C081E0B2
:102300002017310724F402C081E001C080E0F5010C
:10231000EE57FB4F80831F142CF061E0682703C049
:1023200060E001C0682F862F0F900F90CF91DF9152
:102330001F910F91FF90EF90DF90BF90AF900895A5
:102340008D2D81504A8359830E9468108C018E2DF7
:102350000E94BA0E9C014A8159815ECF86B3809556
:102360008E7708950E94AE118823E1F70E940661DE
:1023700008958091750160E040E00E94A2108823DA
:1023800031F480919F049091A004009711F0C79AB6
:102390000895C79808950F931F93CF93DF93EC018F
:1023A0008B010E948D5C82E260E043E056E024E015
:1023B0000E94EA5D80E2BE010E94115E88E2B801DF
:1023C0000E94115E80E36DEE75E00E94115E0E9436
:1023D0009760809172010E948D600E94B211DF911E
:1023E000CF911F910F9108950F93AB0160E123E00E
:1023F00000E00E94BA5D0F910895DF92EF92FF9284
:102400000F931F93CF93DF938091870181FD83C04A
:1024100080E895E06AE675E00E94CB1190919F01FB
:10242000892F887341F0883131F0883221F0803370
:1024300011F0883329F4892F877C886080939F016D
:1024400000E010E065E1E62EF12C08C0C701801B1A
:1024500091090E949761110F182B0F5F0830B0F39C
:10246000D0909F01D12680E060E143E555E026E170
:1024700000E00E94BA5DCD2DD0E0CE0180FF05C006
:1024800082E069E476E00E94F411C1FF05C087E1B3
:102490006CE476E00E94F411C2FF05C08CE26FE4A8
:1024A00076E00E94F411CE01887390700097B1F02D
:1024B000012F13FF05C081E462E576E00E94F4116C
:1024C00004FF05C081E465E576E00E94F41105FF94
:1024D00005C081E468E576E00E94F411C6FF05C0FE
:1024E00086E56BE576E00E94F411D7FE05C08BE629
:1024F0006EE576E00E94F4110E94976080919F0142
:10250000181749F00E94AE11882329F40E94B911CE
:1025100000E010E09BCFDF91CF911F910F91FF90D2
:10252000EF90DF9008951F93CF93DF930E94AE1139
:1025300020E030E011E0482F50E02F5F3F4FBA011C
:10254000022E02C0759567950A94E2F760FD03C0FC
:102550001F5F183091F71150163030F5812F0E940F
:102560000857882309F110937101812F0E940C579D
:1025700081E00E94DB570E948D5C86E160E04BE4C5
:1025800055E024E00E94EA5DC4EAD1E01AE04991F6
:10259000812F68E124E00E94F75C155F1837B9F7D6
:1025A0000E9497600E94B211DF91CF911F91089510
:1025B000CF93DF93EC010E948D5C82E260E043E404
:1025C00055E024E00E94EA5D88E1BE010E94115EB0
:1025D0000E949760809172010E948D60DF91CF917F
:1025E00008951F93CF93DF93EC01162F0E948D5C0B
:1025F00082E260E04DE355E024E00E94EA5D88E17C
:10260000BE010E94115E8CE168E34FE255E00E943A
:10261000195E0E949760112319F48091720101C024
:1026200089E10E948D6082E10E94B56D0E94B21125
:102630000E94AE118823C9F480916B0E833019F487
:10264000A89510926B0E8091750160E040E00E94A9
:10265000A210882331F480918C01882311F4112376
:1026600011F0C79AE5CFC798E3CFDF91CF911F91C3
:10267000089580918104882351F081E995E060E01C
:102680000E94F112809181048E7F809381040895CD
:102690008091870187FD07C0887329F48CEB95E052
:1026A00060E00E94F11208958091870182FD0AC0C6
:1026B0000E94FC58883C910528F489E096E060E08F
:1026C0000E94F1120895EF92FF92CF93DF93A82F0B
:1026D000AF70A6509091B601923074F0292F332735
:1026E00027FD309521503040C1E0D0E002C0CC0F32
:1026F000DD1F2A95E2F79C2FA83008F09CC06A2FB6
:10270000659570E0FB01EE0FFF1FE050FF4F019059
:10271000F081E02DB081992379F4CB2FDD27C7FD1F
:10272000D095D7FF03C0D095C195DF4F9C2FC7FD33
:102730009D5F959595959F5F4091880150E0417010
:10274000507022E030E0241B350B2617370769F460
:102750002091B5012F7009F473C021E094E030910D
:102760008A0130FF03C0919501C020E04B2F55270F
:1027700047FD5095C92FDD27C7FDD095A0FF03C0A9
:10278000C40FD51F04C0BA016C1B7D0BEB01209751
:1027900029F07E019F2D9B2797FF0BC0222349F430
:1027A000BB2339F010820E94F66186E10E94B56D6C
:1027B00041C0CE0184589F4F893F9105B8F4C08332
:1027C00086E00E94DB57CE0183589F4F8B3F9105D7
:1027D00088F5D7FF03C0D095C195DF4FD595C79534
:1027E000D595C795BE01645C462F1FC01C161D06FB
:1027F00014F48DE701C083E8808386E00E94DB57F4
:10280000CE0183589F4F8B3F9105A0F4CE01D7FF97
:1028100003C0909581959F4F64E070E00E947F74A3
:10282000709561957F4F462F445C89E494E065E1A3
:102830000E94426C80E0DF91CF91FF90EF9008956D
:1028400020E08DCF8F929F92AF92BF92CF92DF9276
:10285000EF92FF920F931F93CF93DF93182FEB010B
:102860005A016901802E84FF06C01F70106694E033
:10287000992E05E003C085E0982E04E0802F806645
:10288000181761F0802F8064181741F0809120059F
:10289000882369F0133611F0133449F47E0108944B
:1028A000E11CF11C83E10E94B56D892D18C0992DA2
:1028B0009066191761F0992D9064191741F08823DB
:1028C00009F474C0123619F0123409F06FC07E0199
:1028D0000894E108F10884E10E94B56D802F90E032
:1028E0000E949761882351F0EE24FF24EC1AFD0A20
:1028F000892D0E94F661802F0E94F661A114B10417
:1029000091F481E0C816D10471F4103661F410928C
:10291000200501E0E02EF12C209711F0EE24FF2499
:1029200080E60E94F66120919C0430919D04E21A99
:10293000F30ACE14DF0444F4812F0E94F66183E190
:102940000E94B56D76010AC0EA14FB043CF4812FA5
:102950000E94F66184E10E94B56D7501EC16FD06DA
:10296000A9F0E114F10451F4812F0E94E761D7FF2F
:1029700002C083E101C084E10E94B56D882D83709F
:102980000E94DB5781E08093990402C01092990461
:10299000C701DF91CF911F910F91FF90EF90DF90D2
:1029A000CF90BF90AF909F908F9008957E01A6CF5B
:1029B0000F93772767FD7095552747FD509533276F
:1029C00027FD30950E9422140F9108950F937727C9
:1029D00067FD7095552747FD5095332727FD3095A6
:1029E00002E00E9422140F9108950F93772767FD4C
:1029F0007095552747FD5095332727FD309501E009
:102A00000E9422140F910895E0919804F0E0EE0FD7
:102A1000FF1FE057FB4F80819181089590919804AA
:102A2000992319F4882331F418C0882319F4892FC5
:102A3000815001C080E08093980487E10E94B56DC9
:102A4000E0919804F0E0EE0FFF1FE257FB4F01907A
:102A5000F081E02D8EEB099508958BE195E060E023
:102A60000E94F1120895FC01A0919804B0E0AA0F11
:102A7000BB1FA257BB4F8D939C938FEB099587E1AA
:102A80000E94B56D0895CF93DF93EC018091980477
:102A9000982F9F5F90939804953040F0809398040E
:102AA00088E095E060E00E94F1120FC087E10E948B
:102AB000B56DE0919804F0E0EE0FFF1FE257FB4F79
:102AC000D183C0838FEBFE010995DF91CF910895EB
:102AD00089E494E00E94416B882311F084E105C0F1
:102AE0008091B804882321F081508093B80407C0F6
:102AF0009091630081E091FF80E08093B904809120
:102B0000B90408951092A3041092A5041092A4048D
:102B10001092A204089520919F043091A0042115E1
:102B2000310531F0215030403093A00420939F04B0
:102B3000882369F040918C0150E084EF91E0489F38
:102B40009001499F300D589F300D112402C020E0A4
:102B500030E08091A104882369F06091940170E0D5
:102B600044EF51E0649FC001659F900D749F900DEC
:102B7000112402C080E090E040919F045091A00495
:102B80004217530720F43093A00420939F04209110
:102B90009F043091A0042817390720F49093A004D3
:102BA00080939F040E94B9110895E82FF0E0E0504F
:102BB000FB4FE491F0E0EE0FFF1FE454FB4F208148
:102BC0003181C9010895CF92DF92EF92FF920F9366
:102BD0001F93DF93CF930F92CDB7DEB720E0CC24C5
:102BE000DD24822F29830E94D515092F10E0C00E05
:102BF000D11E29812F5F2430A1F7C6010F90CF91FC
:102C0000DF911F910F91FF90EF90DF90CF9008958B
:102C10001F930E94CF0E41E02091EF043091F00409
:102C20008217930709F440E040939E040E94CF0E60
:102C30009093F0048093EF0485E295E060E00E94B9
:102C4000713580919E04882309F4CBC08091A20441
:102C500080FF14C08091A304982F9F5F9093A304DA
:102C6000943660F083568093A3048091A4049091DD
:102C7000A50401969093A5048093A40480E00E948B
:102C8000E9570E948D5C0E9409610E946313182F0E
:102C90000E948B152091FD043091FE0480919A04CE
:102CA00090919B04821B930B60E270E00E947F7402
:102CB00070939D0460939C046115710591F080915F
:102CC000ED049091EE04821B930B62E070E00E9491
:102CD0007F7470939D0460939C0430939B042093B5
:102CE0009A043093EE042093ED0480918A0185FFCD
:102CF00004C010929D0410929C04E0919804F0E0AE
:102D0000EE0FFF1FE257FB4F0190F081E02D812F66
:102D100009950E9497600E946815882321F0809190
:102D200065008F7E03C0809165008061809365009F
:102D30000E94CF0E8F7190708230910509F04FC0C4
:102D400087E00E94D5159C01E4E0220F331FEA952D
:102D5000E1F768E070E00E947F74409174015527AC
:102D600047FD50954A5F5F4F649FC001659F900D7E
:102D7000749F900D1124820F931F20918A0126FDCC
:102D800005C06091090170910A0102C060EF70E016
:102D90002091080130E02F5F3F4F0E946B74260F97
:102DA000371F35952795209308018091EC04805EAC
:102DB0008093EC04882399F480917301281778F4A8
:102DC000223368F081E10E94B56D80918A0183FF12
:102DD00006C082E390E09093A00480939F04109239
:102DE000A1041F910895ACEBB4E0ECECF4E060E0DA
:102DF000862F806487B9369A408951898D919C913C
:102E0000119796958795840F951F8E7F11969C93A9
:102E10008E9320813181C901840F951F96958795E6
:102E2000918B808B349BFECF349A84B195B1820F05
:102E3000931F96958795819391936F5F1296683053
:102E4000B9F60895EF92FF920F931F93CF93DF93FC
:102E500080918A0184FD44C00E94B9110E948D5C5A
:102E600080E060E045ED50E020E000E00E94985CEA
:102E70008091900184FD08C080E068E345E951E05D
:102E80002AE000E10E94BA5D0E9497608091720181
:102E90000E948D600E94B21100E20E94F316015060
:102EA000E1F70E94E3158C010E94CF0EEC01C057A0
:102EB000DE4F0DC00E94F3160E94E3157C010E94B4
:102EC000AE11882369F4E016F10651F406C00E94A1
:102ED000CF0EC817D90771F703C00E94B911F7CFF9
:102EE000DF91CF911F910F91FF90EF900895ECEB40
:102EF000F4E040E012C067B9369A349BFECF349AB2
:102F000024B135B1820F931F5150A9F7969587953B
:102F1000819391934F5F483031F054E080E090E02E
:102F2000642F6064E8CF0895ECEBF4E020E0822F9A
:102F3000806487B9369A349BFECF349A84B195B1B8
:102F4000880F991F819391932F5F283081F70895FF
:102F5000FF920F931F93CF93DF938091870180FDA2
:102F60003AC08091880190E08170907002E010E09A
:102F7000081B190BF801EE0FFF1FEC5BFE4FC18120
:102F8000D281609687859089C81BD90B0E949417BF
:102F9000F02E802F0E94D515C817D907E4F40E949F
:102FA000AE118823C1F40DC00E9494178F2D0E948A
:102FB000D515C817D9077CF40E94AE11882341F0BB
:102FC0000AC08BED95E06CEC75E00E94CB11ECCF64
:102FD0000E94B911E9CFDF91CF911F910F91FF901E
:102FE00008958EE587B9369A349BFECF349A84B122
:102FF00095B104964091090150910A019A0163E04C
:10300000220F331F6A95E1F7241B350B820F931FA4
:1030100023E0969587952A95E1F790930A0180938E
:103020000901089578941F920F920FB60F92112400
:103030008F938091B7048F5F8093B7048F910F9027
:103040000FBE0F901F90189578941F920F920FB695
:103050000F9211242F933F934F935F936F937F931E
:103060008F939F93AF93BF93EF93FF93F89487B79A
:103070008D7F87BF789481B78E5F81BF90914B041D
:1030800080914D04882379F080919301882349F041
:10309000813051F48091E10E890F8093E10E87FF1A
:1030A00002C01B9A01C01B9880910B01982F915070
:1030B00090930B01882371F48DE480930B0189E4D4
:1030C00094E00E94556B0E94076280916B0E8260B3
:1030D00080936B0EF89487B7826087BF7894FF91D6
:1030E000EF91BF91AF919F918F917F916F915F9180
:1030F0004F913F912F910F900FBE0F901F901895F9
:1031000078941F920F920FB60F9211241F932F9352
:103110003F934F935F936F937F938F939F93AF935F
:10312000BF93EF93FF932091800030918100F8943A
:1031300080917D008F7D80937D0078948091BA048A
:103140009091BB04A901481B590BCA01969587951C
:103150003093BB042093BA041091B604212F215060
:10316000283058F59C012152334055E02737350768
:1031700008F5E12FF0E0EE0FFF1FEC55FB4FAC011F
:103180004C5D554020918E01332727FD3095265FF9
:103190003F4F429FC001439F900D529F900D1124BD
:1031A0006AE070E00E947F74718360831F5F1093F8
:1031B000B6040CC01092B60409C0815A9F402EE29A
:1031C0008F3D920718F481E08093B604F8948091C3
:1031D0007D00806280937D007894FF91EF91BF9194
:1031E000AF919F918F917F916F915F914F913F919F
:1031F0002F911F910F900FBE0F901F901895E3EE27
:10320000FEE09F0181918535E1F3225E3E40C901D8
:103210000895CF93DF930E94AC0EEC0180918B0157
:10322000813019F40E94F31607C0823019F40E940D
:10323000771702C00E9494178EE587B90E9408167E
:103240000E94F11780916B0E833019F4A8951092AB
:103250006B0E0E94AC0E8C1B9D0B2091C70630910B
:10326000C8062817390720F49093C8068093C7062C
:10327000DF91CF9108951F938FEF8ABB1BBA91E81E
:1032800097BB9EE798BB9EE394BB91EC95BB11BAAC
:1032900082BB88E082B987EF83B9109261001092F7
:1032A000620084E1809364008BEF809365000E944C
:1032B00057600E94BC6D80E487B985E886B987E0D5
:1032C00083BF8CE981BF87B7836087BF1FBC8AE05B
:1032D0008EBD10928B0082E880938A0080917D00E1
:1032E000806280937D00EDB7FEB7329785E502C01E
:1032F000808331979EE0E23EF90709F0C8F77894A1
:103300008FE49FE390938F0480938E0489E10E9461
:103310008D600E949457109171010E9493128091C8
:1033200072010E948D6050918C014091940145176B
:1033300078F4652F70E024EF31E0629FC001639F55
:10334000900D729F900D11249093A00480939F0480
:10335000541770F450E024EF31E0429FC001439FC6
:10336000900D529F900D11249093A00480939F0480
:103370000E94B91180919301813039F480918A01C2
:1033800084FD03C087E00E94B56D0E9422170E9451
:1033900054130E9494170E94A8170E94FD110E94C6
:1033A00048130E9439130E94B21180EF90E090936D
:1033B0000A01809309010E94AC692DE088E190E048
:1033C0000FB6F894A89581BD0FBE21BD85E295E0AA
:1033D00060E00E9471358FE291E30E94431581E025
:1033E0000E940E15809172010E948D608091710182
:1033F000181729F081E00E94DB570E94775880ED72
:1034000097E09BBD8ABD80E186BF87B7806187BF9B
:103410000E940919FDCF89E494E00E943E6B089553
:1034200029E282029001112435952795359527953B
:1034300087FD815C86FB880F880B80F9992787FDC3
:103440009095281B390BC90108959C01E5E035953D
:103450002795EA95E1F7AC01440F452F441F550B22
:10346000280F391F892F990F990B8595280F391F20
:10347000241B350BC9010895F8942091D70D309184
:10348000D80D7894C9010895AC0180E060E021E096
:103490000E94EA5D08950F931F93CF93DF93182F37
:1034A00088E198E00E94441A113658F0133628F04B
:1034B000133639F486EE9AE102C08FE49FE30E944E
:1034C000331586E068E040E158E00E94195E4091C3
:1034D0003F06509140068AE268E020E000E00E944A
:1034E000F30E40914106509142068EE468E020E0E0
:1034F0000E94F30E86E060E148E058E00E94195E09
:1035000040914306509144068AE260E120E00E9427
:10351000F30E4091450650914606F4E056954795C6
:10352000FA95E1F78EE460E120E00E94F30E86E672
:1035300060E044E058E00E94195E40913D065091E1
:103540003E068EE460E020E00E94F30E8091C30608
:103550009091C4068937910528F08091C206C82F42
:10356000D0E002C0C0E0D0E082E06CE34EE70E9411
:10357000975E85E06CE143E20E949B5E1BE0812F39
:103580006BE343E00E949B5E1A5F1338C1F716E0BD
:103590000CE3FE01E65BF94F4081602F641B812F35
:1035A0000E949B5E2196C837D10510F0C0E0D0E0A4
:1035B0002091C20630E0C217D30719F01F5F1E37F3
:1035C00041F7DF91CF911F910F9108951F93182F0D
:1035D0008DE698E00E94441A1236E1F0133628F482
:1035E000103631F01136E9F418C01336D1F415C095
:1035F0008FEF97E090930D0180930C011092C60617
:103600001092C5061092C8061092C70687E10E9464
:10361000B56D07C08BE49AE102C08FE49FE30E947E
:10362000331588E06EE578E00E94115E4091C50692
:103630005091C6065695479584E568E00E943D6026
:1036400080E16FE478E00E94115E40910C0150919E
:103650000D015695479584E560E10E943D6088E143
:1036600060E478E00E94115E4091C5065091C60664
:1036700080910C0190910D01481B590B569547956F
:1036800084E568E10E943D6080E267E378E00E94A3
:10369000115E2091C7063091C80684E690E0289F0D
:1036A000A001299F500D389F500D1124A4E056957C
:1036B0004795AA95E1F784E560E220E30E942D603A
:1036C00088E26FE278E00E94115E0E94FF18AC0170
:1036D0008FE368E20E941D5E82E168E34DE158E0FD
:1036E0000E94195E1F91089581EE9FE008950F9347
:1036F00093E0499FA00111244652504F01E022233C
:1037000009F400E023E00E94BA5D0F9108950F9341
:1037100093E0499FA00111244D52504F01E0222314
:1037200009F400E023E00E94BA5D0F910895FF9232
:103730000F931F93F82E062F142F80E860E0402F80
:1037400050E0212F0E942D600A3010F00FE601C0DA
:1037500005E7802F60E04FE2212F0E94F75C4F2D9C
:1037600050E04F5F5F4F802F60E0212F0E942D605F
:103770001F910F91FF9008956F927F928F929F9269
:10378000AF92CF92DF92EF92FF920F931F93CF935E
:10379000DF93EC01162FD42E49016090F90470904C
:1037A000FA048091C8089091C9088619970920E405
:1037B00030E0B9010E947F74462F60932305E091A9
:1037C000FB04F091FC048091C6089091C7088E1B01
:1037D0009F0BB9010E947F74862F609324054423B8
:1037E00021F07092C9086092C808882321F0F093F4
:1037F000C708E093C60880912205882321F48091B0
:103800008A0185FF06C010922305109224051092AC
:10381000220560912305662351F4809124058823B5
:1038200031F480919C0490919D04009781F0409127
:103830008C0150E024EF31E0429FC001439F900D86
:10384000529F900D11249093A00480939F048114A3
:10385000910409F456C08881882309F04BC066237F
:1038600031F180912005882311F5ED2DE61BE7FD50
:10387000E0E0202F30E08E2F992787FD909582176A
:10388000930714F0E02FE150FF27E7FDF0958D2D11
:1038900090E0E817F90749F0EE0FFF1FE80DF91D5A
:1038A00025913491C9010E943315109223051536D4
:1038B00041F4DD2011F0ED2D01C0E02FF0E0319753
:1038C0000FC01436C9F42D2D30E0802F90E0019701
:1038D000281739071CF4ED2DEF5F01C0E0E0F0E0A0
:1038E000EE0FFF1FE80DF91D25913491C9010E94CB
:1038F000331502C040E001C041E08D2D602F0E94D1
:10390000971BE114F10451F098818C2D9C1508F45B
:10391000892FF701E80FF11D549101C050E080910B
:103920002005882309F04FC080912405882329F1C0
:103930004881481B47FD40E0242F332727FD309561
:103940008A2D90E0281739070CF04A2D4883898189
:10395000E114F10459F0C41608F44C2DF701E40FFA
:10396000F11DE4918E1718F4E82F01C0E0E0E9831F
:1039700080E68093D90D109224058881882319F15F
:10398000909123059923F9F04981E114F104B1F0F4
:10399000491B47FD40E09C2D8C1508F4982FF7013A
:1039A000E90FF11DE491242F332727FD30958E2F49
:1039B00090E0281739071CF04E2F01C040E04983E2
:1039C00080E68093D90D103651F1113690F41334FE
:1039D00009F480C0143430F4113279F1123409F052
:1039E0009CC06AC0143409F43FC0153409F095C076
:1039F0004FC01436E9F1153638F4123609F45FC0B9
:103A0000133609F08AC069C01138A1F01F3B21F0BC
:103A1000153609F082C040C01982188212C05523A1
:103A200009F47BC081E090912005911180E08093A2
:103A3000200573C0109220050DC0809120058823B9
:103A400019F01092200569C08881882319F081142B
:103A5000910421F480E00E940E155FC087E10E946E
:103A6000B56D1982188256C08981851709F455C031
:103A7000E114F10409F451C080912005882309F074
:103A80004CC08981851710F48F5F12C0198242C023
:103A90008981882309F441C0E114F10409F43DC08F
:103AA000809120058823C9F58981882319F08150E8
:103AB000898330C059832EC088818A1571F1809125
:103AC0002005882351F588818A1510F48F5F0DC079
:103AD00018820EC08881882301F1809120058823F7
:103AE000E1F48881882319F08150888301C0A8827D
:103AF0008981E114F10461F098819C1508F4C92EC4
:103B0000EC0CF11CF7019491891718F4982F01C05F
:103B100090E0998380E68093D90DDF91CF911F913A
:103B20000F91FF90EF90DF90CF90AF909F908F908C
:103B30007F906F9008954F925F926F927F928F92D5
:103B40009F92AF92BF92CF92DF92EF92FF920F932C
:103B50001F93DF93CF930F92CDB7DEB7D82E85E6B4
:103B60009AE00E94441A8AE498E06D2D41E024EE28
:103B700037E006E05DE6E52E5AE0F52E15E0C12EB1
:103B8000B6E0AB2E0E94BC1B80904A0890904B0878
:103B90008091630081FF07C08AE268E14FE55AE047
:103BA0000E94195E60C182E168E040E55AE00E942F
:103BB000195E8A9480912005882319F0A2E0CA2E0C
:103BC00002C0CC24C394EE24FF2410E1A82CBB2413
:103BD000A7FCB094F4E06F2E712C2701440C551C07
:103BE0008EE791E0480E591E4E2D4F5F80E0612F09
:103BF00020E00E94780FAE14BF0411F491E0911000
:103C000090E0F2012181229526952695237030E0DF
:103C1000A901440F551F420F531F4A5B554F99236B
:103C200011F400E001C00C2D88E1612F23E099839D
:103C30000E94BA5D99819923C1F080912005882363
:103C4000A1F0F201618162956695669563708D2D94
:103C500040E022E00E94F5148295880F880F807C56
:103C6000F20191819F73982B9183AE14BF0421F4CC
:103C700001E0F92DF13009F000E0F2018181880FB7
:103C8000880F85958595FDE08F02C0011124B30151
:103C90000E947F74AB01002311F420E001C02C2DA1
:103CA00082E4612F0E942D600023A9F080912005FD
:103CB000882389F0F2016181660F660F659565952D
:103CC0008D2D41EE2FE10E94F5148F73F201918149
:103CD000907C982B9183AE14BF0421F491E0F92DD0
:103CE000F23009F090E0F2012081277030E0A90164
:103CF000440F551F420F531F475C554F992311F432
:103D000000E001C00C2D88E4612F23E099830E941C
:103D1000BA5D9981992391F080912005882371F0F3
:103D2000F201608167708D2D40E023E00E94F51460
:103D30008770F2019081987F982B9083AE14BF0416
:103D400021F401E0F92DF33009F000E0F2014081A7
:103D5000459545954595002311F420E001C02C2D93
:103D60008AE5612F0E94C40F0023B1F080912005E5
:103D7000882391F0F20160816595659565958D2D9B
:103D80004AEE26E10E94F514880F880F880FF20191
:103D900090819770982B9083185F0894E11CF11C18
:103DA000103309F01ACF80E36EE27AE00E94115ED0
:103DB00040918E01552747FD5095465F5F4FF82D86
:103DC000F43011F421E201C020E28EE460E30E94AD
:103DD0002D60282D243049F48D2D60918E0146EF01
:103DE00028E20E94F51480938E01EE24E394882D3E
:103DF000853009F0EE2480E068E34AE25AE02E2D97
:103E00000E94EA5D46EAA42E44E0B42E06E711E0E3
:103E100090E3F501419151915F01F80121913191B8
:103E20008F01421B530B440F551F892F68E320E27B
:103E300099830E942D609981985E903951F7EE2008
:103E400091F0FD2DF03679F4A6E7B1E0E6EAF4E072
:103E500088E001900D928150E1F781E00E94DB57EC
:103E600087E10E94B56D0F90CF91DF911F910F9167
:103E7000FF90EF90DF90CF90BF90AF909F908F908A
:103E80007F906F905F904F900895AF92CF92EF9296
:103E9000FF920F93AE2CEE24FF24CC240E94BC1B77
:103EA0000F91FF90EF90CF90AF900895EF920F9306
:103EB000DF93CF930F92CDB7DEB7682F83E79AE0F9
:103EC00069830E94441A8CE498E0698142E024EE00
:103ED00037E006E0EE240E94451F80E167E677E0C8
:103EE0000E94115E88E164E377E00E94115E80E247
:103EF00067E477E00E94115E88E268E577E00E945F
:103F0000115E80E367E777E00E94115E0F90CF912A
:103F1000DF910F91EF900895CF92DF92EF92FF9291
:103F20000F931F93DF93CF9300D0CDB7DEB7682FE9
:103F300082EA9AE069830E94441A8EE498E06981DB
:103F400043E024EE37E006E0EE240E94451FEEE059
:103F5000CE2ED12C00E010E0143020F078EFF72EB8
:103F6000F00E01C0F02EC6010E949761E82E1F5F7F
:103F70008AE26F2D412F20E00E94C40F4E2D405D3C
:103F800084E46F2D2E2D0E94F75C085F0894C11CFD
:103F9000D11C193009F708E3CC24DD2410E0812F6F
:103FA00090E00E949761F82EA6014D57554F80E092
:103FB000602F25E00E94E45D4F2D405D80E2602F80
:103FC0002F2D0E94F75C1F5F85E090E0C80ED91E80
:103FD0000850163021F784E568E14BE75AE027E006
:103FE0000E94E45D66E0E62EF12C10E230E084E50C
:103FF000612F45E857E0232F00E03A830E94985C48
:10400000C7010E949761282FC701019629830E944A
:104010009761082F2981422F405D8CE6612F0E9415
:10402000F75C402F405D88E7612F202F0E94F75CEE
:104030003A813F5F185FE2E0F0E0EE0EFF1E3430A1
:10404000B1F60F900F90CF91DF911F910F91FF90DC
:10405000EF90DF90CF9008958F929F92AF92BF9292
:10406000DF92EF92FF920F931F93CF93DF93D82E9F
:104070008AEA9AE00E94441A80E598E06D2D44E0B7
:1040800024EE37E006E0EE24E3940E94451FF09012
:104090005008C1EFD4E010E000E0812CF4E09F2E46
:1040A000A12CB12C88E1612F41E40E94B65D402F24
:1040B0004F5C8EE1612F0E94B65D802F0E94D51566
:1040C000AC018AE2612F0E941D5E0730B1F0688169
:1040D0007981882777FD8095982F24E630E040E0AD
:1040E00050E00E944074A50194010E94B4748AE5D6
:1040F000612FA9010E943D600AC08F2D813011F00F
:1041000040E201C041E28AE5612F0E94720F0F5F19
:10411000185F2296083031F68CE668E247EA5AE0EA
:1041200022E00E94E45D4091090150910A0188E774
:1041300060E320E00E942D608F2D813059F4F092D1
:1041400022058D2D6091740141E82FE70E94F5143E
:1041500080937401DF91CF911F910F91FF90EF90A9
:10416000DF90BF90AF909F908F900895EF920F9344
:10417000E42E40E020E030E000E00E94451F0F9177
:10418000EF900895AF92BF92CF92DF92EF92FF929D
:104190000F931F93DF93CF9300D0CDB7DEB78FE19E
:1041A00061E247E10E949B5E8FE167E347E10E9485
:1041B000975E85E361E247E10E949B5E8FE161E2E9
:1041C00047E10E94975E8BE461E247E10E949B5EBB
:1041D0008BE467E347E10E94975E81E661E247E195
:1041E0000E949B5E8BE461E247E10E94975E8AE257
:1041F0006BE243E00E949B5E89E26CE243E00E9436
:10420000975E86E56BE243E00E949B5E85E56CE28B
:1042100043E00E94975E8091F1049091F20451E78F
:10422000C52ED12CB6010E947F74262F8091F304F5
:104230009091F4040FE81FEFB8010E947F74362FAD
:1042400048E2E42EE20E9AE2F92EF60E8E2D6F2D44
:1042500045E02A8339830E949B5E3981632F625D2A
:104260008E2D45E00E94975E2A81822F845D6F2DFE
:1042700045E00E949B5E8E2D6F2D45E00E94975E6B
:104280008091F7049091F804B6010E947F74262F64
:104290008091F5049091F604B8010E947F74062F76
:1042A00084E5F82EF20E162F165D8F2D612F45E056
:1042B0002A830E949B5E602F625D8F2D45E00E94E5
:1042C000975E2A81822F885A612F45E00E949B5E6B
:1042D0008F2D612F45E00E94975E19EFA12E14E00B
:1042E000B12EBAE3FB2E0DE510E0A8E3EA2EF501AE
:1042F000819191915F0180509C4FB8010E947F7421
:10430000D62ED394CE2CCD188F2D6C2D4D2D0E94F2
:104310009B5E8F2D8F5F6C2D4D2D0E949B5E8F2D90
:104320008E5F6C2D4D2D0E949B5EF5E0FF0E8F2D54
:104330008934E9F60F900F90CF91DF911F910F9183
:10434000FF90EF90DF90CF90BF90AF9008954F9285
:104350005F926F927F928F929F92AF92BF92CF9215
:10436000DF92EF92FF920F931F93DF93CF930F9201
:10437000CDB7DEB7B82E8FEF9AE00E94441A8DE7D2
:1043800098E06B2D45E024EE37E006E0EE24E39460
:104390000E94451F10927D0811E6E12E18E0F12ED3
:1043A000B3E5CB2EB8E0DB2E8601470160E0862F17
:1043B00069830E94D515D4014D915C911197282FE6
:1043C000392F6981421753070CF49A01F4012193A4
:1043D00031934F01D8014D915C911197282F392FBE
:1043E000241735070CF49A01F801219331938F01BA
:1043F0006F5F6730E1F68091520880932205FB2DB4
:10440000F03219F0FF3B71F40BC08F5F80935208BC
:10441000833041F487E10E94B56D81E00E94DB5753
:1044200010925208809152088130B1F0813020F012
:10443000823009F0A4C03FC08CE060E14DEE5AE04C
:1044400021E100E00E94BA5D82E168E14DED5AE0B1
:104450002FE00E94BA5D93C08EE160E140ED5AE02A
:104460002CE000E00E94BA5D82E168E14EEA5AE089
:1044700020E10E94BA5DAFE68A2EA8E09A2E20E0E5
:1044800008E91AE3F8E6AF2EF5ECBF2ED7010D933D
:104490001D937D01F601A192B1926F01822F2983B4
:1044A0000E94D515D4018D939D934D0129812F5FD5
:1044B000273061F764C082E160E14FEB5AE020E110
:1044C00000E00E94BA5D82E168E14EEA5AE020E134
:1044D0000E94BA5DEFE6AE2EE8E0BE2E75E4472EF0
:1044E00071E0572EF20160E4862E912CD7018D9158
:1044F0009D917D01D6016D907D906D019C012619E5
:10450000370937FF03C0309521953F4F23333105DD
:10451000DCF0D5012D913C91318320838901081B6A
:10452000190BC801B4010E947F74061B170B178773
:104530000687C301821B930B9C01B4010E947F7408
:10454000261B370B358F248FA2E0B0E0AA0EBB1ECE
:104550003296BFE6EB16B8E0FB0641F680E090E04D
:10456000F201219131912F01820F931FFDE54F162A
:10457000F1E05F06A9F79093700180936F010E94AC
:10458000C2200F90CF91DF911F910F91FF90EF907C
:10459000DF90CF90BF90AF909F908F907F906F9063
:1045A0005F904F900895282F30E0C901880F991F20
:1045B000A90163E0440F551F6A95E1F7840F951F29
:1045C000A9014F5F5F4FBA01660F771FA3E0440F49
:1045D000551FAA95E1F7640F751F62547E4F209511
:1045E0003095205E3F4FA901440F551FE3E0220F95
:1045F000331FEA95E1F7420F531F82549E4F0E94EA
:10460000E4748AE0E4EFF2E0DF011D928A95E9F7B5
:1046100082E00E94DB570E94775808950F931F9302
:10462000CF93DF93282F30E0E901CC0FDD1FC901C4
:1046300013E0880F991F1A95E1F7C80FD91F8E0153
:1046400002541E4FA9014F5F5F4FCA01880F991F87
:10465000A3E0440F551FAA95E1F7840F951F2095FD
:104660003095205E3F4FA901440F551FE3E0220F14
:10467000331FEA95E1F7420F531F82549E4FB80152
:104680000E94E4748AE0D8011D928A95E9F780912E
:10469000A108CC55DE4F8A8F8B8F84E68C8F82E009
:1046A0000E94DB570E947758DF91CF911F910F91A5
:1046B0000895FF920F931F9385EFE5E4F5E0DF0186
:1046C0001D928A95E9F780913A06AEEBB1E050E091
:1046D00021E030E060E07C91772311F0472F01C0AA
:1046E00040E1641738F5F22E032F162F1F5F802F3D
:1046F00090E0FC01EE0FFF1FEE0FFF1FE80FF91F08
:10470000EB5BFA4F912F9F738081807C892B8064B3
:104710008083F182F39453830F5F141738F3962F3D
:104720009095642F822F8F5F890F390F340F290FD7
:10473000240F840F772359F1832F90E0FC01EE0FB3
:10474000FF1FEE0FFF1FE80FF91FEB5BFA4F4F73D0
:104750008081807C5483842B8068808322832F5FB8
:104760001A968C911A97781719F41182138205C042
:1047700021832F5F852F8F5F8383822F5F5F1A9640
:10478000503219F420933A0604C03F5FA4CF8093BF
:104790003A061F910F91FF900895EEEBF1E080E053
:1047A00090819150903108F48F5F3A9692E0EE3FFD
:1047B000F907B1F708951F93182F80E16DEE7DE0A2
:1047C0000E94115E0E94CD23482F88E760E150E0EF
:1047D00020E00E942D6080E267ED7DE00E94115E86
:1047E000113651F481E60E94F66181E00E940E15B7
:1047F0008BE994E20E9443151F9108950E94CD23F6
:10480000803230F08BED93E20E94431581E00895F1
:1048100080E00895EF92FF920F931F93DF93CF9361
:1048200000D0CDB7DEB7182F813208F07BC08823C7
:1048300019F4442341F476C0803219F4442331F052
:1048400071C0442319F0012F0F5F02C0012F0150E6
:10485000812F4A8369830E94D70E7C01802F0E949A
:10486000D70EFC01D7018C91982F91504A81698114
:10487000903108F057C02081213108F053C06623E1
:10488000A1F10E94FE23882309F04CC0212F30E0C3
:10489000A9014F5F5F4FCA01880F991F13E0440FB2
:1048A000551F1A95E1F7840F951FB901660F771F01
:1048B000A901A3E0440F551FAA95E1F7640F751FE6
:1048C00062547E4F20953095205E3F4FA901440FE2
:1048D000551FE3E0220F331FEA95E1F7420F531F04
:1048E00082549E4F0E94E4741DC0281759F044233F
:1048F00031F08031B8F48F5FF701808313C0D701A6
:104900009C9310C0D701CF010A9604C020813C912E
:1049100031932D93E817F907C9F782E00E94DB571E
:104920000E9477580F900F90CF91DF911F910F91B8
:10493000FF90EF9008956F927F928F929F92AF9227
:10494000BF92CF92DF92EF92FF920F931F93CF937C
:10495000DF93182F81ED9DE00E94441AE0903A0603
:10496000EA9484EA98E0612F44E020ED37E00AE021
:104970000E94451FC090A408CC2011F41092A308F7
:104980001236D9F1133670F41334A9F1143420F42B
:10499000123409F070C031C01036C1F0113609F080
:1049A0006AC045C0103809F452C0113820F41336DB
:1049B00009F061C020C01E3BB9F11F3B09F05BC08C
:1049C00081E08093A2081092A3082EC01C143CF42E
:1049D00081E09091A308911180E08093A3088091D9
:1049E000A3088093A20880919F08882309F443C0FC
:1049F0001092A30840C01092A2088091A3088823B7
:104A0000D1F141E0123609F040E08091A0086091B8
:104A1000A2080E940A248091A208882319F0133664
:104A200009F4CA941092A2080E94592324C08091CC
:104A3000A308882301F18091A0080E94D32210923C
:104A4000A3080E94592381E60E94F66114C01C1439
:104A500094F480919F08882341F00E94FE238823CC
:104A600021F48091A0080E940E231092A30881E5F2
:104A700092E50E94431538E0D32E77247A9423E6FA
:104A8000822E9924BB24BA9466246394E0901F0577
:104A9000E90CFF24F701EE0FFF1FEE0FFF1FEE0DD5
:104AA000FF1DEB5BFA4F4081842F807C09F462C1CB
:104AB00046FF06C04F7380E06D2D20E00E94A40FDA
:104AC0001C14E4F4E701CC0FDD1FCC0FDD1FCE0D6D
:104AD000DF1DCB5BDA4F8981C81681F46D2D695FCC
:104AE00080E048E10E94975E8B818093A0088881D6
:104AF0008F738093A10860929F08B92CF701EE0F85
:104B0000FF1FEE0FFF1FEE0DFF1DEB5BFA4F8081C5
:104B100087FF05C19481C92FDD27C7FDD095AA2441
:104B2000A3949281C912AA2486FD1FC0FE01EE0F34
:104B3000FF1FCE01A3E0880F991FAA95E1F7E80FA8
:104B4000F91FEB53FE4F40814695477050E04353A9
:104B5000524F8091A308882311F400E001C00A2D70
:104B600082E16D2D21E00E94BA5DFE01EE0FFF1F74
:104B7000CE0163E0880F991F6A95E1F7E80FF91FEE
:104B8000EC55FE4F448D552747FD50958DE26D2D18
:104B90002A2D0E942D608091A308882311F420E023
:104BA00001C02A2D8DE26D2D45E20E94F75CFE01C9
:104BB000EE0FFF1FCE0143E0880F991F4A95E1F7E2
:104BC000E80FF91FEC55FE4F438D8091A308882311
:104BD00011F420E001C02A2D86E36D2D0E94780F8C
:104BE000FE01EE0FFF1FCE0123E0880F991F2A95CB
:104BF000E1F7E80FF91FEC55FE4F458D442359F0BE
:104C00008091A308882311F420E001C02A2D8EE4AE
:104C10006D2D0E94C40FFE01EE0FFF1FCE01B3E009
:104C2000880F991FBA95E1F7E80FF91FEC55FE4F71
:104C3000468D442391F023E0429FA00111244F515F
:104C4000504F8091A308882311F400E001C00A2D81
:104C500086E66D2D23E00E94BA5DFE01EE0FFF1F78
:104C6000CE0173E0880F991F7A95E1F7E80FF91FDD
:104C7000E254FE4F21E08581882309F420E0FE0103
:104C8000EE0FFF1FCE0153E0880F991F5A95E1F7F1
:104C9000E80FF91FE254FE4F8681882329F0222372
:104CA00009F498C04AE203C0222361F044E48091F1
:104CB0002005882311F420E001C02A2D89E76D2DFD
:104CC0000E94F75C8A2D813051F55E01AA0CBB1C55
:104CD00033E0CC0FDD1F3A95E1F7AC0EBD1EE4EAE0
:104CE000F1E0AE0EBF1E812FF501648D43E82DE784
:104CF0000E94E614F501848FF701EE0FFF1FEE0FFF
:104D0000FF1FEE0DFF1DEB5BFA4F84818093A0081F
:104D100080818F738093A10810929F08B92CF701AE
:104D2000EE0FFF1FEE0FFF1FEE0DFF1DEB5BFA4FA7
:104D30008181882331F088150CF4882E87150CF0BA
:104D4000782EF701EE0FFF1FEE0FFF1FEE0DFF1D78
:104D5000EB5BFA4F8281882331F088150CF4882EA2
:104D600087150CF0782E9394F8E0DF0E292D27306C
:104D700009F08CCECC20A1F08B2D8F3FF9F4C81414
:104D800064F480911F0590E00197EFEF8F3F9E073D
:104D900011F480E090E080931F057C14ECF414C0C3
:104DA000FB2DFF3F59F480911F0590E001972FEFF5
:104DB0008F3F920761F480E090E009C08B2D863030
:104DC0005CF0992D983040F080911F058F5F8093A3
:104DD0001F0502C043E56BCFDF91CF911F910F916B
:104DE000FF90EF90DF90CF90BF90AF909F908F900B
:104DF0007F906F9008952F923F924F925F926F92A3
:104E00007F928F929F92AF92BF92CF92DF92EF925A
:104E1000FF920F931F935C01CC24DD243B01882477
:104E2000992464E6262E312C412C512CC201B1016B
:104E30006619770988099909A60195010E944074AD
:104E40007B018C0182E390E0A0E0B0E0E80EF91E67
:104E50000A1F1B1FC601B5010E9440740E944074C6
:104E6000BC0188279927A40193010E94407444E063
:104E700096958795779567954A95D1F7E60EF71E33
:104E8000081F191FC801B701A20191010E94927465
:104E9000C9011F910F91FF90EF90DF90CF90BF90CD
:104EA000AF909F908F907F906F905F904F903F90CA
:104EB0002F9008951F93CF93DF939C016115710587
:104EC00011F1132F111F1127111F19F03095219582
:104ED0003F4F77FF0EC0C0E0D4E0709561957F4FE3
:104EE000CE01821B930B0E94FB269E01281B390BCF
:104EF00005C0C9010E94FB26282F392F112319F064
:104F0000309521953F4FC901DF91CF911F910895B1
:104F10006F927F928F929F92AF92BF92CF92DF92C9
:104F2000EF92FF920F931F93DF93CF93CDB7DEB72E
:104F3000982E962F322F802F6E2D222359F0442346
:104F400061F440919C0450919D044115510539F440
:104F500021E001C020E0FF2405C022E001C021E0E3
:104F6000FF24F394332311F0911121E04A2D4336AD
:104F700079F44C2D50E0440F551F8A0173E0000F67
:104F8000111F7A95E1F7041B150B065A1C4F11C02F
:104F9000FA2DF236D9F44C2D50E0440F551F8A01FA
:104FA00093E0000F111F9A95E1F7041B150B055AAA
:104FB0001C4FF80140810E94C40FFF2009F463C018
:104FC000F8016081892D4AEE26E159C0698877246D
:104FD000BB24882051F54C2D50E0440F551F6A0129
:104FE000B3E0CC0CDD1CBA95E1F7C41AD50AAA0CC3
:104FF000BB1CAA0CBB1CCA0CDB1CC60CD71C4EE489
:1050000053E0C40ED51EF6014081552747FD50954B
:105010000E942D60FF20B9F1F6016081892D4CE9D5
:1050200024E60E94E614F6012DC0DD24AA0CBB1C68
:10503000A601E3E0440F551FEA95E1F74C195D091D
:10504000A40EB51EA80CB11CAA0CBB1CF301EA0DE2
:10505000FB1DE25BFC4F4081552747FD50954C59A5
:105060005F4F0E942D60FF2071F08501060D171D16
:10507000025B1C4F892DF80160814CE920E00E9401
:10508000E614F8018083CF91DF911F910F91FF907B
:10509000EF90DF90CF90BF90AF909F908F907F90D8
:1050A0006F9008952F923F924F925F926F927F92EE
:1050B0008F929F92AF92BF92CF92DF92EF92FF9228
:1050C0000F931F93DF93CF93CDB7DEB72A970FB619
:1050D000F894DEBF0FBECDBFD82E84EC9DE00E94B9
:1050E000441A8DE998E06D2D40E020E030E000E0CA
:1050F0007CECE72E7DE0F72ECC2453E0A52E0E9419
:10510000BC1B409195084F5F80E360E020E00E9467
:10511000780FF0909D088091950890E0880F991F76
:10512000FC0123E0EE0FFF1F2A95E1F7E81BF90BC6
:10513000E65AFC4F808160E040E00E94A210882384
:10514000C1F08091950890E0880F991FFC0113E051
:10515000EE0FFF1F1A95E1F7E81BF90BE55AFC4F1C
:10516000808160E040E00E94A210882321F411E0D9
:1051700003C010E001C012E060919508462F50E096
:10518000FA01EE0FFF1FEF50FB4F808191818A31B2
:1051900091051CF010929C0807C02FEF873E9207E4
:1051A0001CF481E080939C082091880130E02170FC
:1051B000307082E090E0821B930B8417950741F4D6
:1051C000643030F48091B501807F11F010929C081A
:1051D00080E16FEB7DE00E94115E0F92EDB7FEB7AC
:1051E000319621E0F11020E080919C0880838D2D84
:1051F00061E041E006E3A0E1EA2EC0909508A12E0F
:1052000088240E9488270F9088E168EB7DE00E9447
:10521000115E0F92EDB7FEB7319621E03F2D313090
:1052200009F020E080919C0880838D2D61E041E0B1
:1052300006E3F8E1EF2EC0909508A12E8824839410
:105240000E9488270F9080E262EB7DE00E94115E51
:105250000F92EDB7FEB7319621E08F2D823009F025
:1052600020E010828D2D61E041E00EE1E0E2EE2EC3
:10527000C090950873E6A72E88240E9488270F9077
:1052800088E26CEA7DE00E94115E0F92EDB7FEB7F6
:10529000319621E09F2D933009F020E010828D2D72
:1052A00061E041E00EE158E2E52EC090950832E65B
:1052B000A32E88240E9488270F90113019F01230F5
:1052C00049F404C080E365EA7DE007C080E36EE94D
:1052D0007DE003C080E366E97DE00E94115E0091FD
:1052E0009508402F50E0812F90E0880F991F880F7C
:1052F000991FBA01660F771F9B01B3E0220F331F7E
:10530000BA95E1F7261B370B820F931F8C559E4FE2
:10531000FC01E655FE4FA081A983FC01E555FE4F37
:10532000B081BA83FC01E455FE4F9080E4E69E0E06
:1053300083559E4FDC018C908E0E2091880130E0C9
:105340002170307082E090E0821B930B84179507E8
:1053500009F062C0043008F05FC08091B501807F21
:1053600009F45AC0EE24FF24870120E030E0B9811F
:105370006B2E772467FC7094A1E24A2E512C292CC5
:10538000332427FC3094F0E4CF2ED22ED801C7016D
:10539000B595A79597958795B30129873A870E9478
:1053A0005A27880F991FB2010E947F74629DC00125
:1053B000639D900D729D900D11246FE3A62EAD0C90
:1053C00064E670E00E946B74EC2DE61B6E2F8A2D54
:1053D0000E944B5E29853A85C901837090700097C1
:1053E00061F48A2D6FE30E944B5E6D2D6695605EC1
:1053F0008FE30E944B5E3A8529852F5F3F4F81E204
:1054000090E0A0E0B0E0E80EF91E0A1F1B1F2E334B
:10541000310509F0BACF7CC0DD249981492E55248D
:1054200047FC509401E210E0A92DBB27A7FDB095E1
:10543000BC83AB8354E6652E712C40E2A42EBA8166
:105440002B2E332427FC3094E82DFF27E7FDF09521
:10545000FE83ED83FD2D21E2F29F70011124C7012F
:10546000B2010E945A27B8010E947F74AB81BC81AF
:105470006A9FC0016B9F900D7A9F900D11243EE5AD
:10548000C32ECD0CB3010E946B74BA2DB61B6B2FCB
:105490008C2D0E944B5EED2DF0E0E370F070F887EC
:1054A000EF83309749F48C2D60E20E944B5E6D2DA6
:1054B000605E8EE50E944B5EC701B1010E945A27D3
:1054C000B8010E947F742D813E81629FC001639F5D
:1054D000900D729F900D11242EE5F22EFD18B30150
:1054E0000E946B74605E8F2D0E944B5E8F81988549
:1054F000009749F48F2D60E20E944B5E6A2D6D1972
:105500008EE50E944B5ED3949D2D9F3109F0A2CF72
:10551000E0919508F0E0EE0FFF1FEF50FB4F408049
:1055200051805201CC24B7FCC094DC2CC601B501DB
:1055300021E230E040E050E00E94B474822F825AB1
:1055400061E04EE30E949B5E4091950820918801A6
:1055500030E02170307082E090E0821B930B242FAA
:1055600030E08217930709F050C0443008F04DC076
:105570008091B501807F09F448C0C601B501605033
:105580007C4F8F4F9F4F22E030E040E050E00E9480
:10559000B474A9816A2F772767FD7095C9010E94AD
:1055A0005A27BC01660F771F882777FD8095982FB3
:1055B000292D97FC2D5F25952595332727FD3095BF
:1055C000432F532F0E94407429E130E040E050E027
:1055D0000E94B47479018A01CA01B9012FED3FEF2D
:1055E0004FEF5FEF0E94B474622F605C8FE34EE375
:1055F0000E94975EC801B70122E030E040E050E031
:105600000E94B47479018A013CC01A141B041C0462
:105610001D0414F4698101C06A81772767FD7095C4
:10562000C2010E945A279C01442737FD4095542F00
:105630001A141B041C041D0414F4692D01C0682DE8
:1056400067FD6D5F65956595772767FD7095872F79
:10565000972F0E94407429E130E040E050E00E9422
:10566000B47479018A01CA01B9012FED3FEF4FEF00
:105670005FEF0E94B474622F605E8FE34EE30E947E
:10568000975EC601B50129E130E040E050E00E949C
:105690004074612CB1E07B2E812C912CA4019301EC
:1056A0000E94B47482E760E3A90120E00E942D60AB
:1056B000C801B70129E130E040E050E00E944074A9
:1056C000A40193010E94B47484E568E0A90120E07C
:1056D0000E942D601A141B041C041D0474F4B9816B
:1056E0006B2F772767FD7095C20144970E945A2758
:1056F000F701E81BF90BCF010BC0FA816F2F772759
:1057000067FD7095C20144960E945A278E199F0921
:105710009C01220F331F220F331F280F391F4427EC
:1057200037FD4095542F84E560E100E3F3E0EF2E70
:105730000E94F75E2A960FB6F894DEBF0FBECDBF6B
:10574000CF91DF911F910F91FF90EF90DF90CF905D
:10575000BF90AF909F908F907F906F905F904F9091
:105760003F902F9008952F923F924F925F926F92A9
:105770007F928F929F92AF92BF92CF92DF92EF92E1
:10578000FF920F931F93DF93CF93CDB7DEB72F9781
:105790000FB6F894DEBF0FBECDBF982E8CE89DE00B
:1057A0000E94441A8AE998E0692D43E020ED37E031
:1057B0000AE0F4E9EF2EFDE0FF2ECC24C394E4E0F0
:1057C000AE2E0E94BC1BF0909A08FA9430909B0871
:1057D000292D203841F4F7FC06C0F092950882E5A7
:1057E00098E20E94431585E168E04CE75DE00E9485
:1057F000195E8AE593E09C838B8376E9472E78E0F7
:10580000572EE1EFF4E0FB87EA8710E16624772466
:105810002F2D332727FD30953A832983C901880F1F
:10582000991FFC0153E0EE0FFF1F5A95E1F7E81BAB
:10583000F90BFE83ED83F62CEB81FC81808160E027
:1058400040E00E94A210882361F0EB81FC818181FD
:1058500060E040E00E94A210882329F4BB24B394A6
:1058600004C0BB2402C042E0B42E2B2D30E03887A8
:105870002F83C901880F991F880F991FA301440F17
:10588000551F9A0103E0220F331F0A95E1F7241BED
:10589000350B820F931F8C559E4FDC01A355BE4FD5
:1058A000FC01E455FE4F3C912081321751F4FC017C
:1058B000E555FE4F86559E4F41E02081FC018081D9
:1058C000281340E0EA85FB8581919191FB87EA8767
:1058D0009C0197FF04C022273327281B390B2A314C
:1058E00031050CF040E0242E8A3191051CF0F201C4
:1058F000108207C0FFEF873E9F071CF421E0F201F2
:1059000020838091880190E081709070E2E0F0E067
:10591000E81BF90BE615F70551F48091B501807F7E
:1059200031F0F301EA56F74F1082222423944F2DD1
:105930004F5F80E0612F20E00E94780F5D864C86EB
:10594000F2013081F1E0F98731111986809120054B
:10595000882351F4DD24D39480919C0490919D047C
:10596000009721F4DD2402C0DD24D39489819A813B
:105970008615970511F421E0311020E00F92EDB764
:10598000FEB73183892D60E04D2D07E2E12ECF2C4B
:10599000AB2C88240E9488270F9029813A812615F4
:1059A000370509F0D2C0332009F0CBC0DD2009F45F
:1059B000CCC0222009F4C9C08F819885880F991F17
:1059C000880F991FED81FE818E0F9F1F8C559E4F72
:1059D000F9858F0F911D86559E4F9F878E87892D44
:1059E000EE85FF8560814CE924E60E94E614EE8591
:1059F000FF858083AAC021E00F92F2018081EDB77C
:105A0000FEB78183892D60E04D2D09E3E12ECF2C77
:105A1000AB2C882483940E9488270F9029813A8197
:105A20002615370509F097C0332D313009F08FC0A6
:105A3000DD2009F490C0222009F48DC08F81988563
:105A4000880F991F880F991FED81FE818E0F9F1F70
:105A50008C559E4FF9858F0F911D84559E4F9887C9
:105A60008F83892DEF81F88560814CE920E00E94C9
:105A7000E614EF81F88580836EC021E00F92EDB7C8
:105A8000FEB71182892D60E04D2D0FE3E12ECF2C62
:105A9000F3E6AF2E88240E9488270F9029813A814F
:105AA0002615370521F421E0332D333009F020E0AD
:105AB0000F92EDB7FEB71182892D60E04D2D07E5FD
:105AC000E12ECF2CE2E6AE2E88240E94882708948F
:105AD000411C511C0F90EC85FD858081882319F4B1
:105AE000222031F008C0222031F48AE34FE705C0BC
:105AF0008BE34EE702C08AE34DE2612F0E94B65D60
:105B0000FB2DF13019F0F23049F404C085E7612F24
:105B10004DE407C085E7612F4CE403C085E7612FA2
:105B200048E40E94B65D0894611C711C2B813C8185
:105B3000225F3F4F3C832B83185F103309F07BCEED
:105B40000CC0332D313009F456CF20E055CF832DD2
:105B5000823009F492CF20E091CF2F960FB6F894BF
:105B6000DEBF0FBECDBFCF91DF911F910F91FF9090
:105B7000EF90DF90CF90BF90AF909F908F907F90ED
:105B80006F905F904F903F902F90089520E030E00D
:105B9000F901E75CF24FE491E81711F4822F0895C0
:105BA0002F5F3F4FEE23A1F780E00895823430F459
:105BB000E82FF0E0E75CF24F8491089580E20895C9
:105BC000EF92FF920F931F93182FF62EE22E862F3F
:105BD000BA010E94115E86E66F2D412F2E2D0E9484
:105BE000771BEE2039F0802F612F40E021E00E94EA
:105BF000F514182F812F1F910F91FF90EF900895AA
:105C0000FF920F931F93F82E1091AF01212F33278E
:105C100027FD309537FF03C0309521953F4F022F68
:105C200025320CF43DC02091440830914508809104
:105C3000420890914308282B392B80914608909177
:105C40004708282B392B8091410890E0282B392BCD
:105C500040913E0850E0242B352B2115310531F4BD
:105C6000812F881F8827881F80933E0811161CF4F7
:105C7000812F845202C0812F8C5D60E040E00E9441
:105C8000A210882359F090913E08992339F491E0AD
:105C900020914108211190E09093410880933E08A3
:105CA00020914408309145082F5F3F4F30934508BD
:105CB0002093440820914208309143082F0D311D54
:105CC00030934308209342080E94CF0E209146084B
:105CD00030914708821B930B8436910508F471C1FB
:105CE0002C593F4F30934708209346082091420893
:105CF00030914308E0914408F0914508C901BF0183
:105D00000E946B74F62E462F50E04E9FC0014F9FAD
:105D1000900D5E9F900D1124281B390B3093430882
:105D200020934208109245081092440800311CF458
:105D3000109241080FC005326CF411161CF4812F2B
:105D40008F5002C0812F815F60E040E00E94A2106E
:105D50008093410880913D0690913E060196909374
:105D60003E0680933D0640913F06509140064F5FAE
:105D70005F4F5093400640933F06FF2049F08091CB
:105D800043069091440601969093440680934306FF
:105D900080914108882349F0809141069091420604
:105DA00001969093420680934106F6942091450611
:105DB000309146062F0D311D30934606209345063F
:105DC0008091B1019091B201909349068093480669
:105DD0006091AF01772767FD709577FF03C07095DD
:105DE00061957F4F662319F4109247061EC06130FB
:105DF00019F4841B950B15C0603168F460FF06C070
:105E0000A4E036952795AA95E1F709C020914306AD
:105E10003091440604C02091410630914206821B15
:105E2000930B9093490680934806809147068130F2
:105E300051F0813018F0823049F514C08091AF01E3
:105E4000882321F120C080914806909149061816B8
:105E50001906E4F08091B1019091B2010097B1F080
:105E600082E012C080914806909149062FEF853C50
:105E700092071CF483E0809347068091B1019091D2
:105E8000B201009719F481E080934706809148069B
:105E90009091490620913F08309140082817390712
:105EA00009F479C020914706213009F065C020919E
:105EB0008A0122FF45C02091B1013091B201211524
:105EC0003105F1F18E31910519F489E10E94B56D2A
:105ED00080914806909149068431910519F48AE130
:105EE0000E94B56D80914806909149068A309105CF
:105EF00019F48BE10E94B56D809148069091490696
:105F0000843091051CF48CE10E94B56D80918A016A
:105F100083FF16C080914806909149068E31910505
:105F200049F08431910531F08A30910519F08430BF
:105F3000910534F482E390E09093A00480939F0451
:105F400080918A0181FF27C08091B001209148068D
:105F50003091490680FF07C08091B1019091B20154
:105F6000821B930B01C0C9016CE370E00E946B744B
:105F7000009789F480E003C0223069F48CE10E942C
:105F8000B56D80918A0183FF06C082E390E0909313
:105F9000A00480939F0420914806309149063093D5
:105FA000400820933F088091B00180FF0AC0809193
:105FB000B1019091B201821B930B9093490680939B
:105FC00048061F910F91FF9008958091AF01992786
:105FD00087FD909597FF03C0909581959F4F982FCF
:105FE000823034F1803124F585959A3024F40E9472
:105FF0001A6390E003C0992787FD90950197FC01F3
:10600000EE0FFF1FEF50FB4F208131818091AF01D8
:1060100087FF05C080E094E0821B930B03C0C90199
:1060200080509C4F26E0969587952A95E1F702C00F
:1060300080E090E00E94002E83E00E941A63E82F27
:10604000F0E0EE0FFF1FE151FB4F80819181805006
:106050009C4FB6E096958795BA95E1F72091B001EF
:1060600022FF0AC08530910538F02091A204222336
:1060700019F423E02093A20420913A0830913B08C0
:106080002F5F3F4F30933B0820933A082091380808
:1060900030913908280F391F309339082093380878
:1060A0000E94CF0E20913C0830913D08821B930B3B
:1060B00023E0883E9207E8F10E94CF0E90933D08BE
:1060C00080933C088091B301823051F485E160E017
:1060D00040E00E94A210882319F087E00E94B56D6D
:1060E000809138089091390860913A0870913B0886
:1060F0000E946B74109239081092380810923B0875
:1061000010923A088091C3069091C406019690932C
:10611000C4068093C3068091C206E82FF0E0E65BD8
:10612000F94F60838F5F8093C206883710F010921A
:10613000C2060895109247061092400610923F063C
:1061400010924406109243061092420610924106A5
:10615000109246061092450608950F931F93182F2C
:1061600080913B06882319F069E27DE002C06CE172
:106170007DE088E00E94115E81E060E144EA51E048
:106180002AE000E10E94BA5D82E460E14FE30E94F0
:10619000B65D82E168E245E15DE00E94195E82E160
:1061A00060E346E05DE00E94195E113609F44AC0E2
:1061B0001F3B21F0103609F04FC004C080E00E9460
:1061C000B56D4AC080913B068823A9F084EF9CE01E
:1061D0000E94D81280913C060E944357882339F0D0
:1061E00087E10E94B56D82E080933B0629C080E084
:1061F0000E94B56D25C0809171018F5F0E94075A82
:106200001091710108C01150113108F01FE0809108
:106210007101181739F0812F8F5F0E94BA598823B6
:1062200091F301C010E01093710181E00E94DB57EF
:106230000E947758809171010E940C570E949A30F9
:1062400080E601C081E60E94F66181E00E940E15A1
:106250008FE291E30E9443151F910F910895AF9231
:10626000BF92DF92EF92FF920F931F93CF93DF9332
:10627000182F80E19BE00E94441A8091200588231A
:10628000A1F4E0912305E7FF10C0E195EA3008F0A2
:10629000E9E0F0E0EE0FFF1FE053F84F2591349155
:1062A000C9010E94331510922305F0908F088FE8E2
:1062B00098E0612F4FE00E94B62086E360E04BE05B
:1062C0005BE00E94195E0E94FC58AC0186E660E02B
:1062D00020E00E942D6080E06AE041E00E94971B70
:1062E000D0908F0880913B06823021F410928E0866
:1062F00010923B06163648F4143690F5103609F421
:1063000056C0113609F075C00AC0113809F456C0DC
:106310001F3B09F465C0103809F06BC053C0809171
:106320008E088823E9F010928E0887E10E94B56DEF
:1063300081E60E94F6610E94775880918F088093D1
:1063400071010E940C570E949A3081E00E94DB5735
:106350000E94775882E00E94DB570E94775849C01C
:10636000809171018D15B9F0812F0E94F6618091A5
:106370008F08809371010E947758809171010E946B
:106380000C570E949A3081E00E94DB570E94775898
:1063900081E00E94B56D153619F481EA90E504C0DC
:1063A000143639F58AE693E40E94331522C081E061
:1063B00080938E0887E10E94B56D1BC081E00E942A
:1063C0000E1517C080918E08882399F081E0809384
:1063D0003B06D0923C068DEA90E30E94431509C02B
:1063E00010928E088091710180938F0881E00E9445
:1063F000E95780918E08882341F0FD1431F06D2D0E
:106400006F5F8F2D8F5F0E94C859CD2DDD27C7FD8F
:10641000D09580911F059E01281B3109C9011816CE
:1064200019065CF0CE01019797FF02C080E090E072
:1064300080931F0510E1DD240BC025303105D4F316
:10644000CE0104978B3091059CF38AE090E0F0CF69
:10645000F0901F05FD0CAF2CBB2495012F5F3F4F23
:10646000442737FD4095542FCA15DB0511F401E18F
:1064700001C000E182E1612F72E0E72E0E94F75E29
:1064800080917101F81629F481E0612F4AE20E949F
:10649000B65D8F2D6FE778E04FE00E94C456CA15B5
:1064A000DB0531F480918E08882311F001E101C0F1
:1064B00000E188E1612F4FE758E02FE00E94BA5DCC
:1064C000D394185F3D2D363019F6DF91CF911F918F
:1064D0000F91FF90EF90DF90BF90AF900895AF9233
:1064E000BF92CF92DF92EF92FF920F931F93CF93C1
:1064F000DF935B016C0110E1E12EF12CC0E0D0E8EC
:1065000000E010E89E0140E050E0CA01B9010E949D
:106510004074A616B706C806D90610F4C027D127BE
:10652000169507950894E108F108E114F10461F467
:10653000CE01DF91CF911F910F91FF90EF90DF90EF
:10654000CF90BF90AF900895C02BD12BDBCFE1E06F
:10655000683068F4E0E070E09B01220F331F220FE7
:10656000331F260F371FA90146575C4F0EC070E03E
:10657000685070409B0153E0220F331F5A95E1F79A
:10658000260F371FA9014E545C4FDA012C91805021
:106590009C4F97FD0FC0B8E080309B078CF0EE2336
:1065A00019F028E030E002C024E030E0240F351F6D
:1065B000F9012081332727FD3095322F222730C063
:1065C000EE2329F0692F9070880F991F03C0692F5F
:1065D00066959170262F30E0FA01E20FF31F61817A
:1065E000772767FD7095AC0155954795649F90019D
:1065F000659F300D749F300D11246081772767FDF2
:10660000709540E052E0481B590B55954795649FA3
:10661000C001659F900D749F900D1124280F391FA4
:10662000C90169E170E00E947F74CB0108952F9247
:106630003F924F925F926F927F929F92AF92BF92E2
:10664000CF92DF92EF92FF920F931F93DF93CF933E
:1066500000D00F92CDB7DEB7182F99249394809174
:10666000A608883008F499248BEC9FE00E94441A15
:10667000992011F05AE001C056E084EC98E0612FB7
:1066800040E020E030E000E071EDE72E7FE0F72E03
:10669000CC24C394A52E0E94BC1B4091A60850E0B8
:1066A0004F5F5F4F84E260E021E00E942D608091A7
:1066B000A608992079F090E008977C0103E0EE0CA1
:1066C000FF1C0A95E1F7E80EF91E22EB33E0E20E1B
:1066D000F31E0CC090E07C01EE0CFF1CEE0CFF1CC6
:1066E000E80EF91E8AE893E0E80EF91E0091C4084E
:1066F0000150D090C508113661F0123628F41434D8
:10670000D1F0153471F50EC01436A9F0153649F5DF
:1067100009C0DD2031F11092C50881E60E94F661C2
:10672000DD241FC0809120058823D9F01D14CCF4EE
:106730008D2D815014C080912005882391F02D2D3E
:10674000332727FD3095992019F089E090E002C0A9
:1067500085E090E02817390724F48D2D8F5F809312
:10676000C5088091C50880932005CE2C4F2C6E2C37
:106770007F2C90E122243324A02EBB24A7FCB094CC
:10678000F30141913F01552747FD509521E0A214A7
:10679000B30409F020E088E1692F99830E942D60FD
:1067A0000894211C311C9981985F983349F79920EE
:1067B00001F1A5E06A2E712C6E0C7F1C90E1F5E0D2
:1067C0002F2E312CF30141913F01552747FD509564
:1067D00021E0A214B30409F020E080E3692F99833B
:1067E0000E942D600894211C311C9981985F903380
:1067F00049F70F3F11F421E0D11020E08CE068E070
:1068000044EC5FE00E94EA5D992019F089E090E095
:1068100002C085E090E021E0A816B90609F020E06A
:106820008CE068E34DEB5FE00E94EA5D992019F08F
:1068300089E090E002C085E090E0A816B90694F4E3
:1068400007FD4EC0A02EBB24A7FCB094AE0CBF1C0D
:10685000812FF50160814CE924E60E94E614F501E0
:1068600080833EC01016E4F5812F6091C3084CEF81
:1068700024E000E00E94D8148093C308909199040A
:10688000992371F1992021F050E194E049E003C08F
:1068900058E092E045E024E6820230011124892F7D
:1068A00090E0909581959F4F869D9001879D300D3A
:1068B000969D300D1124EC2DF42DA52E00E0C9017C
:1068C0006A2D702F0E947F746193260D371D8E2FC5
:1068D0008C198417A0F382E00E94DB570E9477583E
:1068E00080912005882351F0AA24ECE92E2EEFEFA9
:1068F0003E2E4D2C552447FC5094A5C000E01CEFC3
:10690000AA24BB2470E2D72EACC0C90165E0880F71
:10691000991F6A95E1F7992019F064E070E002C0D0
:1069200062E070E00E947F74462F062F055C3701FD
:106930006A0C711CF3018081992787FD909555E0C1
:10694000880F991F5A95E1F7B1010E947F74562F65
:1069500090E2D92ED60E2F5F3F4F8D2D90E09B8376
:106960008A834216530609F050C082349105ACF474
:106970008AE3C82EC40E625E8C2D45E059830E94C6
:10698000975E5981EA81FB81E134F10531F0652F91
:10699000615E8C2D45E00E94975EFD2DF03430F451
:1069A000802F81506D2D45E00E94975E2A813B81AA
:1069B0002F33310594F401506D2D6F5F802F45E02A
:1069C0000E94975E8A819B818E33910531F06D2DF7
:1069D0006E5F802F45E00E94975E80919C049091AD
:1069E0009D04009741F4123631F0133621F0123431
:1069F00011F0133439F5812FF30160814CE924E65D
:106A00000E94E614F30180831DC02A813B8121345A
:106A100031052CF4615E802F43E00E94975E3D2D8E
:106A2000303428F4802F6D2D43E00E94975E8A81D8
:106A30009B818F33910534F46D2D6F5F802F43E080
:106A40000E94975EA3942A2D30E0992019F089E0E6
:106A500090E002C085E090E0281739070CF455CF8C
:106A60004DCFC8016091A6080E94A732BCE3EB2E6F
:106A7000EA0C9C01A5E036952795AA95E1F76D2DC6
:106A8000621B8E2D0E944B5E950123703070211584
:106A9000310521F48E2D60E20E944B5E0894A11C0A
:106AA000B11C005E1F4F90E4A916B104D1F68CE52D
:106AB00060E040E40E949B5E0F900F900F90CF919A
:106AC000DF911F910F91FF90EF90DF90CF90BF90DB
:106AD000AF909F907F906F905F904F903F902F90DE
:106AE00008952F923F924F925F926F927F928F9272
:106AF0009F92AF92BF92CF92DF92EF92FF920F934D
:106B00001F93DF93CF93CDB7DEB7A2970FB6F8945C
:106B1000DEBF0FBECDBF8F8F98A36A8B80919E047E
:106B2000882309F474C080912105882319F08150CD
:106B3000809321058091CB069091CC062091C906C7
:106B40003091CA06820F931F2091CD063091CE0658
:106B5000820F931F2091CF063091D006820F931F92
:106B600020915407309155072C01421A530A920183
:106B700057FE03C0309521953F4F41E02130340747
:106B80003CF0909355078093540781E08093A104D3
:106B900080918901863FD9F1909108019233B8F133
:106BA000909151079F5F90935107903160F0209131
:106BB0005207309153072F5F3F4F30935307209375
:106BC0005207109251079091A104992321F010923D
:106BD000530710925207209152073091530799277B
:106BE00087FD90950A9667E771E0869FA001879FD1
:106BF000500D969F500D11244217530740F42370F7
:106C000030702130310519F480E10E94B56D80911A
:106C10008801582F51705F5F598781FF02C01D8620
:106C200002C063E06D876090BC01662009F44AC031
:106C30008985E82FF0E0EE0FFF1FEF50FB4FA0809B
:106C4000B180CC24B7FCC094DC2C9D85E92FF0E00A
:106C5000EE0FFF1FEF50FB4F20813181442737FD9E
:106C60004095542FCA01B9010E9440747B018C01E8
:106C7000C601B501A60195010E944074E60EF71EFB
:106C8000081F191F662D70E080E090E0EAE0660FB3
:106C9000771F881F991FEA95D1F724E630E040E07E
:106CA00050E00E94B474B901CA010E9440746E158C
:106CB0007F058007910730F4C801B7010E946F3249
:106CC0004C0102C088249924B40180E090E024E6BD
:106CD00030E040E050E00E9440746B8F7C8F8D8FDD
:106CE0009E8F64E4662E61E0762EA9ECB6E0BE8B42
:106CF000AD8BFE013196F88FEF8B50E0252E51E0E1
:106D0000352E24EA31E03F872E8741EF54E05A8F39
:106D1000498F2901F98BE88BBC8BAB8BEE24FF24C8
:106D20001B865A89517059A3AE2C8E2D0E94D51501
:106D30009C01D30111968D919C911297281B390BC0
:106D4000B901882777FD8095982F4AE0660F771F55
:106D5000881F991F4A95D1F7121613062CF45D96D9
:106D60002D913C915E9703C0F3012785308924362D
:106D7000310514F424E630E0442737FD4095542FC4
:106D80000E94B4748901FCEF21303F072CF024E00D
:106D90000030120724F405C000E01CEF02C000E040
:106DA00014E080918A0180FF0FC08091880190E0FB
:106DB0008170907042E050E0481B590BE416F506D4
:106DC00019F4109501951F4FA98DBA8D0D931D9340
:106DD000BA8FA98FC8010F968F319105F0F4B4E0F6
:106DE000EB16F1047CF48A2D8F5F0E941A6390E009
:106DF0000197E1E0F0E002C0EE0FFF1F8A95E2F795
:106E0000CF0108C081E090E00E2C02C0880F991FCE
:106E10000A94E2F7FB85F82BFB872A2D243008F033
:106E20007AC139A1332309F05FC08091B00181FF9D
:106E30005BC06701CC0CDD1C4EE751E0C40ED51ED3
:106E4000D60111968C911197807C09F44DC08C91DC
:106E500085958595859561E040E00E94A210882384
:106E600009F442C0D601EC91E770F0E0DF01AA0F0F
:106E7000BB1FAA55BB4FEE0FFF1FEA58FE4F8D9167
:106E80009C91119720813181821B930B62E070E00D
:106E90000E947F74F701EE0FFF1FE158FE4F208123
:106EA000422F440F440F45954595552747FD509572
:106EB000649FC001659F900D749F900D11246FE138
:106EC00070E00E947F74660F771F660F771F229510
:106ED000269526952370213019F0223029F403C01D
:106EE000060F171F01C08B018114910409F1B985A8
:106EF000AB1619F0ED85AE16D9F46091BC0170E0C7
:106F000080E090E04AE0660F771F881F991F4A953E
:106F1000D1F79801442737FD4095542F0E944074C3
:106F20002B8D3C8D4D8D5E8D0E94B474022F132FDE
:106F3000F201EA54FE4F808160E040E00E94A2101E
:106F4000882369F0F201E954FE4F808160E040E05F
:106F50000E94A210882329F4CC24C39404C0CC241A
:106F600002C032E0C32E8091880190E08170907061
:106F700022E0A22EB12CA81AB90AAE14BF0469F5FA
:106F80008091B501807F49F1C80180509C4F62E03B
:106F900070E00E947F749B01EC2DF0E0EE0FFF1F6C
:106FA000EE0FFF1FA701440F551FCA01A3E0880F72
:106FB000991FAA95E1F7841B950BE80FF91FE25B77
:106FC000FC4F6081772767FD7095C9010E945A27A1
:106FD000AC01440F551F30E028C031E010161106F7
:106FE0000CF430E08C2D90E0A701440F551FFA01FE
:106FF00063E0EE0FFF1F6A95E1F7E41BF50B880FC6
:10700000991F880F991FE80FF91FEC55FE4FE30FEA
:10701000F11DE655FE4F6081772767FD7095C80129
:107020003AA30E945A27AC013AA1EC2DF0E0EE0FF2
:10703000FF1FEE0FFF1FB701660F771FCB0113E095
:10704000880F991F1A95E1F7861B970BE80FF91F18
:10705000EC55FE4FE30FF11DE455FE4F608177279D
:1070600067FD70956C597F4F882777FD8095982F25
:10707000DA019D01442737FD4095542F0E9440744A
:1070800024E630E040E050E00E94B474022F132F59
:10709000AE14BF0499F58091B501982F907F09F443
:1070A00066C60050144063C6D101ED91FC91119762
:1070B000608180918A0180FD6195772767FD7095D9
:1070C000872F972F63587F4F8F4F9F4F20E034E0DB
:1070D000201B310B442737FD4095542F0E944074EC
:1070E00020E038E040E050E00E94B4742030B8E086
:1070F0003B07B0E04B07B0E05B0739F4D101ED91FD
:10710000FC912081332727FD3095220F331FE8891A
:10711000F98931832083AB89BC890D931D93BC8B86
:10712000AB8B0894E11CF11CE2E0F0E06E0E7F1ED8
:10713000288939892E5F3F4F398B288B2E0E3F1EB1
:107140004EE050E0440E551E57E0E516F10409F0FC
:10715000EBCD0091B9016B85062380915607809590
:10716000802319F088E10E94B56D0093560780E0F6
:1071700094E09093D8068093D7069093DA06809394
:10718000D906E6EAF4E026E731E0A1EEB6E0BD017B
:1071900081919191D9014D915D919D01841B950B38
:1071A000880F991FDB018D939D93BD01B4E0EE3AEA
:1071B000FB0771F78091AE049091AF04880F991F7F
:1071C0009093EA068093E9068091B0049091B1040F
:1071D000880F991F9093EC068093EB068091B20480
:1071E0009091B304880F991F9093EE068093ED065B
:1071F0008091B4049091B504880F991F9093F00684
:107200008093EF06E1E1F7E0FC87EB8721EF36E0C2
:107210004191519161917191D9014D935D939D017E
:10722000B7E0E135FB07A1F7C090BC01CC2009F421
:107230007AC0E985AE2EBB24AA0CBB1C29EC422ED9
:1072400026E0522EA40CB51CD5012D903C90442470
:1072500037FC4094542CBD850B2F10E0000F111FFC
:107260000753194FF80120813181442737FD40959C
:10727000542FCA01B9010E9440743B014C01C20164
:10728000B101A20191010E944074660E771E881E12
:10729000991EDD24EE24FF248AE0CC0CDD1CEE1CBC
:1072A000FF1C8A95D1F7C701B60124E630E040E023
:1072B00050E00E94B474B901CA010E94407466157E
:1072C00077058805990578F5C401B3010E946F32EE
:1072D000BC0180E090E024E630E040E050E00E9415
:1072E00040743B014C01C201B101A70196010E940B
:1072F0004074A40193010E94B474D5012D933C9372
:10730000F80160817181882777FD8095982FA7010A
:1073100096010E944074A40193010E94B474D801A4
:1073200011963C932E93E090BA018E2D807E09F445
:10733000DEC0B9852B2F30E0220F331FF901E75350
:10734000F94F40815181CE010196280F391FD90193
:10735000ED91FC91BD856B2F70E0660F771FDB010F
:10736000A753B94F2D913C91860F971FDC018D914A
:107370009C91BA89B1FD05C0E40FF51F280F391F94
:1073800004C020E030E0E0E0F0E0A091BB01AA23DF
:1073900049F0B0E0AA0FBB1FA953B94F0D911C9142
:1073A000119702C000E010E0E2FE03C0F095E19505
:1073B000FF4FE3FE03C0309521953F4FE4FE03C02D
:1073C000109501951F4F8091BA018295869587701F
:1073D000823071F1833020F4813009F088C007C019
:1073E000833009F459C0843009F081C06CC0C901F0
:1073F00068E070E00E947F747B01C90160E870E082
:107400000E947F7429014E185F087201E61AF70A7C
:10741000C90160E072E00E947F74E61AF70AC801B1
:107420008E1B9F0B9093DC068093DB06CF0120C060
:10743000CF0168E070E00E947F747B01CF0160E8BB
:1074400070E00E947F743F016E187F087301E61A96
:10745000F70ACF0160E072E00E947F74E61AF70A33
:10746000C801821B930B9093DC068093DB06C90155
:1074700062E070E00E947F74600F711FCB018E0D7F
:107480009F1D9093DE068093DD066E197F09709331
:10749000E0066093DF062BC0C8018E1B9F0B909304
:1074A000DC068093DB06E00FF11FCF01820F931FF4
:1074B0009093DE068093DD06E21BF30BF093E0066B
:1074C000E093DF0614C0C8018E1B9F0B9093DC066F
:1074D0008093DB06C801820F931F9093DE06809392
:1074E000DD06021B130B1093E0060093DF0680916C
:1074F0009E04882311F00E94E52F80E4E1E1F7E08B
:10750000DF011D928A95E9F7BA89B1FF2DC08091FC
:10751000880190E08170907022E030E0281B390BE8
:1075200080E090E0ED89FE89AF89B88D2817390792
:1075300029F01182108211961C921E9201963296A9
:1075400012968430910591F71092E2061092E106AE
:107550001092E4061092E3061092E6061092E506F9
:107560001092E8061092E70686E893E090930101F6
:10757000809300019C012F5F3F4F309303012093C4
:1075800002019C012E5F3F4F3093050120930401BF
:107590000396909307018093060127E1422E28E08D
:1075A000522E97E9692E97E0792E87E5282E87E0FD
:1075B000382E19861D8689850E94D70E7C01FC0114
:1075C00080818150803108F0ADC2838161E040E06C
:1075D0000E94A210D2019C918823A1F4292F1C9211
:1075E000F7019181892F8850823008F08AC2878103
:1075F0008E70843009F485C2993009F04BC000E0E8
:107600001CEF4AC021E0911120E081E0D2018C936F
:10761000D7011196EC913E2F3150832F90E0DC0181
:10762000AA0FBB1FA753B94F0D911C91119734316D
:1076300060F0B9853B1748F4DC01AA0FBB1FAA0F05
:10764000BB1FAF5EB84F0D911C91D70117963C91AF
:107650001797832F807381F0832F8295837090E03A
:10766000019741E050E002C0440F551F8A95E2F7B0
:10767000CA015D85582B5D8736FF0EC0E53060F48A
:10768000F0E0EE0FFF1FE250FF4FC7010896918315
:10769000808302C000E010E0D7011796CC901797C6
:1076A000C6FC0BC018968C911897882331F02AA33A
:1076B0000E94BA0E080F191F2AA1F701868188239C
:1076C00021F48581882309F458C1D3016D917D91FE
:1076D0008D919C911397222389F420E031E040E0C2
:1076E00050E00E94B47450954095309521953F4FDD
:1076F0004F4F5F4F4801820E931E5AC08C2D8E70E3
:10770000843051F5D701EC91F0E0EE0FFF1FE1510D
:10771000F94F60817181882777FD8095982F20E04F
:1077200034E640E050E00E944074F30160837183CE
:1077300082839383D70112962C911297222361F0B2
:10774000332727FD3095432F532F0E94B474F30144
:107750002083318342835383D3016D917D918D9139
:107760009C91139720E031E040E050E00E94B47417
:1077700050954095309521953F4F4F4F5F4F4801B1
:10778000820E931E8114910499F0F701258197FED2
:1077900022952F7030E044E650E0249FC001259FE1
:1077A000900D349F900D1124D10111969C938E93CE
:1077B000F10180819181009799F020919E0422230C
:1077C00019F0019791838083D1018D919C9111973C
:1077D000009731F0F3016081718182819381B7C09C
:1077E0008114910409F4C9C0D70116968C9116979B
:1077F000882309F4B4C080919E04882309F476C0DC
:1078000012962C9112972223B1F0332727FD309541
:1078100037FF03C0309521953F4F332727FD309523
:10782000432F532F60E070E080E293E00E94B47435
:1078300059016A0106C0A12CB12CF0E2CF2EF3E071
:10784000DF2EF701868118141904FCF48F7090E084
:107850000097F1F144E650E0849F9001859F300D40
:10786000949F300D1124442737FD4095542FC601B5
:10787000B5010E94B474F30180819181A281B3812A
:10788000280F391F4A1F5B1F2CC082958F7090E014
:107890000097F1F044E650E0849F9001859F300D01
:1078A000949F300D1124442737FD4095542FC60175
:1078B000B5010E94B47459016A01D3012D913D9123
:1078C0004D915C9113972A193B094C095D0909C038
:1078D0009801442737FD4095542F542F432F322FC2
:1078E0002227F3012083318342835383D3016D9197
:1078F0007D918D919C9120E031E040E050E00E942C
:10790000B474C801AA2797FDA095BA2F18141904BA
:1079100034F482179307A407B50734F012C0281770
:1079200039074A075B076CF4222717FD2095322F91
:10793000322F212F102F0027F30100831183228380
:107940003383D3016D917D918D919C91139720E0AC
:1079500031E040E050E00E94B47489010EC0C801DB
:10796000AA2797FDA095BA2FBA2FA92F982F88275D
:10797000F30180839183A283B383D70114966C9122
:107980001497633061F1643028F4613051F0623053
:10799000A0F444C0653069F1653038F1663081F596
:1079A0002BC0F7018181893029F417FD35C00050C3
:1079B00012400EC017FF32C02CC0D70111968C9117
:1079C0001197893041F41016110604F100501E4F32
:1079D000000F111F23C010161106DCF01FC017FF87
:1079E0001DC0109501951F4F19C01016110674F097
:1079F00010C017FF0EC010C0101611063CF00CC0CE
:107A00006750C8010E94A7328C0108C000E014E052
:107A100005C000E010E002C000E01CEFF701878124
:107A200080FD13C0E181EE2381F0E53070F4F0E0D9
:107A30003197EE0FFF1F21E030E02C0F3D1FE20FCA
:107A4000F31F80819181080F191FB801882777FDE6
:107A50008095982FD70112962C911297332727FDE6
:107A60003095432F532F0E944074F701008110E09E
:107A700001501040278126952770213071F0F801C0
:107A8000EE0FFF1FEE0FFF1F223069F5EF5EF84F7C
:107A9000608371838283938334C024E630E040E0C6
:107AA00050E00E94B474E22EC32EDA01000F111FC1
:107AB000000F111F0F5E184FF801208131814281A4
:107AC00053816E2D7C2DCD010E94407420E034E066
:107AD00040E050E00E94B474D8012D933D934D9343
:107AE0005C9313970EC0EF5EF84F20813181428185
:107AF0005381260F371F481F591F2083318342832C
:107B00005383B985BF5FB9870894411C511CE4E0D9
:107B1000F0E06E0E7F1E22E030E0220E331EB03207
:107B200009F049CD0E94CF0E8C01ED84E0FE05C026
:107B3000882319F48EE10E94B56DE1FE0BC0C801E7
:107B400090708034910519F08834910519F48FE113
:107B50000E94B56DE2FE0DC010700038110531F0C5
:107B60000838110519F00039110519F480E20E9456
:107B7000B56DBFEF4B2EB4E05B2E3F8D28A1832F58
:107B8000922F9A87898722243324598A488AAB8581
:107B9000BC85ED90FD900D911C91C801B70124E6C4
:107BA00030E040E050E00E94B474EB85FC85208317
:107BB000318342835383A889B9892D933D93B98B2F
:107BC000A88BEE85FF85E35AFE4F80819181EE857B
:107BD000FF85E55AFE4F2081BAE02B026001112497
:107BE000E8EEF3E0CE0EDF1EEE85FF85E65AFE4F8F
:107BF00020812B0250011124A8E14A2EACEF5A2E0D
:107C0000A40CB51C96014C2D232F8C159D0514F446
:107C1000482F292F842E922E8A149B040CF44501A0
:107C2000E114F1040105110569F19401442737FDC0
:107C30004095542F1E141F041006110654F4B6016B
:107C4000882777FD8095982F621B730B840B950B0B
:107C50000DC0C501AA2797FDA095BA2F29013A01A9
:107C6000481A590A6A0A7B0AC301B201A80197019E
:107C70000E94407420EA36E841E050E00E94B4746B
:107C800079018A01C4010E94251A3C01882477FCED
:107C90008094982C6E0C7F1C801E911EC6010E9441
:107CA000251A8C01C5010E94251A222717FD20954F
:107CB000322F061517052805390514F43801490136
:107CC000AA2797FDA095BA2F84017301681679063B
:107CD0008A069B0614F47C018D01EE85FF85E45A2B
:107CE000FE4F8081882341F010950095F094E09438
:107CF000E11CF11C011D111DF4EACF2EF1E0DF2E75
:107D0000C20CD31CF601E358FD4F8081882389F013
:107D100060E040E00E94A210882359F0F601E2588A
:107D2000FD4F80810E94BA0E7C010027F7FC009570
:107D3000102FF894A985BA85ED92FD92BA87A9878C
:107D40007894EB85FC853496FC87EB87E2E04E2E39
:107D5000512C240C351C2E853F852B5F3F4F3F87D0
:107D60002E8730E22316310409F011CF04C08F7042
:107D700009F09AC9C3C9A2960FB6F894DEBF0FBE28
:107D8000CDBFCF91DF911F910F91FF90EF90DF90CA
:107D9000CF90BF90AF909F908F907F906F905F90AB
:107DA0004F903F902F900895EF92FF920F931F9363
:107DB000DF93CF93CDB7DEB7C054D0400FB6F89461
:107DC000DEBF0FBECDBF8E010F5F1F4FC80163E046
:107DD0000E94713581E2E82EF12CEC0EFD1EC701E8
:107DE00061E00E947135E0E0F3E041815281608101
:107DF000D8012D913C91D7018D919C9111976623CB
:107E000029F0B901681B790BCB0102C0821B930BCF
:107E1000840F951F73E0883E97072CF4ACEF8931EF
:107E20009A0724F005C088EE93E002C088E19CEF39
:107E30009283818335960E5F1F4F62E070E0E60EFD
:107E4000F71E73E0E035F70781F68091880190E036
:107E50008170907022E030E0281B390B80E090E0C8
:107E60002817390721F0FC01EA57FC4F10820196D0
:107E700084309105A9F786E00E94DB5781E00E94DB
:107E8000B56DC05CDF4F0FB6F894DEBF0FBECDBF3F
:107E9000CF91DF911F910F91FF90EF9008952F9256
:107EA0003F924F925F926F927F928F929F92AF928A
:107EB000BF92CF92DF92EF92FF920F931F93DF93C7
:107EC000CF930F92CDB7DEB7109186011F70813826
:107ED00009F477C0823888F48332F1F1843230F4C7
:107EE0008032E1F0823209F07EC045C0813609F46B
:107EF0005DC0803809F077C01BC08438F9F0853840
:107F000038F4823809F44AC0833809F06CC040C0A4
:107F10008538E1F08F3B09F066C059C0153009F093
:107F200062C08091A20491E089278093A2044DC091
:107F30000E9404150E94431580E805C08FE291E37A
:107F40000E94431584E80E94F6614DC08DED9AE4CD
:107F50000E94431585E8F7CF812F8F5F80938601BC
:107F6000863010F01092860181E00E94DB5783E199
:107F70000E94B56D38C0112319F0812F815001C0C6
:107F800085E08093860181E00E94DB5784E1F0CF99
:107F90008BE49AE10E94331583E8D5CF0E94446FA9
:107FA0008DE394E70E94331582E8CDCF8091470698
:107FB000823021F483E08093470607C0153099F49E
:107FC00002C00E949A300E94821587E1D1CF81E0E1
:107FD0000E94F66183E00E94F66182E00E94F661F1
:107FE00081E0809337088091B80160E040E00E9412
:107FF000A210882331F080913708882311F40E9461
:10800000D43E8091B80160E040E00E94A2108093CD
:10801000370880918601803108F0D3C09091080123
:1080200080917301981710F496E001C094E0B4EACF
:10803000EB2EB1E0FB2E0AE0D7014D917D01802FA0
:1080400060E024E099830E94F75C055F998108371E
:1080500099F7492F406884E260E10E94720F84E240
:1080600068E146E50E94B65D80914706882399F055
:10807000823011F406E001C004E0409148065091BE
:1080800049068EE560E1202F0E94F30E83E368E14C
:1080900040E00E9417104091B60183E04802A00121
:1080A00011244C50584F84E260E123E000E00E942C
:1080B000BA5D8091B5018F7031F089E360E140EFE6
:1080C00057E00E94195EAEE0EA2EA1E0FA2EF0E041
:1080D000CF2EF1E0DF2E66247724EFE19E2EF7010C
:1080E00001917F01D601ED91FD916D01808187FDA8
:1080F0008D5F85958595843E0CF484EEA82E8D3198
:1081000014F07CE1A72E862D81508230F8F4802F68
:1081100064E046E30E949B5E2091880130E02625C2
:10812000372520FD04C08091B5018F7061F4802F48
:1081300081506EE143E00E949B5E802F8F5F6EE175
:1081400043E00E949B5E992D9A1914C0802F8B5199
:108150006BE346E30E94975E802E8A94882D6AE343
:1081600043E00E94975E882D6CE343E00E94975E97
:108170000A0D9BE36DEF862E800E5DEFA52EA90EF6
:10818000882D6A2D47E099830E949B5E9981692F13
:108190006D5F882D47E00E94975E802F8D5F6A2D6E
:1081A00047E00E949B5E882D6A2D47E00E94975E03
:1081B0000894611C711CB4E06B16710409F08FCF38
:1081C00027C080E060E044EA51E02AE001E10E943B
:1081D000BA5D9091080180917301981710F442E004
:1081E00001C040E084E560E00E94720F8091470684
:1081F000882371F0823011F402E001C000E0409168
:108200004806509149068FE660E0202F0E94F30E49
:10821000123008F085C045E2E42E45E0F42E00E07F
:1082200039E1A32EB12C2BE1922E90E2692E712C14
:1082300080E8482E512CF701219031907F011130B8
:1082400011F1802F8370899DC02C1124D02ED694DB
:10825000D694DD0CDD0CDD0CF8E2DF0EC101B301BC
:108260000E947F749B01C101B2010E947F74AB0127
:10827000421B530B420D531D8C2D8F5D6D2D20E243
:108280000E942D6048C0043018F4B2E2CB2E02C028
:10829000AEE5CA2E802F8370D82EDD0CDD0CD80EF3
:1082A00026E2D20EC10137FE04C088279927821921
:1082B00093098A9DA0018B9D500D9A9D500D11240C
:1082C00040505E4F452F550F550B45954595842ED3
:1082D0004A3114F0E9E18E2E8C2D89516D2D43E346
:1082E00025E50E94695E6D2D62508C2D45E00E944F
:1082F0009B5E1214130414F4C39401C0C8186D2DAE
:108300006F5F8C2D482D0E94975E6D2D61508C2DD6
:10831000482D0E94975E0F5F083009F08CCF8AC00D
:10832000153008F07DC00E94C220123061F0812F0C
:10833000880F810F880F8950912F9150192F110F9D
:10834000190F110F02C080E016E0C82E992787FD93
:1083500090952C01440C551C480E591E60E2D62EF7
:10836000EE24FF2452E0852E912C880E991E3C01AC
:108370001AC00E9414105C018C2D60E040E00E9445
:10838000A210082FA501440D551D8AE06D2D23E094
:108390000E94BA5D0894E11CF11C83E090E0480E55
:1083A000591E98E0D90EC394C701860D971D8816F3
:1083B0009906FCF6812F992787FD90952C01440C96
:1083C000551C480E591E30E2D32EEE24FF2422E025
:1083D000822E912C880E991E3C011AC00E94141006
:1083E0005C01812F60E040E00E94A210082FA501EF
:1083F000440D551D85E66D2D23E00E94BA5D08945D
:10840000E11CF11CA3E0B0E04A0E5B1EB8E0DB0EFD
:108410001F5FC701860D971D88169906FCF60AC0D6
:108420004091A4045091A5048CE368E224E004E0A8
:108430000E94F30E0F90CF91DF911F910F91FF904B
:10844000EF90DF90CF90BF90AF909F908F907F90F4
:108450006F905F904F903F902F90089518161CF0EA
:1084600010921F050895282F332727FD30959091EE
:108470001F05291B3109462F50E04217530724F4EA
:10848000861B80931F0508954650504024173507DA
:1084900024F48A5F861B80931F050895AF92CF92C4
:1084A000DF92EF92FF920F931F93DF93CF930F9280
:1084B000CDB7DEB7182F83E89BE00E94441A81E90C
:1084C00098E0612F42E020ED37E00AE07EE8E72EF9
:1084D0007BE0F72ECC2456E0A52E0E94BC1BF0902A
:1084E00091088F2D67E00E942E4288E068E77BE0CC
:1084F0000E94115E31E08F2D813009F030E08091D3
:10850000BA0182958695877090E0AC01440F551FA3
:10851000480F591F440F551F475A544F84E568E0D0
:1085200026E0032F39830E94BA5D3981332399F005
:108530006091BA01629566956770812F40E024E0F2
:108540000E94E6148295880F807E9091BA019F71F7
:10855000982B9093BA0180E16EE47BE00E94115E5B
:1085600001E0EF2DE23009F000E084E560E14091A8
:10857000BB01202F0E94780F002349F0812F6091CA
:10858000BB0140E024E20E94E6148093BB0188E135
:1085900063E47BE00E94115E4091BC01FF2DF3304B
:1085A00011F421E401C020E484E568E150E00E9478
:1085B0002D608F2D833049F4812F6091BC0140E004
:1085C00024E60E94E6148093BC010091BA0106954E
:1085D0000695017080E265E37BE00E94115ECF2C7E
:1085E000DD24C7FCD09421E0E4E0CE16D10409F0EC
:1085F00020E084E560E2402F0E94871BFF2DF430CD
:1086000079F4812F602F40E021E00E94E614817010
:10861000880F880F9091BA019B7F982B9093BA0195
:108620000091BA01069506950695017088E267E209
:108630007BE00E94115E21E085E0C816D10409F0BC
:1086400020E084E568E2402F0E94871BEF2DE53093
:1086500081F4812F602F40E021E00E94E6148170B8
:10866000880F880F880F9091BA01977F982B90936D
:10867000BA010091BA010295017080E369E17BE0E3
:108680000E94115E21E0F6E0CF16D10409F020E04F
:1086900084E560E3402F0E94871B8F2D863079F49C
:1086A000812F602F40E021E00E94E61481708295C6
:1086B000807F9091BA019F7E982B9093BA010F9082
:1086C000CF91DF911F910F91FF90EF90DF90CF90AE
:1086D000AF900895AF92BF92CF92DF92EF92FF9248
:1086E0000F931F93DF93CF930F92CDB7DEB7D82EA2
:1086F00082EE9CE00E94441A83E998E06D2D41E0EF
:1087000020ED37E00AE0A8EEEA2EACE0FA2EFBE01E
:10871000CF2EE0E1AE2E0E94BC1B10919308F0908A
:108720009408812F67E00E942E422091710130E071
:108730002F5F3F4F442737FD4095542F8AE260E07A
:1087400001E172E0E72E0E94F75E2D2D253451F0F5
:10875000263418F4243401F511C03D2D343671F05F
:108760003536D1F41130C1F4FF20B1F080912005ED
:10877000882391F08091940881500CC0113061F4ED
:108780004F2D493048F480912005882329F08091AD
:1087900094088F5F8093940880911F05882309F0C7
:1087A00088C088E06DED7CE00E94115E113031F4EC
:1087B00081E090E020912005222311F080E090E0FC
:1087C000082F00618CE368E044EA51E02AE00E944F
:1087D000BA5D80912005882359F48091230587FF95
:1087E00007C081E080932005109223051092940821
:1087F00080912005882381F020912305332727FDD0
:1088000030958F2D90E08217930734F41092200555
:108810001092230510929408113009F04DC08091F8
:108820002005882309F448C080919408909123057D
:10883000891B8093940887FF02C01092940880914E
:1088400094088A301CF089E08093940810922305E4
:10885000AF2CBB24F501EC55FE4F80810E94C62D44
:10886000682F20919C0430919D042115310549F415
:108870007D2D723631F0733621F0723411F073347D
:1088800031F48D2D40E021E40E94E614682F862FFC
:108890000E94D62D482FF501EC55FE4F80838F2D79
:1088A000880F8F0D880F845C68E021E00E94F75CE0
:1088B00003C098E0E92E02C080E1E82E80911F05F8
:1088C000823008F084C08E2D67ED7CE00E94115E3E
:1088D0004091B1015091B201123099F4FF2039F466
:1088E00080912005882309F01AC421E019C48F2D36
:1088F000813039F480912005882329F020E002E0BE
:1089000004C020E00DC420E001E087E46E2D0E9449
:10891000F30E123009F059C080912005882339F4F4
:1089200080919C0490919D04009709F44EC0FF2013
:1089300029F09F2D913009F048C022C08091B101EB
:108940009091B2010CE3A02EB12CB5010E946B7482
:108950008D2D40E02BE30E94E6142CE3482F4203C8
:10896000900111248091B1019091B201B5010E9452
:108970006B74280F391F3093B2012093B10125C0C9
:108980008091B1019091B2016CE370E00E946B7430
:10899000082F0E5F8D2D602F41E02EE30E94E6141C
:1089A000081B602F772767FD70952091B1013091EA
:1089B000B201261B370B3093B2012093B10137FF70
:1089C00004C01092B2011092B10168E0E60E8091ED
:1089D0001F058330F8F48E2D6FEC7CE00E94115E51
:1089E00001E0133009F000E08CE36E2D402F0E946F
:1089F0001710002349F08D2D6091AF0147EC29E35A
:108A00000E94E6148093AF0178E0E70E8E2D893343
:108A100008F088C380911F058430C8F58E2D68EC5E
:108A20007CE00E94115E91E0143009F090E08091AA
:108A3000B001282F217030E0A901440F551FA3E099
:108A4000220F331FAA95E1F7420F531F4D54534F86
:108A50008CE36E2D2AE0092F99830E94BA5D9981DB
:108A6000992379F06091B00161708D2D40E021E093
:108A70000E94E61481709091B0019E7F982B909394
:108A8000B00198E0E90EEE2DE93308F04BC3809178
:108A90001F05853030F50091B5010F708E2D6CEA01
:108AA0007CE00E94115E21E0153009F020E08CE3AB
:108AB0006E2D402F0E94771B153069F48D2D602F8D
:108AC00040E021E00E94E6148F709091B501907F04
:108AD000982B9093B501F8E0EF0E2E2D293308F076
:108AE00021C380911F05863040F50091B5010295A4
:108AF0000F708E2D65EA7CE00E94115E21E0163039
:108B000009F020E08CE36E2D402F0E94771B163079
:108B100071F48D2D602F40E021E00E94E6148295D3
:108B2000807F9091B5019F70982B9093B50138E0AC
:108B3000E30E4E2D493308F0F5C280911F058730B2
:108B400050F58E2D6CE97CE00E94115E91E01730AB
:108B500009F090E04091B60186E04802A00111249E
:108B60004358534F8CE36E2D26E0092F99830E94C2
:108B7000BA5D9981992349F08D2D6091B60140E04D
:108B800024E00E94E6148093B60168E0E60E7E2D94
:108B9000793308F0C7C280911F05883008F58E2D03
:108BA00065E77CE00E94115E01E0183009F000E00A
:108BB00086E36E2D4091B801202F0E94C40F002340
:108BC00049F08D2D6091B8014AEE26E10E94E6142D
:108BD0008093B80188E0E80E9E2D993308F0A2C278
:108BE00080911F05893008F051C08E2D6CE67CE025
:108BF0000E94115E9CE3AA24BB24A5014C59534F4B
:108C0000FA1411F4193061F02091B90130E00A2C06
:108C100002C0359527950A94E2F7022F017001C032
:108C200002E0892F6E2D21E099830E94BA5D08949D
:108C3000A11CB11C99819A5F9636F9F6193001F59D
:108C4000ED2DE03631F080919C0490919D040097C9
:108C5000B9F08D2D0E94F6611092200581E090E020
:108C60000F2C02C0880F991F0A94E2F72091B901D6
:108C700028272093B90182E00E94DB570E94775891
:108C8000F8E0EF0E2E2D293308F04CC280911F051D
:108C90008A3008F0E3C08E2D6EE57CE00E94115E04
:108CA0004091B30186E0489FA00111244B5B534FD4
:108CB0001A3041F4FF2031F480912005882321F0FF
:108CC00002E003C000E001C001E084E26E2D26E076
:108CD0000E94BA5D8091B301882321F0833009F0AE
:108CE0004DC009C086E66E2D40E45CE020E00E94A5
:108CF000EA5D9CE308C082E76E2D4DE35CE020E076
:108D00000E94EA5D98E44091B401552747FD5095D3
:108D1000440F551F440F551F485D534F1A3049F4F7
:108D20003F2D313031F480912005882321F002E07D
:108D300003C000E001C001E0892F6E2D24E099837B
:108D40000E94BA5D9981892F865D4091B70192E3B7
:108D50004902A0011124445D5E4F1A3049F46F2D81
:108D6000623031F490912005992321F022E003C074
:108D700020E001C021E06E2D0E942D608091B301A2
:108D8000813001F582E46E2D49E15CE020E00E9433
:108D9000EA5D4091B401552747FD50954F5F5F4F05
:108DA0001A3049F47F2D713031F4809120058823E9
:108DB00021F022E003C020E001C021E08EE76E2D0B
:108DC0000E942D601A3009F043C08091200588234D
:108DD00031F480919C0490919D040097C9F18F2DEE
:108DE000813079F0813018F0823091F522C08D2DDC
:108DF0006091B30140E023E00E94E6148093B30148
:108E000027C08091B301882311F0833031F48D2D78
:108E10006091B4014EEF24E007C08130C9F48D2D7C
:108E20006091B40140E02CE70E94E6148093B40105
:108E30000FC08091B301882311F0833049F48D2D48
:108E40006091B7014CEF2AE00E94E6148093B701CD
:108E500098E0E90EEE2DE93308F064C180911F051A
:108E60008B3008F07AC08091B301882311F08330F1
:108E700019F58E2D6AE07CE00E94115E4091BD01E3
:108E800085E04802A00111244F515F4F1B3011F4BF
:108E900021E201C020E28EE46E2D0E942D601B3085
:108EA00009F055C08D2D6091BD014CEE24E10E946A
:108EB000E6148093BD014BC08130B9F401E01B3052
:108EC00009F000E080E06E2D44EF5BE0202F0E946F
:108ED000EA5D0023E1F1FD2DF038C9F581E08093D2
:108EE0006D0E80E00E94B56D32C08E2D6BEE7BE082
:108EF0000E94115E8091B40187FD03C083301CF491
:108F000003C080E001C082E08093B40149E08402A4
:108F1000A00111244153544F1B3031F4809120059E
:108F2000882321F002E003C000E001C001E08CE3EF
:108F30006E2D29E00E94BA5D1B3049F48D2D6091A1
:108F4000B40140E022E00E94E6148093B40128E0DE
:108F5000E20E3E2D393308F0E5C080911F058C30BC
:108F600098F58E2D65EC7BE00E94115E31E01C309F
:108F700009F030E08091BA01817090E0AC01440FBB
:108F8000551F480F591F4254544F8CE36E2D23E058
:108F9000032F39830E94BA5D3981332379F06091C0
:108FA000BA0161708D2D40E021E00E94E6148170CD
:108FB0009091BA019E7F982B9093BA0148E0E40EFD
:108FC0006E2D693308F0AEC080911F058D3040F5DD
:108FD0000091BA01069501708E2D64EB7BE00E9432
:108FE000115E21E01D3009F020E08CE36E2D402F52
:108FF0000E94771B1D3071F48D2D602F40E021E021
:109000000E94E6148170880F9091BA019D7F982B81
:109010009093BA0178E0E70E8E2D893308F082C074
:1090200080911F058E3040F50091B00106950170CA
:109030008E2D6CEA7BE00E94115E21E01E3009F06B
:1090400020E08CE36E2D402F0E94771B1E3071F4C0
:109050008D2D602F40E021E00E94E6148170880F82
:109060009091B0019D7F982B9093B00198E0E90E0C
:10907000EE2DE93308F056C080911F058F3048F57A
:109080000091B0010695069501708E2D63EA7BE094
:109090000E94115E21E01F3009F020E08CE36E2D6C
:1090A000402F0E94771B1F3079F48D2D602F40E0F8
:1090B00021E00E94E6148170880F880F9091B00122
:1090C0009B7F982B9093B001F8E0EF0E2E2D293363
:1090D00048F580911F05803128F58091210588236E
:1090E00019F421E0103109F020E080E06E2D4FE806
:1090F0005BE00E94EA5D1031A9F43D2D303891F417
:109100001092200589E18093210580E80E94F66194
:1091100010923B068DEA90E30E94431503C022E0C3
:1091200000E0F3CB0F90CF91DF911F910F91FF9053
:10913000EF90DF90CF90BF90AF9008956F927F92A5
:109140008F929F92AF92BF92CF92DF92EF92FF9257
:109150000F931F93DF93CF930F92CDB7DEB7B82E47
:109160008DE29FE00E94441A89EA98E06B2D47E067
:1091700020ED37E00AE07DE3E72E7FE0F72ECC24F8
:10918000C3945CE0A52E0E94BC1B8090A9088A9421
:10919000D090AA08882D66E00E942E4218E0CC24C8
:1091A000992487FC909490911F059C0D9C3009F4A4
:1091B0004FC1E92EFF248E149F0439F480912005BD
:1091C000882329F022E0A22E04C0AA2402C0AA24E7
:1091D000A39480E0612F4AE25FE022E000E09983FF
:1091E0000E94BA5D9981993010F048E301C041E3D3
:1091F000490F8CE0612F0E94B65DF701EE0FFF1F53
:10920000EE0DFF1DE450FC4F408187E0489FA00118
:1092100011244953514FDD2011F000E001C00A2D07
:1092200088E1612F27E00E94BA5DC701880F991F6E
:109230008E0D9F1D8C559E4FFC01E85AFD4F2081DD
:10924000253008F4F6C0FC01EA5AFD4F283008F436
:10925000F9C040819D2D9130D1F53BC020E001C087
:109260002A2D88E4612F0E94780FF701EE0FFF1F6F
:10927000EE0DFF1DE550FC4F4081552747FD5095F1
:10928000ED2DE23011F020E001C02A2D88E7612F9A
:109290000E942D6000E035C020E001C02A2D88E446
:1092A000612F0E94C40FF701EE0FFF1FEE0DFF1D8F
:1092B000E550FC4F4081FD2DF23011F020E001C05F
:1092C0002A2D80E6612F0E94C40F01E01AC020E021
:1092D00001C02A2D88E4612F0E94780FF701EE0F5C
:1092E000FF1FEE0DFF1DE550FC4F40818D2D82309C
:1092F00011F020E001C02A2D86E6612F0E94780F30
:1093000002E080912005882339F480919C0490919B
:109310009D04009709F486C0AA2009F483C09D2DFE
:109320009130D1F1913020F0923009F07BC046C0ED
:109330003701660C771C6E0C7F1CECEFF3E06E0EB1
:109340007F1E8B2DF301608140E02DE00E94E6142A
:10935000F3018083202F30E0853028F0883030F40E
:1093600081E090E005C080E090E002C082E090E003
:109370002817390709F456C0C701880F991F8E0DA9
:109380009F1D8C559E4FFC01EA5AFD4F1082895A51
:109390009D4FFC01108246C0013041F0C701880F8B
:1093A000991FE80EF91E8AEF93E031C03701660C71
:1093B000771C6E0C7F1C8AEF93E01AC0013089F095
:1093C000C701880F991F0230F1F0E80EF91E8BEFEC
:1093D00093E0E80EF91E8B2DF701608143E82DE73D
:1093E0001DC03701660C771C6E0C7F1C8BEF93E061
:1093F000680E791E8B2DF30160814AEE26E10E94F2
:10940000E614F3010EC0E80EF91E8BEF93E0E80EB0
:10941000F91E8B2DF701608140E024E20E94E614E2
:10942000F7018083C394185FFC2DF73009F0BBCEA1
:109430000FC08A5A9D4FFC014081FD2DF13009F08B
:109440000DCF0ECF40818D2D813009F025CF26CF55
:109450000F90CF91DF911F910F91FF90EF90DF90D0
:10946000CF90BF90AF909F908F907F906F90089516
:109470006F927F928F929F92AF92BF92CF92DF9224
:10948000EF92FF920F931F93CF93DF93982E8FE36A
:109490009FE00E94441A8BEA98E0692D48E020ED95
:1094A00037E00AE01FE4E12E1FE0F12ECC24C39444
:1094B000B0E1AB2E0E94BC1B6090AB086A94809018
:1094C000AC08862D66E00E942E42A8E0FA2EDD242C
:1094D000772467FC709440911F054D0D403109F4CD
:1094E0005DC0A42EBB244F5F80E06F2D20E00E9462
:1094F000A40FEE24E501CC0FDD1FCE5DDB4F85010F
:10950000000F111F0F5D1B4F6A147B0471F48E1442
:1095100061F480912005882359F480919C049091F6
:109520009D04009739F421E001C020E0CC2405C05F
:1095300022E001C021E0CC24C394EE2091F48EE11E
:109540006F2DF80140810E94C40FCC20D9F0892DE5
:10955000F80160814AEE26E10E94E614F80180835A
:1095600011C04881552747FD509580E66F2D0E9418
:109570002D60CC2039F0892D688143E82DE70E94C9
:10958000E6148883E394FE2DF33009F0BDCFD39425
:1095900088E0F80EED2DE73009F09DCFDF91CF91F7
:1095A0001F910F91FF90EF90DF90CF90BF90AF9001
:1095B0009F908F907F906F900895AF92BF92CF92BF
:1095C000DF92EF92FF920F931F93DF93CF9300D020
:1095D000CDB7DEB7182F80919301813019F048E1A3
:1095E000C42E02C03AE1C32E2BEFB22EBC0C8EE18A
:1095F0009AE00E94441A88E498E0612F40E024EE4B
:1096000037E006E0EC2C0E94451FF0904808D0900F
:1096100049088F2D67E00E942E4260911F058C2D16
:1096200090E0462F50E09C012750304042175307EE
:1096300061F42F2D30E004972817390714F48FEFC9
:1096400001C081E0680F60931F05113629F11236C1
:1096500078F4143409F448C0153420F4123408F4B2
:109660006AC063C0153419F1103609F064C009C02E
:10967000143608F45AC01436B9F1153609F05BC037
:1096800016C0FF2009F457C081E090912005911188
:1096900080E0809320054FC080912005882309F445
:1096A0004AC01092200581E60E94F66144C02F2D29
:1096B000213059F4DD2049F080912005882329F0DC
:1096C000809149088150809349082F2D30E08B2DDF
:1096D000992787FD90952817390769F5DD2059F1FD
:1096E0008091490881501EC03F2D313061F48D2D8D
:1096F000893048F480912005882329F08091490819
:109700008F5F809349082F2D30E08B2D992787FD9F
:1097100090952817390779F49D2D973060F4809142
:1097200049088F5F8093490806C0809120058823EF
:1097300011F41092490880911F05882309F089C00F
:1097400088E063E17AE00E94115EEF2DE13031F4B0
:1097500081E090E020912005222311F080E090E04C
:10976000082F006182E468E045E951E02AE00E94A8
:10977000BA5D80912005882359F48091230587FFE5
:1097800007C081E0809320051092230510924908BC
:1097900080912005882381F020912305332727FD20
:1097A00030958D2D90E08217930734F410922005A8
:1097B0001092230510924908FF2DF13009F04CC09A
:1097C00080912005882309F447C080914908909131
:1097D0002305891B8093490887FF02C0109249081E
:1097E000809149088A301CF089E0809349081092E2
:1097F0002305AD2CBB24F501EB56FE4F80810E9462
:10980000C62D682F20919C0430919D0421153105AF
:1098100041F4123631F0133621F0123411F01334C2
:1098200031F4812F40E021E40E94F514682F862F47
:109830000E94D62D482FF501EB56FE4F80838D2DCB
:10984000880F8D0D880F8E5B68E021E00E94F75C29
:1098500003C098E0E92E02C080E1E82E80911F0548
:109860008230A0F5C0908701C694C694C69427E0C4
:10987000C2228E2D6CE07AE00E94115E91E03F2DB5
:10988000323009F090E046E08C2D849FA001112435
:109890004F51564F8CE56E2D26E0092F9A830E947A
:1098A000BA5D9A81992381F0812F6C2D40E026E0EA
:1098B0000E94F5148770880F880F880F9091870198
:1098C000977C982B9093870198E0E90E80911F0573
:1098D000833058F5C09093018E2D66ED79E00E949B
:1098E000115E91E0EF2DE33009F090E046E0FC2DB1
:1098F000F49FA00111244753564F8CE56E2D26E0AE
:10990000092F9A830E94BA5D9A81992341F0812F91
:109910006C2D40E021E00E94F5148093930128E033
:10992000E20E3E2D393308F0FFC380919301813060
:1099300041F580911F05843030F58E2D6BEB79E079
:109940000E94115E409191018F2D843011F421E429
:1099500001C020E486E66E2D50E00E942D609F2D10
:10996000943049F4812F6091910141E024E60E94F6
:10997000F51480939101E8E0EE0EFE2DF93318F016
:10998000D3C304E001C005E080919301815082308F
:1099900038F580911F05801710F58E2D6BEA79E060
:1099A0000E94115E40919201F01611F421E401C071
:1099B00020E486E66E2D50E00E942D60F01649F4FA
:1099C000812F6091920140E025E00E94F514809380
:1099D000920128E0E20E3E2D393308F0A5C30F5F57
:1099E00080911F05801720F58E2D62EA79E00E9494
:1099F000115E40917201F01611F421E401C020E4DF
:109A000086E66E2D50E00E942D60F01659F4812FED
:109A1000609172014AE02DE20E94F5148093720178
:109A20000E948D6088E0E80E9E2D993308F07CC37B
:109A3000C02EC39480911F058C1508F58E2D62E908
:109A400079E00E94115E40917301FC1411F421E44D
:109A500001C020E486E66E2D0E945E0FFC1449F4DE
:109A6000812F6091730148E228E70E94F5148093EA
:109A70007301E8E0EE0EFE2DF93308F055C3C394F0
:109A800080911F058C1560F58E2D61E879E00E94AC
:109A9000115E40918901552747FD5095465F5F4F04
:109AA000FC1411F421E401C020E486E66E2D0E942E
:109AB0002D608091A90D6E2D4DE60E94B65DFC14BF
:109AC00049F4812F6091890146EF2EE60E94F5143A
:109AD0008093890128E0E20E3E2D393308F024C33B
:109AE000C39480911F058C1550F58E2D66E779E0A3
:109AF0000E94115E91E0FC1090E040918B0150E0DB
:109B0000440F551F440F551F4759564F86E66E2D7B
:109B100024E0092F9A830E94BA5D9A81992349F023
:109B2000812F60918B0140E022E00E94F514809328
:109B30008B0188E0E80E9E2D993308F0F5C2C3949E
:109B400080911F058C15C8F480918A01817021E0F5
:109B5000FC1020E06E2D48E559E0012F0E94E02D19
:109B6000817090918A019E7F982B90938A01E8E002
:109B7000EE0EFE2DF93308F0D7C2C39480911F0575
:109B80008C15D8F480918A018695817021E0FC10B3
:109B900020E06E2D4CE459E0012F0E94E02D8170F1
:109BA000880F90918A019D7F982B90938A0128E0DD
:109BB000E20E3E2D393308F0B7C2C39480911F05E1
:109BC0008C15E8F480918A0186958695817021E054
:109BD000FC1020E06E2D4DE359E0012F0E94E02D96
:109BE0008170880F880F90918A019B7F982B9093AA
:109BF0008A0188E0E80E9E2D993308F095C2C3943F
:109C000080911F058C15F8F480918A0186958695C0
:109C10008695817021E0FC1020E06E2D4FE259E026
:109C2000012F0E94E02D8170880F880F880F90917E
:109C30008A01977F982B90938A01E8E0EE0EFE2D23
:109C4000F93308F071C2C39480911F058C1500F59B
:109C50008E2D62E279E00E94115E01E0FC1000E0CE
:109C600080E66E2D40917501202F0E94C40F0023C5
:109C700049F0812F609175014AEE26E10E94F514AA
:109C80008093750128E0E20E3E2D393308F04CC276
:109C9000C394BB2480911F058C1508F048C0BB20DD
:109CA00019F462E179E002C062E079E08E2D0E9451
:109CB000115EBB2019F4A0908C0102C0A090940109
:109CC000AA20A9F08A2D95E0899FA0011124FC14F7
:109CD00011F421E401C020E486E66E2D0E942D607F
:109CE0008091A90D6E2D43E70E94B65D0AC001E088
:109CF000FC1000E086E66E2D4EEF58E023E00E9457
:109D0000BA5DFC1439F4812F6A2D40E028E70E94E7
:109D1000F514A82EBB2019F4A0928C0102C0A092C9
:109D20009401E8E0EE0EFE2DF93308F0FDC1C39476
:109D3000B3942B2D223009F0ADCF80911F058C15E7
:109D4000F8F480918A0182958F708095817021E06E
:109D5000FC1020E06E2D40EF58E0012F0E94E02D16
:109D6000809581708295807F90918A019F7E982B4B
:109D700090938A0138E0E30E8E2D893308F0D4C128
:109D8000C39480911F058C15F8F480919001829501
:109D90008F708095817021E0FC1020E06E2D44EEE4
:109DA00058E0012F0E94E02D809581708295807F80
:109DB000909190019F7E982B9093900198E0E90EEE
:109DC000EE2DE93308F0B0C1C39480911F058C15C6
:109DD000D8F4809187018095817021E0FC1020E00B
:109DE0006E2D43ED58E0012F0E94E02D809581708B
:109DF000909187019E7F982B90938701F8E0EF0E5A
:109E00002E2D293308F090C1C39480911F058C1525
:109E1000E8F48091870186958095817021E0FC109F
:109E200020E06E2D44EC58E0012F0E94E02D80953B
:109E30008170880F909187019D7F982B9093870167
:109E400038E0E30E8E2D893308F06EC1C394809103
:109E50001F058C1508F086C08E2D69EB78E00E94F6
:109E6000115E92E4AA24BB24A5014055574FE0910E
:109E70009F01F0E00A2C02C0F595E7950A94E2F7FD
:109E8000E170F070892F6E2D21E00E2F9A830E94D1
:109E9000BA5D0894A11CB11C9A819A5F923721F790
:109EA000FC1409F059C08091490890912305891B41
:109EB0008093490887FF02C01092490880914908A1
:109EC0008A301CF089E080934908109223058D2D7B
:109ED000880F8D0D880F4D2D50E04955574F8E5BE3
:109EE0006E2D21E002E00E94BA5D103631F08091C3
:109EF0009C0490919D04009779F1812F0E94F66156
:109F00001092200581E090E002C0880F991FDA943A
:109F1000E2F790919F01982790939F01803151F033
:109F2000803271F0883099F493FF02C09F7C0DC09D
:109F300098600BC094FF02C0977D07C0906105C078
:109F400095FF02C0977E01C0906290939F0181E0CF
:109F50000E94DB570E94775898E0E90EEE2DE93316
:109F600008F0E2C0C39480911F058C15F8F480912D
:109F70008701869586958095817021E0FC1020E010
:109F80006E2D48E958E0012F0E94E02D80958170E8
:109F9000880F880F909187019B7F982B9093870162
:109FA000F8E0EF0E2E2D293308F0BEC0C394809147
:109FB0001F058C1500F590918701991F9927991F0E
:109FC00081E0891B21E0FC1020E06E2D4AE858E07A
:109FD000012F0E94E02D8095879588278795909185
:109FE00087019F77982B9093870138E0E30E8E2DA1
:109FF000893308F099C0C39480911F058C1508F52A
:10A0000080918A018295869587708095817021E084
:10A01000FC1020E06E2D40E858E0012F0E94E02D5A
:10A02000809581708295880F807E90918A019F7DB6
:10A03000982B90938A0198E0E90EEE2DE93308F011
:10A0400073C0C39480911F058C1518F580918A0107
:10A0500082958695869583708095817021E0FC10AD
:10A0600020E06E2D48E758E0012F0E94E02D8095FA
:10A0700081708295880F880F807C90918A019F7BE8
:10A08000982B90938A01F8E0EF0E2E2D293308F0DB
:10A090004BC0C39480911F058C1508F045C086E025
:10A0A0006E2D43E758E00E94195E3E2D383390F440
:10A0B00034E290E0832F6E2D45E857E0292F00E031
:10A0C00039839A830E94985C9A819F5F3981385EB8
:10A0D000943081F788E0E80E9E2D993328F5DD2431
:10A0E000D394FC10DD24409188014F5C82E16E2DF9
:10A0F0002D2D0E94F75C94E200E00F5F892F6E2DFA
:10A10000402F20E09A830E94780F9A81985E043055
:10A11000A1F7DD2049F0812F6091880140E023E024
:10A120000E94F514809388010F900F90CF91DF91DA
:10A130001F910F91FF90EF90DF90CF90BF90AF9065
:10A1400008958F929F92AF92BF92CF92DF92EF923B
:10A15000FF920F931F93DF93CF930F92CDB7DEB78C
:10A16000C82E88E79FE00E94441A8DEA98E06C2D83
:10A1700049E020ED37E00AE0FAE0EF2E0E94451FAB
:10A180001091AD081150812F66E00E942E422C2DB7
:10A19000203899F480E80E94F66189E180932105D6
:10A1A000193019F40E94B56205C0183018F4812FD7
:10A1B0000E94276381E00E94B56DDD24E8E0FE2E59
:10A1C000A12EBB24A7FCB09480911F058D0D883073
:10A1D00081F1882E992494012F5F3F4F442737FD4A
:10A1E0004095542FA814B90411F401E101C000E115
:10A1F00082E16F2D72E0E72E0E94F75EF401EE0F10
:10A20000FF1FE450F64E85919491AC018091210599
:10A21000882321F421E0A814B90409F020E088E1A2
:10A220006F2D0E94EA5D38E0F30ED3948D2D8730B8
:10A2300059F6EF2DE93308F04FC0809121058823AE
:10A2400021F4DD24D394183009F0DD2486E06F2D4D
:10A250004AE65FE00E94195E9AE556E0A52EB12C11
:10A26000E0918D01F0E0E852FB4F449150E00A2C60
:10A2700002C0559547950A94E2F7437050704B59C8
:10A28000504F892F6F2D21E00D2D99830E94BA5DCB
:10A290002EEF3FEFA20EB31E99819A5F923701F71E
:10A2A000DD2049F08C2D60918D0140E027E10E9476
:10A2B000F51480938D016F2D685F693368F4809188
:10A2C0002105882319F421E0193009F020E086E007
:10A2D00041E55FE00E94EA5D0F90CF91DF911F9111
:10A2E0000F91FF90EF90DF90CF90BF90AF909F9035
:10A2F0008F9008954F925F926F927F928F929F926C
:10A30000BF92CF92DF92EF92FF920F931F93DF9352
:10A31000CF9300D0CDB7DEB7182F86EB9FE00E9419
:10A32000441A81EC98E0612F46E020ED37E00AE026
:10A3300050E1E52E0E94451F6090C1086A94862D69
:10A3400066E00E942E42103611F0143641F467FC8C
:10A3500006C06092A60887E193E30E944315CC24CF
:10A36000DD24EE24E39418E0F12E772467FC70944A
:10A3700030911F053C0DBB24B394383028F4BB2426
:10A380008E2D883028F074C09E2D973008F070C054
:10A39000032F10E091E06016710609F090E0DD20D7
:10A3A00019F0DD24D39401C0D92E80E06F2D43EB4A
:10A3B0005FE0292F3A8399830E94EA5D3A8199816F
:10A3C000393010F482E101C087E1A8014F5F5F4F8F
:10A3D0006F2D292F0E942D60BB2079F0085010406E
:10A3E0002801B3E0440C551CBA95E1F7400E511E0C
:10A3F000E2EBF3E04E0E5F1E0BC02801440C551C2F
:10A40000440C551C400E511E8AE893E0480E591E1C
:10A4100042010AE2F40141914F01552747FD509551
:10A42000802F6F2D20E00E942D600B5E033991F785
:10A43000F8E0FF0EE394BB20B1F085E090E0480E19
:10A44000591E0AE2F20141912F01552747FD50950F
:10A45000802F6F2D20E00E942D600B5E0E3791F74C
:10A46000F8E0FF0EE394C3948C2D873009F080CF81
:10A47000DD2029F480911F058F5F80931F050F90C9
:10A480000F90CF91DF911F910F91FF90EF90DF9090
:10A49000CF90BF909F908F907F906F905F904F90E4
:10A4A0000895AF92BF92CF92DF92EF92FF920F93F7
:10A4B0001F93CF93DF93F82E87EA98E06F2D4DE03E
:10A4C0000E94B62080919F08882319F08BEB9EE0B4
:10A4D00002C081EB9EE00E94441A182F8091A008D0
:10A4E0000E94D70EEC01812F8A5F60E0488120E056
:10A4F0000E94A40FA090A7088A2D66E00E942E4219
:10A5000018E0EE24BB24A7FCB09420911F052E0D6B
:10A51000822F90E0DD24D394A816B90609F0DD243B
:10A52000263009F4FAC0273090F4223009F457C0DD
:10A53000233030F4222309F1213009F0E8C134C07E
:10A54000243009F499C0253008F0BAC069C02A3017
:10A5500009F46BC12B3038F4283009F420C12930BC
:10A5600008F044C1F1C02C3009F49CC12C3008F42F
:10A570007AC12D3009F0CBC1B2C18CE0612F4AEA1B
:10A580005EE00E94195E84E5612F49812D2D0E94B5
:10A59000780FDD2009F4BBC18F2D698141E024E2F1
:10A5A0000E94E6148983B3C18CE0612F43EA5EE028
:10A5B0000E94195E4A81552747FD50952D2D206434
:10A5C00084E5612F0E942D60DD2009F4A0C18F2D4C
:10A5D0006A8143E82DE70E94E6148A8398C18F813F
:10A5E00086FF03C049E95EE002C042E95EE08CE01C
:10A5F000612F0E94195E4885552747FD50952D2DE6
:10A60000206484E5612F0E942D60DD2009F47FC164
:10A610008F2D688543E82DE70E94E614888777C16F
:10A62000CF80C294C694C694E3E0CE2281E0C822D3
:10A630008CE0612F47E85EE00E94195E43E09C2DAC
:10A64000949FA00111244058514F84E5612F23E0CD
:10A650000D2D0E94BA5DDD2009F459C18F2D6C2D9E
:10A6600040E021E00E94E61481708295880F880FF7
:10A67000807C9F819F7B90C08CE0612F4BE75EE0E8
:10A680000E94195E8F81817090E0AC01440F551FCC
:10A69000480F591F4C58514F84E5612F23E00D2D71
:10A6A0000E94BA5DDD2009F432C16F8161708F2D87
:10A6B00040E021E00E94E61481709F819E7F6CC083
:10A6C0008CE0612F4DE65EE020E00E94EA5D4C8167
:10A6D00083E0489FA00111244F51504F84E5612F22
:10A6E00023E00D2D0E94BA5DDD2009F410C18F2DED
:10A6F0006C8140E026E10E94E6148C83873008F4E8
:10A7000006C19F2D903609F002C187508093A6089C
:10A7100087E193E30E944315FAC08CE0612F46E67F
:10A720005EE00E94195E8EE4612F4B812D2D0E9408
:10A73000C40FDD2009F4EBC08F2D6B814AEE26E1BA
:10A740000E94E6148B83E3C08CE0612F4EE55EE04F
:10A750000E94195E0F810295037049F02D2D20642F
:10A7600084E5612F402F50E00E942D6007C084E5F2
:10A77000612F4AE55EE02D2D0E94EA5DDD2009F49F
:10A78000C6C08F2D602F40E023E00E94E614837046
:10A790008295807F9F819F7C982B9F83B8C08CE09F
:10A7A000612F43E55EE00E94195E4F814695477038
:10A7B00050E063E0440F551F6A95E1F7465C514F46
:10A7C00084E5612F28E00D2D0E94BA5DDD2009F49B
:10A7D0009EC06F81669567708F2D40E022E00E94D9
:10A7E000E6148770880F9F81917FD6CF8CE0612F10
:10A7F0004FE25EE00E94195E4D8142954F7080E607
:10A80000612F50E02D2D0E942D60DD2009F47FC0C6
:10A810006D8162956F708F2D40E02FE00E94E614ED
:10A820008295807F9D819F701BC08CE0612F46E2E6
:10A830005EE00E94195E4D814F7080E6612F50E00E
:10A840002D2D0E942D60DD2009F461C06D816F7097
:10A850008F2D40E02FE00E94E6148F709D81907F45
:10A86000982B9D8354C08CE0612F4BE15EE00E94E9
:10A87000195E4E8142954F7080E6612F50E02D2D7C
:10A880000E942D60DD2009F442C06E8162956F70D8
:10A890008F2D40E02FE00E94E6148295807F9E81FC
:10A8A0009F701AC08CE0612F42E15EE00E94195E49
:10A8B0004E814F7080E6612F50E02D2D0E942D605B
:10A8C000DD2029F16E816F708F2D40E02FE00E9416
:10A8D000E6148F709E81907F982B9E8318C08CE029
:10A8E000612F40E05EE02D2D0E94EA5DDD2079F0D1
:10A8F0008F2D803861F40E94F6618091A0080E943B
:10A90000D32281E00E94B56D80E00E940E15E39491
:10A91000185F9E2D973009F0F8CDDF91CF911F91F0
:10A920000F91FF90EF90DF90CF90BF90AF90089580
:10A930005F926F927F928F929F92AF92BF92CF92CF
:10A94000DF92EF92FF920F931F93CF93DF93D82E56
:10A950008AE99FE00E94441A8FEB98E06D2D45E054
:10A9600020ED37E00AE071EAE72E7FE0F72E51E1B3
:10A97000C52E11E1A12E0E94BC1BF090BF08FA94D5
:10A980008090C0088F2D66E00E942E428D2D803869
:10A9900021F59F2D903108F5EF2DFF27E7FDF0956C
:10A9A00080911F05E81BF109EE0FFF1FEB5DFA4FC9
:10A9B000C081D1818F2D0E94E70EFC01882069F4AF
:10A9C0008281882319F0D095C195DF4FD483C3834A
:10A9D00082E00E94DB570E94775818E099245524A2
:10A9E00053946F2C772467FC709400911F05090D18
:10A9F000003109F4E1C0802F0E94E70EEC018A814A
:10AA00006B817C81882319F0709561957F4FA02E12
:10AA1000BB24F501EE0FFF1FEB5DFA4F2081318162
:10AA2000261B370B2333310524F0F501E155F74F91
:10AA300008C09FEF2E3C39072CF4F501E155F74F84
:10AA400085258083402F4F5F80E0612F20E00E94AA
:10AA5000A40FF501E155F74F8081882311F04FE7EE
:10AA600001C04EE78BE4612F20E00E94F75CEE24EA
:10AA70006A147B0471F48E1461F48091200588239C
:10AA800059F480919C0490919D04009739F401E061
:10AA900001C000E0CC2405C002E001C001E0CC24EC
:10AAA000C3948E2D823009F43FC0833009F45DC019
:10AAB0008130C1F04B815C81202F206280E3612FC7
:10AAC0000E942D60CC2009F46BC06B817C818D2DA0
:10AAD00048E15CEF28EE33E002E00E9422149C8300
:10AAE0008B835EC048814456552747FD509588E4C6
:10AAF000612F202F0E942D60CC2009F451C0688165
:10AB0000645668838091BA0181FF04C08D2D43E8AB
:10AB10002DE703C08D2D4CE924E60E94E6148883BE
:10AB200088818C5988833CC049814C59552747FD01
:10AB3000509586E6612F202F0E942D60CC2081F158
:10AB400069816C5969838091BA0181FF04C08D2DA0
:10AB500043E82DE703C08D2D4CE924E60E94E6145E
:10AB600089838981845689831BC08A8190E0AC01E6
:10AB7000440F551F480F591F4D56504F8CE6612FFB
:10AB800023E00E94BA5DCC2059F08D2D6A8140E00F
:10AB900021E00E94E61491E0882309F490E09A8372
:10ABA000E3949E2D943009F063CF9394185F892D20
:10ABB000873009F01ACF1FC001E09F2D903109F0B6
:10ABC00000E080912105882311F020E001C0202FB2
:10ABD00082E1612F42E85FE00E94EA5D002359F0C4
:10ABE0008D2D803841F489E18093210580E80E9411
:10ABF000F6610E94D43EDF91CF911F910F91FF909B
:10AC0000EF90DF90CF90BF90AF909F908F907F900C
:10AC10006F905F900895F8942091D70D3091D80DE2
:10AC20007894C9010895CF93DF93C4E4D1E080E61E
:10AC3000FE0111928A95E9F78AE08093440189E147
:10AC4000809372018AE58093730181E0809388018B
:10AC50002196FE0120E032E080E891E021933193DB
:10AC600095878487938F828F41E0E335F407B1F7AE
:10AC700085E991E063E870E14AE050E00E94D57414
:10AC800080E090E029913991820F931FE1E0CD356A
:10AC9000DE07C1F79093700180936F01DF91CF9130
:10ACA00008951F93CF93DF938AEC98E060E00E94B1
:10ACB000375A64E471E080E6FB0111928A95E9F766
:10ACC0008AEC98E040E650E00E94C35A182FC5E98C
:10ACD000D1E088810E94C62D0E94D62D8993F1E093
:10ACE000CF39DF07B1F7809144018A3028F4809191
:10ACF00081048160809381048AE0809344011D3443
:10AD000068F0E5E4F1E020E030E081919191280FD6
:10AD1000391F81E0ED35F807C1F702C020E030E0CF
:10AD200081E040916F01509170014217530709F083
:10AD300080E0DF91CF911F9108951F93182FE4EACF
:10AD4000F1E025EA32E0DF01C9011D920197E9F740
:10AD5000CF0168E770E14AE050E00E94D574812F8E
:10AD600090E001966AE070E00E947F74605D6093FD
:10AD7000A901805D8093AA018AE08093AE0180E002
:10AD80000E9427631F910895CF92DF92EF92FF9266
:10AD90000F931F93DF93CF930F92CDB7DEB76B0165
:10ADA000803160F5682F6F5F8AEC98E049830E94DC
:10ADB000375A4981042F10E0C60160E270E050E08C
:10ADC0000E94F6748AEC98E0B6014AE050E00E94D6
:10ADD000C35A8A30910591F48AEC98E00E94295A6E
:10ADE000F601E00FF11F2AE030E006C0B9010E9431
:10ADF0006B74805D8293CB010097C1F70F90CF9168
:10AE0000DF911F910F91FF90EF90DF90CF90089509
:10AE10008F5F0E94BA5908951F93CF93DF93182F25
:10AE2000803168F5682F6F5F8AEC98E00E94375A8E
:10AE300064EA71E025EA32E0FB01C9011192019751
:10AE4000E9F78AEC98E045EA52E00E94C35A8F3F46
:10AE5000910509F018F4812F0E949D56C4EAD1E0B3
:10AE600088810E94C62D0E94D62D899391E0CE3A0A
:10AE7000D907B1F78AE08093AE010E948215DF9175
:10AE8000CF911F9108950F931F93DF93CF93CDB769
:10AE9000DEB760970FB6F894DEBF0FBECDBF682F48
:10AEA0006F5F062F0AC0102F1F5F812F688B0E94D3
:10AEB000BA596889882329F0012F0031A0F30031A5
:10AEC00039F18AEC98E00E94375A602F6F5F83ED6A
:10AED00098E042E028E532E00E94A95B8E010F5F16
:10AEE0001F4F06C083ED98E0B8010E94245BA8952F
:10AEF0008AEC98E0B8014FE050E00E94525A482F87
:10AF0000882381F783ED98E00E94D25B81E001C045
:10AF100080E060960FB6F894DEBF0FBECDBFCF9134
:10AF2000DF911F910F910895EF920F931F930E944D
:10AF3000A559882341F00E94105987FD04C00E9442
:10AF40005156882381F588E690E161E00E94F11274
:10AF500086E590E10E94D8120E947F590E94135604
:10AF60008AEC98E060E041E024E431E000E610E0A3
:10AF700078ECE72E0E94015C8036910529F087E489
:10AF800090E160E00E94F11280E00E949D568AEC00
:10AF900098E061E042E024EA31E005EA12E058EC92
:10AFA000E52E0E94015C809171010E940C571F9157
:10AFB0000F91EF900895882359F09091E608982B0F
:10AFC0009093E6080E94CF0E9093E8088093E708DC
:10AFD0000895EF920F931F93CF93DF931091E6089C
:10AFE000112309F47EC0882309F076C00E94CF0E99
:10AFF0002091E7083091E808AC01421B530B44361E
:10B00000510508F46EC068C081E08093E508812F87
:10B0100090E0EC01C470D07012FF03C023E02093D5
:10B02000E5081092E60880FF1CC08CED98E061E115
:10B0300041E024E431E000E610E0F4E1EF2E0E946C
:10B04000015C8036910511F480E020C08091E20817
:10B05000823021F48091E608816029C087E390E185
:10B0600035C081FF36C08CED98E061E142E024EA12
:10B0700031E005EA12E0E4E1EE2E0E94015C52E0CC
:10B08000853A950739F4809171018F5F61E10E94E3
:10B09000C8591FC08091E2088230A1F48091E6086F
:10B0A000982F92609093E608209719F0866080931D
:10B0B000E6080E94CF0E845690409093E808809353
:10B0C000E70807C0209729F487E290E160E00E943A
:10B0D000F1121092E50805C08091E508882309F473
:10B0E00093CFDF91CF911F910F91EF9008950AC0F8
:10B0F00081E00E94E95780916B0E833019F4A89586
:10B1000010926B0E8091E608882391F70895DF93E3
:10B11000CF930F92CDB7DEB7682F70E084E0660F53
:10B12000771F8A95E1F7CE01019641E050E00E9439
:10B13000FD7489810F90CF91DF910895DF93CF93B4
:10B140000F92CDB7DEB76983682F70E094E0660F89
:10B15000771F9A95E1F7CE01019641E050E00E94F9
:10B16000CA600F90CF91DF91089589EE98E060E07A
:10B1700070E040E450E00E94CA6008958BEE98E0D1
:10B1800062E070E041E050E00E94CA6008950F93D1
:10B190001F93182F082F04C0802F0E948758082F54
:10B1A000802F0E9487588823B9F7802F6091EB0881
:10B1B0000E949E581093EB080E94BE581F910F9159
:10B1C00008951F931091EB08112359F0812F0E94CD
:10B1D00087588093EB080E94BE58812F60E00E9440
:10B1E0009E58812F1F910895F8942091D70D30918A
:10B1F000D80D7894C9010895EF92FF92CF93DF9311
:10B200008091EB08C0E0D0E003C02F960E948758E1
:10B210008823D9F7CE01DF91CF91FF90EF90089569
:10B22000CF92DF92EF92FF920F931F93CF93DF9312
:10B2300080E8E9E2F9E0DF011D928A95E9F70DEE79
:10B2400018E0C0E0D0E08C2FC43139F4D090EB0886
:10B250003BEEE32E38E0F32E0BC07E01EE0CFF1C1C
:10B26000EC0EFD1E2DEE38E0E20EF31ED801DC9050
:10B2700090E0C82EC3941DC08D2D84508C3738F4B7
:10B28000ED2DF0E0E75DF64F8081882361F0992392
:10B2900029F0892F60E00E949E580DC0F7011082AE
:10B2A0000E94B55808C0C0828D2D0E9487589D2DE0
:10B2B000D82EDD2009F721960D5F1F4FC531D1052E
:10B2C00011F604E0E02FF0E0E75DF64F808188237F
:10B2D00049F4802F6091EB080E949E580093EB0880
:10B2E0000E94BE580F5F003869F780E0DF91CF9170
:10B2F0001F910F91FF90EF90DF90CF9008951F93D3
:10B3000080E4E9EEF8E0DF01982F1D929A95E9F7C5
:10B3100094E09093E9088093EA0880E18093EC0838
:10B3200084E001C0812F182F1F5F612F0E949E585B
:10B330001038C1F78FE760E00E949E5884E0809348
:10B34000EB080E94B5581F91089589EE98E060E0DF
:10B3500070E040E450E00E94FD748091E908843080
:10B3600039F481E09091EA08903419F080E0089572
:10B3700080E0089590E0FC01EE0FFF1FE80FF91F39
:10B38000E751F74F81E09481992309F480E0089513
:10B39000DF93CF9300D00F92CDB7DEB790E0FC01E2
:10B3A000EE0FFF1FE80FF91FDE011196E351F74F73
:10B3B00023E001900D922150E1F770E0DC01AA0F2B
:10B3C000BB1FA80FB91FFB01EE0FFF1FE60FF71FF2
:10B3D000A351B74FE351F74F83E001900D92815095
:10B3E000E1F7FB01EE0FFF1FE60FF71FE351F74FE9
:10B3F000DE01119683E00D9001928150E1F70E94E9
:10B40000B5580F900F900F90CF91DF910895DF9373
:10B41000CF930F92CDB7DEB790E09C01220F331F80
:10B42000280F391FF901E751F74F84812351374F16
:10B4300093E0D9011D929A95E9F789830E94B55846
:10B440008981882311F00E94C7580F90CF91DF9116
:10B450000895FC01808190E0FC01EE0FFF1FE80FD2
:10B46000F91FE251F74F918180819F700895FC018F
:10B4700060831282118270E0CB01880F991F860FC2
:10B48000971FDC01A751B74F14962C911497238373
:10B490001482158216828151974FFC01808182951A
:10B4A0008F7008958F929F92AF92BF92CF92DF924A
:10B4B000EF92FF920F931F93DF93CF930F92CDB72D
:10B4C000DEB78C015B01FC01808190E0FC01EE0F96
:10B4D000FF1FE80FF91FE251F74F80812181922F62
:10B4E0009F70F80121813281821B930BE42EF52E8F
:10B4F0008E159F0508F47C0167014E010894811C9C
:10B50000911C25C0F8016381662321F184818F5F3E
:10B51000848370E0B4E0660F771FBA95E1F7680F97
:10B52000711DC40141E050E00E94FD748981F50164
:10B5300081935F01F80184818F3030F01482838120
:10B540000E948758F80183830894C108D108C11468
:10B55000D104C1F6F801818192818E0D9F1D8C1955
:10B560009D09928381838E2D8C190F90CF91DF914D
:10B570001F910F91FF90EF90DF90CF90BF90AF9011
:10B580009F908F9008958F929F92AF92BF92DF927B
:10B59000EF92FF920F931F93CF93DF938C015B0188
:10B5A0007A01C0E0D0E045E0842E912C880E991EEF
:10B5B0003BC0F801858190E08F779070009741F44F
:10B5C000C801B40141E050E00E94525A813079F53F
:10B5D000F80145813FE7D32ED4222D2D30E0C7015D
:10B5E0008C1B9D0B8217930710F4DE2CDC1AB5011F
:10B5F0006C0F7D1F47FF08C0CB0160E070E04D2D50
:10B6000050E00E94F6740AC0C8014D2D50E00E941F
:10B61000525A8D1519F0C80FD11D09C0CD0DD11D7D
:10B62000F80185818D198583CE15DF0510F2CE01D5
:10B63000DF91CF911F910F91FF90EF90DF90BF901E
:10B64000AF909F908F9008959F92AF92BF92CF92AC
:10B65000DF92EF92FF920F931F93CF93DF93EC0152
:10B660008B01C42E8B81882389F489819A8100976C
:10B6700069F4E880FF240E94E1588B83F701EE0F04
:10B68000FF1FEE0DFF1DE751F74F8483DC2C6FE0A9
:10B69000962E44C0EF80F8840E94CF0EE81AF90A73
:10B6A000F7FE02C082E004C08B81882319F481E098
:10B6B0008E8337C09C819F3080F01C820E94875807
:10B6C000882339F4EB800E94E158682F8E2D0E9468
:10B6D0009E588B810E9487588B838B81882339F3F6
:10B6E0006C81992D961BED2C9D1508F4E92EAE2C3E
:10B6F000BB2470E06F5F7F4F90E054E0880F991F8C
:10B700005A95E1F7680F791FC801A5010E94CA6028
:10B710000A0D1B1D8C818E0D8C83DE18DD2009F037
:10B72000B9CF2C2D30E02D19310989819A81820FF2
:10B73000931F9A8389838C2D8D19DF91CF911F914F
:10B740000F91FF90EF90DF90CF90BF90AF909F90C0
:10B7500008950F931F93CF93DF93EC0189016883C2
:10B760001A82198270E0CB01880F991F860F971FEC
:10B77000FC01E751F74F24812B831C821D821E821E
:10B78000FC01E251F74F10824295407F41830E94B5
:10B79000CF0E080F191F18870F83DF91CF911F91CC
:10B7A0000F9108951F93CF93DF93EC01888190E070
:10B7B000FC01EE0FFF1FE80FF91FE251F74F8981DF
:10B7C00080839A819F708181807F892B81838B8187
:10B7D000882389F00E948758182F882361F08B8175
:10B7E00060E00E949E580E94B558112331F0812FCD
:10B7F0000E94C75802C010E0F6CFDF91CF911F9191
:10B8000008954F925F926F927F929F92AF92BF92F4
:10B81000CF92DF92EF92FF920F931F93DF93CF931C
:10B820000F92CDB7DEB75C01290168012E2D30E003
:10B830000E94A95B1982720100E010E081E03E01E4
:10B840000894611C711CF70191917F01992341F4C7
:10B85000882349F49081992349F4992493941EC034
:10B86000882371F403C09924939401C09924998189
:10B870009F3718F40C151D0561F5882379F001C078
:10B8800099248981882321F180688983C501B301C6
:10B8900041E00E94245B8130D1F025C0898188235A
:10B8A000B9F0C501B30141E00E94245B8130D9F4B5
:10B8B0004981B801641B7109640D751DC5010E94A1
:10B8C000245B9981891719F0981B99830CC0198200
:10B8D000892D99819F5F99830F5F1F4FC016D106F5
:10B8E00008F0B1CF05C089818F776801C81AD108E7
:10B8F000C5010E94D25BC6010F90CF91DF911F91CD
:10B900000F91FF90EF90DF90CF90BF90AF909F90FE
:10B910007F906F905F904F90089580E094E0E9EA07
:10B92000F9E0DF019C011D9221503040E1F70895BC
:10B930000F931F93CF93DF93DA011196FA0144918D
:10B94000ED012196FD01A491B0E0179613E0B595A5
:10B95000A7951A95E1F71A2FDE011196FE01949131
:10B96000929FE0011124AC0FBD1F00FD08C001FF34
:10B9700008C09091D90D51E096FD04C002C051E07D
:10B9800001C050E066956695669570E09B0136951E
:10B99000322F22273795279590E0280F391F610F06
:10B9A000711D7695762F662777956795680F791FB5
:10B9B000042F10E014C0E901C755D64F80E090E095
:10B9C00008C0FD01E80FF91FE4915111E095E993DA
:10B9D00001968417B0F3A00FB11F20583F4F2617D0
:10B9E000370749F7DF91CF911F910F910895FF928B
:10B9F0000F931F93CF93DF93942F46313CF4440F62
:10BA0000490F440F22FFABC0440FA9C0482F4A5F23
:10BA1000092F112707FD109520FD09C021FF0AC03D
:10BA20003091D90DFF24F39436FD05C003C0FF24E7
:10BA3000F39401C0FF2466956695669570E076954F
:10BA4000762F662777956795680F711DEB01C755AF
:10BA5000D64F22FF4FC09E3209F04A5FC80180973F
:10BA600060E170E00E947F7480EA90E0689F90013E
:10BA7000699F300D789F300D1124C801880F991FE0
:10BA800053E0000F111F5A95E1F7800F911F280F07
:10BA9000391F2C5C3E4E85E0882369F0F9019491B2
:10BAA000E056FF4F54912F5F3F4FF9016491E056EC
:10BAB000FF4F749104C060E050E090E070E0FF2020
:10BAC00021F09095609550957095DE01AF57BF4F6E
:10BAD000FDE0A93ABF0740F498836983FE01E0586E
:10BAE000FF4F50837C93229681508F3FC1F12F5F8F
:10BAF0003F4FD2CF23FF0DC0FF2011F08FEF01C0C9
:10BB000080E06755764FFB01808321964F5F91E07F
:10BB100001C090E09801220F331F220F331F200F26
:10BB2000311F2F50304F85E0F9012F5F3F4FE491D7
:10BB3000992311F0843039F0FDE0C93ADF0718F499
:10BB4000F110E095E993815079F75DE0C93AD507A6
:10BB500030F4FF2011F08FEF01C080E08883842F44
:10BB6000DF91CF911F910F91FF90089520E00E94E7
:10BB7000F75C0895CF92DF92EF92FF920F931F939D
:10BB8000CF93DF93162FF22EF0E1EF2EE022C42E9A
:10BB9000E6016E01D52EE6010CC0EE2011F04881C1
:10BBA00002C0FE014491612F202F0E94F75CFA949D
:10BBB0002196FF2091F7DF91CF911F910F91FF9078
:10BBC000EF90DF90CF9008950F9300E00E94BA5D50
:10BBD0000F910895CF92DF92FF920F931F93CF930F
:10BBE000DF93162F022FA0E1FA2EF222C42EE601D7
:10BBF0006E01D52EE601FF2011F0488102C0FE0142
:10BC000044912196442329F0612F202F0E94F75C54
:10BC1000F2CFDF91CF911F910F91FF90DF90CF90E6
:10BC20000895982FAB0180E0692F20E00E94EA5D23
:10BC3000089520E00E94EA5D0895EF92FF920F932D
:10BC40001F93DF93CF930F92CDB7DEB7182F062F38
:10BC50007A01982F9C5E95504E2D4F704A301CF003
:10BC6000495C28E002C0405D20E0892F602F998365
:10BC70000E94F75C9981911731F0B4E0F694E79453
:10BC8000BA95E1F7E8CF0F90CF91DF911F910F9117
:10BC9000FF90EF900895E62FE695E695E695F0E0A3
:10BCA000F695FE2FEE27F795E795E80FF11DE7557E
:10BCB000F64F8DE0E93AF80758F4677081E090E0BC
:10BCC00002C0880F991F6A95E2F7208128272083F8
:10BCD000089547FF02C0840F4195E62FE695E6954B
:10BCE000E695F0E0F695FE2FEE27F795E795E80F3D
:10BCF000F11DE755F64F6770A1E0B0E001C0AA0F53
:10BD00006A95EAF711C08DE0E93AF80778F4822FD6
:10BD100090E09C013595279580FF04C080818A279B
:10BD20008083206841503196442369F708952FEFAE
:10BD30000E94695E08950F931F93CF93DF93C82FDE
:10BD4000D0E0E62FE695E695E695F0E0F695FE2F35
:10BD5000EE27F795E795EC0FFD1FE755F64F062FF9
:10BD600010E0242F332727FD3095200F311FC90104
:10BD700068E070E00E947F747695762F662777954D
:10BD800067956C0F7D1F6755764F0770107081E0C7
:10BD900090E002C0880F991F0A95E2F78195908183
:10BDA000892708C0E058FF4F8DE0E93AF807D0F442
:10BDB000808180958083E617F707A0F38DE0E93A4C
:10BDC000F80780F4C90168E070E00E947F7421E008
:10BDD00030E002C0220F331F8A95E2F7219580815F
:10BDE00082278083DF91CF911F910F9108952F9229
:10BDF0003F924F925F926F927F928F929F92AF92FB
:10BE0000BF92CF92DF92EF92FF920F931F93DF9337
:10BE1000CF9300D00F92CDB7DEB7182F662E590101
:10BE20006A01F02E802F05FF04C004FF04C002E069
:10BE300003C000E001C001E0E7FE04C0E194222459
:10BE4000239401C02224D7FE0BC0D094C094B09498
:10BE5000A094A11CB11CC11CD11C4424439401C05A
:10BE6000442482FF06C09CE09093A90D3AE0932EF3
:10BE700005C096E09093A90D25E0922E86FF2FC075
:10BE80004110190D28EEA21623E0B20620E0C206EA
:10BE900020E0D20614F0190D06C034E6A316B10452
:10BEA000C104D10414F0190D06C08AE0A816B1042B
:10BEB000C104D1040CF0190D002391F0023039F4C3
:10BEC000E4E6AE16B104C104D10454F4190DFAE04D
:10BED000AF16B104C104D1041CF4190D01C0191B23
:10BEE0008091A90D810F8093A90D023011F420EFEC
:10BEF000F20E5524539492E0792E88242E2D332768
:10BF000027FD3095862D8A5F89833B832A8370C005
:10BF1000C601B5012AE030E040E050E00E94B47470
:10BF2000E62E80E3382E3E0C812F662D432D2F2DDB
:10BF30000E94F75C0515D9F5F2FE23C08E2D8150C5
:10BF4000833008F47394C601B5012AE030E040E084
:10BF500050E00E94B474CA01B9012AE030E040E028
:10BF600050E00E94B474623011F06430C1F4E32DEB
:10BF7000E43319F4812E839413C0812E8A94739430
:10BF80000FC01250812F8F5FF0FE05C0662D47E075
:10BF90000E949B5E05C069810E944B5E01C0812E9C
:10BFA000FAE0AF16B104C104D1040CF000E0C60100
:10BFB000B5012AE030E040E050E00E94B47459013D
:10BFC0006A01211531054105510581F4002331F045
:10BFD000023059F4252D223040F408C0F4FE10C080
:10BFE000222021F430EFF30E01C000E01919539420
:10BFF000852D90E0EA81FB81E817F9070CF088CFE6
:10C00000882061F0662D645F882D472D0E94975E21
:10C01000662D635F882D472D0E94975E442039F07E
:10C02000812F8919662D4DE22F2D0E94F75C0F900C
:10C030000F900F90CF91DF911F910F91FF90EF9094
:10C04000DF90CF90BF90AF909F908F907F906F9038
:10C050005F904F903F902F900895EF920F93022F93
:10C06000FA019F01442737FD4095542F75E0E72ED4
:10C070000E94F75E0F91EF90089520E00E942D60DE
:10C080000895A998AB98AC988BBBAD9AAD98AB9A34
:10C09000A99A089520E030E006C045E04A95F1F7FE
:10C0A00000002F5F3F4F28173907BCF30895AA9867
:10C0B00085E08A95F1F7000085E08A95F1F70000A8
:10C0C000AA9A8CED95E00E944A6082EE0E9441603F
:10C0D0008EEA0E94416081EA0E94416086EA0E94E5
:10C0E000416084EA0E94416082EA0E94416080ECE3
:10C0F0000E9441608FE20E94416085E20E9441609F
:10C1000081E80E94416082E20E9441608FEA0E94C1
:10C11000416082E28093720108951F93182F81E895
:10C120000E944160812F0E9441601F9108951F93DA
:10C13000CF93DF9310E0C9EAD9E084E00E94416028
:10C1400080E10E944160812F806B0E944160A9982C
:10C15000AB9AAC98FE0180E290819BBBAD9AAD9802
:10C1600091819BBBAD9AAD9892819BBBAD9AAD98E6
:10C1700093819BBB3496AD9AAD98815069F7C058B6
:10C18000DF4FAB9AA99A1F5F1830B9F6DF91CF91B4
:10C190001F910895BF92CF92DF92EF92FF920F937B
:10C1A0001F93CF93DF93EA01E82EF92E062F172F66
:10C1B00021C0F701B1907F0168010894C11CD11C16
:10C1C00004C0009739F00E9409198091E50890E0B9
:10C1D00082709070E199F5CF1FBB0EBBE09A8DB3D2
:10C1E000B81631F0BDBA8FB7F894E29AE19A8FBFD2
:10C1F000219786012097E9F6DF91CF911F910F914A
:10C20000FF90EF90DF90CF90BF9008958093DA0D6C
:10C2100008958091DA0D1092DA0D0895FC01808165
:10C22000982F990F9E70807F892B8083662321F041
:10C230009160807F892B808381818F5F8183928150
:10C24000992391F020812F7079F4933659F0242F9F
:10C2500020622093DA0D903111F4803118F0808142
:10C260008F7C8083118212828281883009F443C0DE
:10C27000893058F4813009F446C08130A0F0823012
:10C28000D1F1843009F052C036C08F3549F1803683
:10C2900020F4803109F04AC02EC0813689F0823600
:10C2A00009F044C03DC08081982F9F709F30F1F508
:10C2B00091E6928391819131E0F08F7C808319C067
:10C2C00040664093DA0D9081892F82958F708F5F41
:10C2D00083708295807F9F7C982B90838FE508C028
:10C2E0008181883111F4406818C08832F9F480E106
:10C2F0008283118208959181903328F090E0959582
:10C30000879582831182828190E00197218130E0BC
:10C3100082239323009751F440644093DA0D0895EB
:10C320008181803418F088E08283118208958E30F4
:10C3300091056CF4FC01EE0FFF1FE80FF91FE355A8
:10C34000F24F90819F7081E09F30E9F53FC08231CC
:10C3500031F1833160F48F30C9F0803118F48E30C0
:10C3600091F52AC0803161F0813169F513C08431C3
:10C3700051F08431D0F08531E1F0863121F51EC0D5
:10C3800091B194701DC093B390781AC090916300DE
:10C39000917016C0909163009095987011C0809133
:10C3A000630083FF12C091B102C091B19095907467
:10C3B00007C091B1907104C093B3F9CF91B190725D
:10C3C00081E0992319F480E0089580E008958F704A
:10C3D0008E3058F490E0FC01EE0FFF1FE80FF91FBC
:10C3E000E355F24F82E68283118208958F708E307A
:10C3F00068F490E0FC01EE0FFF1FE80FF91FE35512
:10C40000F24F83E6828380818F7C808308950F932F
:10C410001F93CF93DF938091D70D9091D80D019604
:10C420009093D80D8093D70D8091D90D8F5F809315
:10C43000D90D06B3009540E050E010E001C0AE0118
:10C44000EA012196CA01880F991F840F951FB80130
:10C450000C2E02C0759567950A94E2F761707070B2
:10C460008355924F50E00E940E61C630D10539F7D6
:10C4700000B30095C0E0D0E0FE01EC50F64EE49130
:10C480009E012A5F3F4FC901880F991F820F931F9A
:10C490008355924FE02361E009F460E09E012A5F3A
:10C4A000422F50E00E940E612196C830D10521F73D
:10C4B000DF91CF911F910F910895FF920F931F93DA
:10C4C000CF93DF93F82EEEEBF1E080E090E0582F71
:10C4D0009C014081F41638F0442329F001963A96E5
:10C4E00081329105A1F75032B9F1E901CC0FDD1F7E
:10C4F000C901A3E0880F991FAA95E1F7C80FD91FBA
:10C500008E0102541E4FA9014F5F5F4FCA01880F71
:10C51000991FE3E0440F551FEA95E1F7840F951F3B
:10C5200020953095205E3F4FA901440F551F63E0D1
:10C53000220F331F6A95E1F7420F531F82549E4F1B
:10C54000B8010E94E4748AE0D8011D928A95E9F747
:10C55000CC55DE4FFA8E02C00EEB11E0C801DF9120
:10C56000CF911F910F91FF90089580E491E0EEEB41
:10C57000F1E0DF019C011D9221503040E1F7089568
:10C58000EAE8F3E088E2DF011D928A95E9F7B896C0
:10C5900088E4DF011D928A95E9F70895282F30E09D
:10C5A0008830C0F4462F572FDA01F901EE0FFF1F34
:10C5B000EE0FFF1FE20FF31FE657FC4F95E0899F38
:10C5C000C001112481579C4F2D912193E817F90741
:10C5D000D9F70895462F572FDA0128503040F90136
:10C5E00093E0EE0FFF1F9A95E1F7E20FF31FEE5471
:10C5F000FC4F99E0899FC00111248D589C4F2D91CB
:10C600002193E817F907D9F7089590E00197FC0105
:10C61000EE0FFF1FE80FF91FEC55FE4FDF01A85A80
:10C62000BD4F6C93DF01AA5ABD4F4C93E95AFD4FA1
:10C6300020830895E0918801F0E0EE0FFF1FEE0FD8
:10C64000FF1FE80FF11DE151FB4F849108958F9278
:10C650009F92AF92BF92CF92DF92EF92FF920F9391
:10C660001F93DF93CF93CDB7DEB76D970FB6F894D6
:10C67000DEBF0FBECDBFF82EDE011596E6E2F1E07B
:10C6800085E001900D928150E1F7DE011A96E1E21A
:10C69000F1E085E001900D928150E1F7DE011F96F7
:10C6A000ECE1F1E085E001900D928150E1F7DE01CF
:10C6B0005496E7E1F1E085E001900D928150E1F7B9
:10C6C000DE015996E2E1F1E085E001900D928150A2
:10C6D000E1F719821A821B821C82E0918D01F0E041
:10C6E000E852FB4F26E030E011E0E491CE2EDD244D
:10C6F000BE016F5F7F4F0FC04F5F5F4FA417B5073D
:10C7000011F4FC01108344305105B1F71F5F225032
:10C710003040153081F040E050E0C601022E02C0EA
:10C72000959587950A94E2F783709070DC011196D5
:10C73000860F971FE1CFFF2041F50E94B5628981E6
:10C740000E945D628C0181E00E941A63F80181837E
:10C7500074E6F72EF2828A810E945D628C0182E08B
:10C760000E941A63F8018183F2828B810E945D62CC
:10C770008C0183E00E941A63F8018183F2828C812C
:10C780000E945D628C0184E07EC0FF2DF13071F467
:10C790008B810E945D62FC0188E081838CE9828349
:10C7A000F3828781817F84608783D7C18F2D823018
:10C7B000E9F58B810E945D62FC0108E001836CE970
:10C7C000F62EF28285E183838781817F846087836F
:10C7D0008EE00E945D62FC0182E2818314E6128396
:10C7E0008EE00E945D62FC010183F28284E183831A
:10C7F0008781817F846087838EE00E945D62FC0177
:10C800000183128381E083838781817F84608783B2
:10C8100083E00E941A63482F8BE062E02DE90E94BA
:10C8200005638CE061E042E220E095C1EF2DE3304A
:10C8300081F50E94B562E9808E2D0E945D628C01B7
:10C8400081E00E941A63F801818354E6F52EF2829A
:10C850008E2D0E945D628C0182E00E941A63F801B5
:10C8600081838CE98283EA808E2D0E945D628C0137
:10C8700081E00E941A63F8018183F2828E2D0E946A
:10C880005D628C0182E00E941A63F8018183F2826A
:10C8900064C1FF2DF43081F50E94B562EA808E2DCF
:10C8A0000E945D628C0182E00E941A63F80181831C
:10C8B00044E6F42EF2828E2D0E945D628C0184E0AB
:10C8C0000E941A63F8018183F282EC808E2D0E940F
:10C8D0005D628C0182E00E941A63F8018183F2821A
:10C8E0008E2D0E945D628C0184E00E941A63F80123
:10C8F00081838CE9828331C1FF2DF53009F0D0C0EE
:10C900000E94B5620E94C06281E00E945D62FC01EB
:10C910003AE0C32EC18224E6B22EB28282E00E94A7
:10C920005D62FC019BE0D92ED182B28283E00E943D
:10C930005D62FC018CE0E82EE182B28284E00E941C
:10C940005D628C0181E00E941A63F8018183B282EA
:10C9500085E00E945D628C0183E00E941A63F80109
:10C960008183B28204E0A02EA38287E08483878142
:10C970008160878385E00E945D628C0183E00E9474
:10C980001A63F8018183B282F38218E0812E8482D7
:10C9900087818160878385E00E945D628C0183E0EE
:10C9A0000E941A63F8018183B282B6E0BB2EB38283
:10C9B000A9E09A2E948287818160878385E00E9416
:10C9C0005D62FC0181828CE9828381E083838781BF
:10C9D000817F8460878386E00E945D62FC01918292
:10C9E0008EE1828388EF83838BE00E945D628C01FD
:10C9F00083E00E941A63F801818376E4972E928285
:10CA0000A382C4828781816087838BE00E945D62FC
:10CA10008C0183E00E941A63F80181839282F38281
:10CA2000D4828781816087838BE00E945D628C0164
:10CA300083E00E941A63F80181839282B382E482C8
:10CA40008781816087838091BA018F718062809332
:10CA5000BA018FE18093BB0180E0BE016B5F7F4F25
:10CA60000E94CE6281E0BE01665F7F4F0E94CE626F
:10CA700082E0BE01615F7F4F0E94CE6283E0BE0113
:10CA80006C5E7F4F0E94CE628E01075E1F4F84E076
:10CA9000B8010E94CE6285E0B8010E94CE625DC0FE
:10CAA000FF2DF630B1F486E00E945D62FC01F18258
:10CAB00082E3828388EF838314E6108786E00E94F6
:10CAC0005D62FC01F1828EEC828388E083831087B3
:10CAD00044C08F2D873009F040C08FE00E945D6216
:10CAE000FC0184E2818384E6828388E8868380E196
:10CAF0000E945D62FC0189E081830EE602838AE088
:10CB0000838380E10E945D62FC0118E0118382E969
:10CB100082838BE083838781817F8460878380E148
:10CB20000E945D62FC01118302838CE08383878114
:10CB3000817F8460878381E06BE043E224E20E948E
:10CB4000056382E061E043E229E60E94056383E039
:10CB500062E043E227E90E94056382E00E94DB571E
:10CB60000E9477586D960FB6F894DEBF0FBECDBF0A
:10CB7000CF91DF911F910F91FF90EF90DF90CF90B9
:10CB8000BF90AF909F908F9008956F927F928F92F9
:10CB90009F92AF92BF92CF92DF92EF92FF920F934C
:10CBA0001F93CF93DF938091BA0181FF03C060E0B0
:10CBB00075E002C060E074E09091B70184E69802ED
:10CBC000C0011124885A9D4FE091BD01FF27E7FD68
:10CBD000F09548EE53E0E49F9001E59F300DF49FFF
:10CBE000300D112428533045AA24BB24A81AB90AB1
:10CBF000281B390BF5E2EF2EF5E0FF2E4091B40132
:10CC0000440F485F50E0440F551F440F551F4552D5
:10CC1000524FEBEDFDE0CC24DD24C61AD70AA8E57F
:10CC2000B2E0A81BB90B1CC0E701699079907E01A6
:10CC30004B01661677060CF4430184018C149D04A5
:10CC40000CF48601005A164FE501C01BD10B2C0FC6
:10CC50003D1F0A0F1B1F1183008393838283349629
:10CC6000E417F50709F731832083938382831582C4
:10CC70001482DF91CF911F910F91FF90EF90DF9081
:10CC8000CF90BF90AF909F908F907F906F900895BE
:10CC9000E0912B01F0912C018193F0932C01E09312
:10CCA0002B010895FF920F931F93CF93DF93B9E069
:10CCB000FB2E90E120E0C82FD0E08E0101701070B3
:10CCC000201711F4905F07C0892F90E001970E9410
:10CCD0004866202F90E1FA9431F0D595C795AE01C2
:10CCE0004068842FE8CF892F90E00F960E94486615
:10CCF000DF91CF911F910F91FF9008951F93CF93D4
:10CD0000DF93182F2BED3DE030932C0120932B0166
:10CD100080913101877471F08091B401882319F0FA
:10CD2000813029F402C080E803C080E901C088E9AD
:10CD3000809331018091310187FF0BC086E190E043
:10CD40000E949761882329F4809131018F77809325
:10CD500031018091310187FD5AC085E160E040E0FA
:10CD60000E94A210882309F452C080913101806290
:10CD700080933101809171018F5F80933201E3E3F1
:10CD8000F1E0A5E2B5E080E01CC02D913D91359524
:10CD9000279520503E4F37FD05C093E02F3F3907C0
:10CDA00024F405C020E030E002C02FEF33E0932FE1
:10CDB0009370482F440F440F942B908321838F5FEF
:10CDC0003296811711F7C1E3D1E089910E94526632
:10CDD00081E0CF33D807C9F780912B0190912C01C6
:10CDE000019790932C0180932B018FEF90E00E948C
:10CDF000486680E090E00E9448668BED9DE090934D
:10CE0000300180932F01DF91CF911F910895809180
:10CE100031018F7DADCF1F920F920FB60F9211246B
:10CE20002F938F939F93EF93FF9388B391E089277C
:10CE300088BBE0912F01F09130012191F0933001F6
:10CE4000E0932F01822F90E097BD86BD293C08F02A
:10CE5000C09A80916B0E816080936B0EFF91EF9171
:10CE60009F918F912F910F900FBE0F901F9018954B
:10CE70001F920F920FB60F9211242F933F938F930F
:10CE80009F93EF93FF9388B391E0892788BBE0914C
:10CE90002B01F0912C01208130E020FD04C088B5E9
:10CEA00099B5809603C088B599B5409699BD88BD5F
:10CEB000C90195958795009791F4CF0101969093BC
:10CEC0002C0180932B018181882351F4809178007B
:10CED000909179008053984F99BD88BD01C080839F
:10CEE00080916B0E816080936B0EFF91EF919F910B
:10CEF0008F913F912F910F900FBE0F901F9018951B
:10CF0000EDE7F0E08081857E808317981F9AAAE87C
:10CF1000B0E01C9210928B0082E88C93808180623A
:10CF200080830895EDE7F0E080818F7D8083179AFC
:10CF3000AAE8B0E01C9210928B008AE08C9380816A
:10CF40008861808308951F920F920FB60F9211246B
:10CF50008F939F93AF93BF93EF93FF938091770E3F
:10CF6000882321F01F9A1092770E04C01F9881E049
:10CF70008093770EA0912D01B0912E01FD0181913A
:10CF800091919093870080938600F0932E01E09317
:10CF90002D0180916E0E90916F0E9093850080937D
:10CFA000840012968D919C911397009759F483E217
:10CFB0009EE090932E0180932D018091BA018170A3
:10CFC0008093770E80916B0E816080936B0EFF9142
:10CFD000EF91BF91AF919F918F910F900FBE0F90E6
:10CFE0001F901895AF92BF92CF92DF92EF92FF926F
:10CFF0000F931F93CF93DF938091BA0181FF03C0FA
:10D0000040E055E002C040E054E0F090B401FF0C75
:10D0100080E1F80E2091B70184E6280290011124E6
:10D02000285A3D4FE091BD01FF27E7FDF09568EEDE
:10D0300073E0E69FC001E79F900DF69F900D1124CD
:10D0400088539045CC24DD24C21AD30A821B930B4B
:10D0500068EFE62EEF0CE3E2FEE000271127041B49
:10D06000150B68E572E0621B730B21C0AE2DB0E0BA
:10D07000AA0FBB1FAB5DBA4FAC901196BC90D50107
:10D080004A175B070CF4DA01A017B1070CF4D801BA
:10D09000A05AB64FE601CA1BDB0B8C0F9D1F3183D4
:10D0A0002083A60FB71FB383A2833496E394EF14B3
:10D0B000E8F23183208393838283885E9340909348
:10D0C0006F0E80936E0E15821482DF91CF911F91A7
:10D0D0000F91FF90EF90DF90CF90BF90AF900895A9
:10D0E0001F920F920FB60F9211242F933F934F93DD
:10D0F0005F936F937F938F939F93AF93BF93EF93C0
:10D10000FF9378940E94F267FF91EF91BF91AF91E6
:10D110009F918F917F916F915F914F913F912F914F
:10D120000F900FBE0F901F9018952091740E3091A4
:10D13000750E90E0822793279070880F991F805A70
:10D14000954EFC0145915491232F332742275327B5
:10D150005093750E4093740E08959091700E9695AD
:10D160009695982B9093700E8091710E8F5F80939F
:10D17000710E843068F0E091720EF091730E91930D
:10D18000F093730EE093720E1092700E1092710E67
:10D19000089503C080E00E94AD688091710E8823DD
:10D1A000C9F7E091720EF091730E108208958823F2
:10D1B00039F08091760E8F5F8093760E80E803C001
:10D1C0001092760E80EC0E94AD688091760E8530CC
:10D1D000B8F708950F931F93182F0E94956808E0E1
:10D1E000812F81700E94D76816950150C9F71F9151
:10D1F0000F91089580EC0E94AD6880E80E94AD68B0
:10D2000080E80E94AD6880E80E94AD6880E80E94D6
:10D21000AD6880E80E94AD6880E80E94AD6880EC4F
:10D220000E94AD680895AF92BF92CF92DF92EF92C5
:10D23000FF920F931F93CF93DF938BED9DE090931D
:10D240002C0180932B019093730E8093720E109299
:10D25000750E1092740E1092700E1092710E109244
:10D26000760E0E94FA688091B4010E94EA6880916B
:10D270006D0E0E94EA6880E00E94EA6810926D0ECE
:10D2800005E215E054E0C52ED12CF8012081318152
:10D29000C901880F991F820F931FB6010E947F74E6
:10D2A000EB0122813381C901880F991F820F931FDF
:10D2B000B6010E947F7460507C4FC050DC4FF8E094
:10D2C000C030DF0710F0CFEFD7E07B0128E06030FF
:10D2D000720720F0AFEFEA2EA7E0FA2E8C2F0E9403
:10D2E000EA685E019B2D9F708E2D8295807F892B31
:10D2F0000E94EA68C701F4E096958795FA95E1F7F0
:10D300000E94EA680C5F1F4F25E00533120709F001
:10D31000BCCF0091750E8091740E0E94EA68802F38
:10D320000E94EA680E94FA680E94C96880917800A9
:10D3300090917900805C9346909379008093780077
:10D34000C09ADF91CF911F910F91FF90EF90DF90E6
:10D35000CF90BF90AF9008958091B30190916C0EE3
:10D36000981709F494C080936C0E8130F9F08130E5
:10D3700030F08230F1F1833009F089C05EC00E9444
:10D3800080671EBC80E49CE99BBD8ABD1DBC1CBCA3
:10D3900087B7837C87BF8CE386BF8FE380937C0055
:10D3A00087B7806187BF1FBC8AE021C00E94806769
:10D3B0001EBC1DBC1CBC80E797E199BD88BD80EAFE
:10D3C0009FE0909379008093780087B7837C87BF34
:10D3D0008CE386BF8FE380937C0087B7886087BF2C
:10D3E00080917D00816080937D001FBC82E08EBDB6
:10D3F0004EC00E9480671EBC88EC90E0909379003C
:10D40000809378008CE291E09DBD8CBD80EE9BEA1C
:10D4100097BD86BD87B7837C87BF8CE386BF8FE3CC
:10D4200080937C0087B7806287BF80917D00816098
:10D4300080937D001FBC8AE1DACF1EBC80E49CE9AA
:10D440009BBD8ABD1DBC1CBC87B7837C87BF8091F8
:10D450007D008E7F80937D008CE386BF8FE3809379
:10D460007C0087B7806187BF1FBC8AE08EBD0E94A9
:10D47000F26780E593EC909387008093860088E8BC
:10D4800093E190938500809384000E94926780913D
:10D49000B301813051F0813028F0823051F0833077
:10D4A00079F40CC00E94C565089578940E941369B0
:10D4B0000895789486E00E947E6608950E94C5656E
:10D4C00008951F920F920FB60F9211242F933F933E
:10D4D0004F935F936F937F938F939F93AF93BF937C
:10D4E000EF93FF938091B3018230C1F480E492EA1C
:10D4F00097BD86BD80917800909179008F3F91050E
:10D5000038F488E598E9909379008093780008C012
:10D5100088EC90E090937900809378000E94AC6949
:10D52000FF91EF91BF91AF919F918F917F916F91FB
:10D530005F914F913F912F910F900FBE0F901F90D1
:10D5400018951F920F920FB60F9211242F933F93AD
:10D550004F935F936F937F938F939F93AF93BF93FB
:10D56000EF93FF938CB59DB52091780E222321F087
:10D57000C09A1092780E04C0C09821E02093780ED3
:10D58000A0913F01B0914001FD01219131913BBD3E
:10D590002ABDF0934001E0933F012091C5063091F0
:10D5A000C6062817390720F49093C6068093C5064F
:10D5B00020910C0130910D018217930720F4909374
:10D5C0000D0180930C0112968D919C9113970097F9
:10D5D000D9F48BED9DE09093400180933F018091C1
:10D5E000BA01809581708093780E87B78F7E87BF50
:10D5F0000E94AC698091B301882311F0833021F43B
:10D6000087B7806187BF789480916B0E816080932B
:10D610006B0EFF91EF91BF91AF919F918F917F9191
:10D620006F915F914F913F912F910F900FBE0F908F
:10D630001F901895909187019873903121F463E0C1
:10D640000E945F740895983111F486950895983278
:10D6500011F4880F0895903319F4982F990F890FBA
:10D660000895FC01A5E6B0E08C918B7F8C93148229
:10D6700015821082118216A617A608950E94316B9A
:10D68000089521E0FC018481882309F420E0822FA1
:10D690000895FC0181819081891B877098E0981B17
:10D6A00081E0933008F480E00895FC0184818823B0
:10D6B000F9F08150848382819381890F828386A5CA
:10D6C000882309F44CC087A5982F915097A78823E9
:10D6D00031F08091650084608093650008958091A9
:10D6E00065008B7F809365008091920187A70895E4
:10D6F0001B98809165008B7F8093650085818823CE
:10D7000019F081508583089580819181891739F1BD
:10D7100090E0DF01A80FB91F16962C91169722836F
:10D7200056962C91569724831E962C911E972383F0
:10D730005E962C915E972583D0962C91D09726A744
:10D7400017A696962C919697322F315096963C9329
:10D750009697222321F40196877090708083089514
:10D760008F929F92AF92BF92CF92EF92FF920F93C0
:10D770001F93DF93CF9300D0CDB7DEB74C01122FAC
:10D780004A8369830E94496B4A816981882331F108
:10D7900080918701887311F1F401A180BB24C50138
:10D7A000019697E0F92EF8228081F816B9F06623E9
:10D7B00029F080919101865F860F01C080E0A80C5E
:10D7C000B91CF5018683842F0E941A6BF501868BA4
:10D7D000168FE0AA06A3C686F401F1820F900F907F
:10D7E000CF91DF911F910F91FF90EF90CF90BF905D
:10D7F000AF909F908F900895AF92BF92CF92EF928B
:10D800000F93DF93CF9300D00F92CDB7DEB75C01BB
:10D810002B834A8369830E94496B2B814A816981EA
:10D82000882329F180918701887309F1662329F003
:10D8300080919101865F860F01C080E0F5018283AF
:10D84000842F2B834A8369830E941A6BF50184839A
:10D850002B812583E6A617A6C382808181834A8116
:10D860006981002321F00150C5010E94B06B0F9027
:10D870000F900F90CF91DF910F91EF90CF90BF90CD
:10D88000AF900895CF92EF920F93CF93DF93EC0177
:10D8900080918701869586958695877028819981E4
:10D8A000291709F05CC1E62FF0E0E132F10508F03C
:10D8B00056C1EA5BFF4FEE0FFF1F0590F491E02D7C
:10D8C0000994CE0166E44AE0DEC0CE0166E444E19C
:10D8D000DAC0CE0166E44EE1D6C0CE0164E64AE08D
:10D8E00022E002E0EE24E39452E0C52E36C1CE01E0
:10D8F0006FE545E022E00AE0EE24E394CC240E94A8
:10D90000B06BCE016FE545E02AE001E00E94B06B0C
:10D91000CE016FE545E022E00AE01FC1CE0160E5DF
:10D920004AE023E002E0EE24CC24CA940E94B06BCB
:10D93000CE016CE34AE023E0CC24C3940E94B06B98
:10D94000CE0166E44AE021E000E032E0E32E96C03A
:10D95000CE0166E445E021E001E0EE24E394CC242E
:10D960000E94B06BCE0162E34FE022E00E94B06BF8
:10D97000CE0160E54FE022E0F0C0CE016EE645E06A
:10D9800021E002E0EE24E394CC240E94B06BCE01AF
:10D990006CE745E021E02AC0CE0162E345E025E0E6
:10D9A00000E0EE24CC240E94B06BCE016AE545E095
:10D9B00025E00E94B06BCE016EE643E024E002E079
:10D9C000CCC0CE0160E545E02AE003E0EE24E3941C
:10D9D000CC240E94B06BCE0160E545E024E101E07B
:10D9E0000E94B06BCE0160E545E02AE003E0B5C0DF
:10D9F000CE016AE044E125E002E0EE24E394CC2489
:10DA0000C394ABC0CE0162E344E02AE002E0EE241E
:10DA1000E394CC240E94B06BCE0166E448E024E19C
:10DA200001E00E94B06BCE0162E348E02AE002E030
:10DA30000E94B06BCE0166E444E024E101E08DC0B9
:10DA4000CE0168E745E02AE00AE016C0CE0168E7AB
:10DA500045E022E30AC0CE0160E044E12AE001E0B3
:10DA60000BC0CE0160E044E12AE002E005C0CE0137
:10DA700060E044E12AE003E0EE24E394CC246DC0AE
:10DA8000CE0166E448E221E000E048C0813009F4BC
:10DA900066C0CE016BE405C0813009F460C0CE01E0
:10DAA00061E44AE021E000E041C0CE01642F46E09D
:10DAB000F9CFCE0166E44AE022E0E6CF813009F4F6
:10DAC0004EC0CE0166E44AE022E0EDCFCE0168E729
:10DAD000E8CFCE0168E74AE021E01FC0CE016AE747
:10DAE0004AE021E00FC0CE016CE74AE021E004C02B
:10DAF000CE0168E74FE023E003E010C0CE0168E705
:10DB00004FE023E002E00AC0CE0168E74FE023E0E7
:10DB100004C0CE0166E444E129E101E0EE24E3948F
:10DB200006C0CE0166E44AE022E002E0EE24CC2406
:10DB30000E94FC6B14C0CE016CE344E123E002E0E0
:10DB4000EE24CC24C3940E94B06BCE0160E544E186
:10DB500023E0EE24E394CC24CA940E94B06BDF91BE
:10DB6000CF910F91EF90CF900895682F89E494E0C2
:10DB700046E40E94426C0895109818981092900004
:10DB80008FEC89B959981AB886E08093950001C046
:10DB90008CB15F99FDCF1092DD0E1092C10E1092E4
:10DBA000C20E1092C30E1092C40E1092B90E1092B3
:10DBB000BA0E1092BB0E1092BC0E8FEF9FEFAFEF1C
:10DBC000BFEF8093D50E9093D60EA093D70EB0934F
:10DBD000D80E81E08093DE0E0895549857980895EA
:10DBE0001F93182F80E060E040E65CE121E00E9496
:10DBF000EA5D80E660E0412F21E00E94F75C1F9122
:10DC00000895282F30E0F901ED57F14F90819617D4
:10DC100031F4F901E358F14F9081941729F18330E1
:10DC200098F4C901880F991FFC0153E0EE0FFF1F04
:10DC30005A95E1F7E81BF90BE457F14F1082F9010F
:10DC4000E757F14F108205C0F901ED54F14F8FE312
:10DC50008083F901ED57F14F60832358314FF9016B
:10DC6000408381E080937A0E08950F93853251F0BE
:10DC7000863218F48432B9F408C0823871F08338DF
:10DC800091F406C08EEC9EE60CC083E393E709C0D6
:10DC90000E94ED6D8BE49AE104C00E94ED6D8FE46B
:10DCA0009FE30E94331580E067E442E00E94016E2A
:10DCB00083E067E443E00E94016E81E067E444E0B2
:10DCC0000E94016E84E067E445E00E94016E85E0F9
:10DCD00067E447E00E94016E84E30E94F06D82E1F8
:10DCE00068E040E85CE10E94195E80918C0E882318
:10DCF00009F18EE468E04091B60E20E00E94F75CE6
:10DD000082E768E04091B80E20E00E94F75C86E070
:10DD100060E14CE85EE022E004E10E94BA5D8EE141
:10DD200060E140E420E00E94F75C84E260E14EE8BC
:10DD30005EE004C08CE060E141E451E024E10E9437
:10DD4000EA5D82E160E246E75CE10E94195E809153
:10DD50008C0E8823D1F08EE460E24091B70E20E073
:10DD60000E94F75C80E068E24AE95EE023E004E1BB
:10DD70000E94BA5D84E268E240E420E00E94F75C21
:10DD80008AE268E24DE95EE004C08CE068E241E4CA
:10DD900051E024E10E94EA5D0F910895853251F02F
:10DDA000863218F48432B9F408C0823871F08338AE
:10DDB00091F406C083EC90E70CC085E39EE609C0B1
:10DDC0000E94ED6D8BE49AE104C00E94ED6D8FE43A
:10DDD0009FE30E94331580E062E547E00E94016EF8
:10DDE00081E062E548E00E94016E85E067E447E07B
:10DDF0000E94016E83E30E94F06D80E068E044EAD7
:10DE00005CE10E94195E80918C0E8823D1F080E045
:10DE100005C09E3211F4138208C08F5FE82FF0E036
:10DE2000E457F14F90819923A1F780918C0E8823BC
:10DE300019F04CE85EE002C041E451E08CE060E1A2
:10DE400004C08CE060E141E451E024E10E94EA5D1D
:10DE500082E768E04091B80E20E00E94F75C86E01F
:10DE600060E241E95CE10E94195E80919A0E88238C
:10DE700019F04AE95EE002C041E451E08CE068E25A
:10DE800024E10E94EA5D089540E01DC0842F90E0E7
:10DE9000FC01E757F14F10829C01220F331FF9015B
:10DEA000A3E0EE0FFF1FAA95E1F7E21BF30BE45787
:10DEB000F14F1082FC01ED57F14F10828358914FC2
:10DEC000FC0110824F5F433008F34093790E82E0EB
:10DED00067E441E00E94016E81E080937A0E549ADB
:10DEE000579A08951F920F920FB60F9211241F9305
:10DEF0002F933F934F935F936F937F938F939F9352
:10DF0000AF93BF93EF93FF934CB18BB18C7189F0BA
:10DF100010927E0E10927D0E1092840E1092830E3F
:10DF200082E067E441E00E94016E81E080937A0E16
:10DF300040E08AB180917A0E8530C9F1863040F494
:10DF40008330C9F08430E0F4813009F0C6C009C0E4
:10DF5000873009F446C0873070F1883009F0BDC0C1
:10DF600055C0473421F0423509F0B7C002C083E004
:10DF70005CC085E05AC0473409F056C084E055C003
:10DF8000413409F051C087E080937A0E87E4809392
:10DF90007C0E81E080937B0E80E006C0E82FF0E0ED
:10DFA000E757F14F10828F5F8330C0F32CC04D34A0
:10DFB000D9F586E03AC04334B9F587E080937A0E0C
:10DFC00082E580937C0E81E080937B0E80E006C02A
:10DFD000E82FF0E0E757F14F10828F5F8330C0F3F6
:10DFE00012C04C3209F588E080937A0E81E080936C
:10DFF0007B0E80E006C0E82FF0E0E757F14F10827B
:10E000008F5F8330C0F38093790E67C04A3229F066
:10E0100070917B0E4C3281F40BC080917C0E873462
:10E0200019F481E08093DD0E81E080937A0E55C073
:10E030007F5F70937B0E51C010917C0E50E02EC01C
:10E04000852F90E0FC01ED57F14F2081121729F543
:10E05000FC01E358F14F20817217F9F4DC01A75756
:10E06000B14F6C916D30C8F49C01220F331FC90170
:10E07000E3E0880F991FEA95E1F7821B930BFC01FF
:10E08000E60FF11DE457F14F40836F5F6C93860FED
:10E09000911D8457914FFC0110825F5F533080F2D5
:10E0A00050917C0E30917B0E23E013C0822F90E0C4
:10E0B000FC01ED57F14F6081561751F4FC01E35814
:10E0C000F14F6081361721F48D54914FFC0140834C
:10E0D0002F5F263058F32093790EFF91EF91BF9177
:10E0E000AF919F918F917F916F915F914F913F91F0
:10E0F0002F911F910F900FBE0F901F901895EF92C8
:10E10000FF920F931F93CF93DF93E82EE7017E01D9
:10E11000F92EE70100E020E030E0A9011FC01D3228
:10E12000E1F0812F80538A30C8F4CA01B9012AE096
:10E1300030E040E050E00E9440749B01AC01812F30
:10E14000992787FD9095C097AA2797FDA095BA2F8C
:10E15000280F391F4A1F5B1F01C001E019911123CD
:10E16000F1F6002339F050954095309521953F4FB9
:10E170004F4F5F4FB901CA01DF91CF911F910F91AE
:10E18000FF90EF900895EF92FF920F931F938138C5
:10E1900009F495C0823870F48432E9F0853220F4B5
:10E1A000803209F097C036C0853271F0803809F0AE
:10E1B00091C069C08338C1F08338D8F0843821F128
:10E1C000853809F087C01AC08091E00E813031F1A6
:10E1D00083E393E706C08091E00E8130F9F08EEC86
:10E1E0009EE60E94331576C00E94ED6D8BE49AE1A5
:10E1F000F8CF0E94ED6D8FE49FE3F3CF81E0809331
:10E20000E00E1092DE0E63C081E08093E00E8093FA
:10E21000DE0E5DC08091E00E813019F41092E00EA8
:10E2200059C08091B90E9091BA0EA091BB0EB091D9
:10E23000BC0E0097A105B10589F48091BD0E9091A7
:10E24000BE0EA091BF0EB091C00E8093B90E9093F8
:10E25000BA0EA093BB0EB093BC0E08C01092B90EBC
:10E260001092BA0E1092BB0E1092BC0E8091BD0E91
:10E270009091BE0EA091BF0EB091C00E0097A10567
:10E28000B10529F503C081E08093E00E8091D10EA5
:10E290009091D20EA091D30EB091D40E8093B90E6E
:10E2A0009093BA0EA093BB0EB093BC0E8093BD0E9C
:10E2B0009093BE0EA093BF0EB093C00E08C01092F4
:10E2C000CD0E1092CE0E1092CF0E1092D00E87E18E
:10E2D0000E94B56D82E30E94F06D86E068E041ED3A
:10E2E0005CE10E94195E80E668E14CEC5CE10E9412
:10E2F000195E8CE060E247EC5CE10E94195E80E60A
:10E3000068E242EC5CE10E94195E8091DE0E813091
:10E3100029F48CE660E34FEB5CE104C086E660E341
:10E320004BEB5CE10E94195E2091B90E3091BA0E60
:10E330004091BB0E5091BC0E88E760E200E296E08F
:10E34000E92E0E94F75E8091830E873411F01092BF
:10E35000DD0E80E067E449E00E94016E81E067E441
:10E360004BE00E94016E83E067E44AE00E94016E88
:10E3700084E067E446E00E94016E85E067E447E0E0
:10E380000E94016E8091DD0E882309F46CC010920A
:10E39000DD0E8CE89EE00E947F707B018C018AE993
:10E3A0009EE00E947F70E61AF70A080B190BE092B4
:10E3B000D10EF092D20E0093D30E1093D40E809112
:10E3C000CD0E9091CE0EA091CF0EB091D00E8E15A5
:10E3D0009F05A007B10744F4E092CD0EF092CE0E57
:10E3E0000093CF0E1093D00E8091B90E9091BA0E7B
:10E3F000A091BB0EB091BC0EE81AF90A0A0B1B0BD8
:10E40000E092C10EF092C20E0093C30E1093C40EA0
:10E410008091C50E9091C60EA091C70EB091C80E06
:10E42000A8019701281B390B4A0B5B0B2093C90EDF
:10E430003093CA0E4093CB0E5093CC0EE092C50E93
:10E44000F092C60E0093C70E1093C80E57FD0BC076
:10E450008091B70E81333CF08091DE0E882319F055
:10E4600087E10E94B56D80918C0E882309F45CC011
:10E470008EE468E04091B80E20E00E94F75C809145
:10E48000B70E81330CF45EC02091C10E3091C20EE4
:10E490004091C30E5091C40E8CE360E104E217E09A
:10E4A000E12E0E94F75E8091B90E9091BA0EA09174
:10E4B000BB0EB091BC0E2091CD0E3091CE0E40918E
:10E4C000CF0E5091D00EB7FD04C0281B390B4A0B5C
:10E4D0005B0B88E760E100E2B6E0EB2E0E94F75E9E
:10E4E00082E468E14091B60E20E00E94F75C209142
:10E4F000C90E3091CA0E4091CB0E5091CC0E8CE3D8
:10E5000068E204E2A6E0EA2E0E94F75E82E460E39D
:10E510004091B60E20E00E94F75C88E460E348EB8F
:10E520005CE10E94195E0EC08CE060E141E451E0C4
:10E5300024E10E94EA5D8CE068E241E451E024E1DC
:10E540000E94EA5D1F910F91FF90EF900895AF92A6
:10E55000BF92CF92DF92EF92FF920F931F93CF93D0
:10E56000DF93EC016881662309F46DC0772767FDAE
:10E570007095872F972F2AE030E040E050E00E940E
:10E580004074605E7140804090402981332727FDB0
:10E59000309520533040442737FD4095542F620F6B
:10E5A000731F841F951F20E13EE040E050E00E9471
:10E5B00040745B016C016A81772767FD7095872F36
:10E5C000972F28E532E040E050E00E9440747B0144
:10E5D0008C016B81772767FD7095872F972F2CE330
:10E5E00030E040E050E00E944074E60EF71E081F45
:10E5F000191F80E692E8AFEFBFEFE80EF91E0A1F81
:10E600001B1F6C81772767FD7095872F972F2AE056
:10E6100030E040E050E00E944074E60EF71E081F14
:10E62000191F8D81992787FD9095C097AA2797FD7F
:10E63000A095BA2FE80EF91E0A1F1B1FEA0CFB1C3F
:10E640000C1D1D1D03C0EE24FF248701B701C80166
:10E65000DF91CF911F910F91FF90EF90DF90CF90BE
:10E66000BF90AF9008950F93803611F1813630F44A
:10E67000843279F0853209F047C008C0823899F0B9
:10E68000833861F0813609F03FC02AC085E39EE6F9
:10E6900002C083EC90E70E94331536C00E94ED6DF6
:10E6A0008BE49AE1F8CF0E94ED6D8FE49FE3F3CF06
:10E6B0008091DF0E882389F481E08093DF0E8091C2
:10E6C000D50E9091D60EA091D70EB091D80E1816F7
:10E6D00019061A061B06C4F00BC01092DF0E14C0F8
:10E6E0008091DF0E813081F48091A80E882361F043
:10E6F00088EA9EE00E94A7726093D50E7093D60EB2
:10E700008093D70E9093D80E8091DD0E882371F000
:10E7100088EA9EE00E94A7726093D90E7093DA0E89
:10E720008093DB0E9093DC0E1092DD0E80E062E5AC
:10E7300041E00E94016E81E062E549E00E94016EC5
:10E7400083E062E542E00E94016E85E067E447E015
:10E750000E94016E81E30E94F06D8CE068E04FEE54
:10E760005CE10E94195E80918C0E882351F182E752
:10E7700068E04091B80E20E00E94F75C8CE060E118
:10E780004CE85EE022E004E10E94BA5D84E260E1D0
:10E790004AE324E00E94F75C80E360E14EE85EE03B
:10E7A00022E00E94BA5D88E460E14AE324E00E942E
:10E7B000F75C84E560E140E95EE022E00E94BA5D3A
:10E7C00007C08CE060E141E451E024E10E94EA5D91
:10E7D0008091DF0E8130D9F480918C0E8823B9F0BE
:10E7E0008CE060E249EE5CE10E94195E4091D90E36
:10E7F0005091DA0E8091D50E9091D60E481B590B90
:10E800008EE168E224E004E00E94F30E34C08CE064
:10E8100060E244EE5CE10E94195E80919A0E8823CA
:10E8200019F18CE068E24AE95EE022E004E10E942E
:10E83000BA5D84E268E24FE224E00E94F75C80E384
:10E8400068E24CE95EE022E00E94BA5D88E468E29A
:10E850004FE224E00E94F75C84E568E24EE95EE066
:10E8600022E00E94BA5D07C08CE068E241E451E01A
:10E8700024E10E94EA5D0F9108950E943373089588
:10E88000629FD001739FF001829FE00DF11D649F94
:10E89000E00DF11D929FF00D839FF00D749FF00D20
:10E8A000659FF00D9927729FB00DE11DF91F639FC1
:10E8B000B00DE11DF91FBD01CF0111240895991B71
:10E8C00079E004C0991F961708F0961B881F7A9567
:10E8D000C9F780950895AA1BBB1B51E107C0AA1F69
:10E8E000BB1FA617B70710F0A61BB70B881F991FF1
:10E8F0005A95A9F780959095BC01CD01089597FB95
:10E90000092E07260AD077FD04D0E5DF06D00020C7
:10E910001AF4709561957F4F0895F6F7909581955B
:10E920009F4F0895A1E21A2EAA1BBB1BFD010DC02B
:10E93000AA1FBB1FEE1FFF1FA217B307E407F507AF
:10E9400020F0A21BB30BE40BF50B661F771F881F8B
:10E95000991F1A9469F760957095809590959B0121
:10E96000AC01BD01CF01089597FB092E05260ED0FD
:10E9700057FD04D0D7DF0AD0001C38F450954095DD
:10E98000309521953F4F4F4F5F4F0895F6F7909583
:10E990008095709561957F4F8F4F9F4F0895EE0F33
:10E9A000FF1F0590F491E02D0994FB01DC0141501B
:10E9B000504048F005900D920020C9F701C01D920B
:10E9C00041505040E0F708956817790768F4FB015B
:10E9D000DC01E40FF51FA40FB51F02C002900E92D8
:10E9E00041505040D8F708950C940D75DC0101C0DA
:10E9F0006D9341505040E0F70895DC01CB01FC01DC
:10EA0000E199FECF06C0FFBBEEBBE09A31960DB296
:10EA10000D9241505040B8F70895FB01DC0102C04F
:10EA200001900D9241505040D8F70895F894FFCFCF
:10EA300086038703880389034AF0004DFF072204F9
:10EA40007C5E9CCE003264E2F1003264645A505A1B
:10EA50006450463C46649CEC1E465ADB0D230EDB9C
:10EA60000DFF0000AA05FF09FF0DFF135414AADBD8
:04EA70000D3F000056
:00000001FF
